 javaaccessbridge

 Timestamp is 9f7cb903 (reproducible build file hash)

 Preferred load address is 0000000180000000

 Start         Length     Name                   Class
 0001:00000000 000105b0H .text$mn                CODE
 0001:000105b0 00000036H .text$mn$00             CODE
 0001:000105e6 00000092H .text$x                 CODE
 0002:00000000 00000258H .idata$5                DATA
 0002:00000258 00000038H .00cfg                  DATA
 0002:00000290 00000008H .CRT$XCA                DATA
 0002:00000298 00000008H .CRT$XCZ                DATA
 0002:000002a0 00000008H .CRT$XIA                DATA
 0002:000002a8 00000008H .CRT$XIZ                DATA
 0002:000002b0 00000008H .CRT$XPA                DATA
 0002:000002b8 00000008H .CRT$XPZ                DATA
 0002:000002c0 00000008H .CRT$XTA                DATA
 0002:000002c8 00000008H .CRT$XTZ                DATA
 0002:000002d0 00000000H .gehcont$y              DATA
 0002:000002d0 00000000H .gfids$y                DATA
 0002:000002d0 0000f930H .rdata                  DATA
 0002:0000fc00 00000000H .rdata$CastGuardVftablesA DATA
 0002:0000fc00 00000000H .rdata$CastGuardVftablesC DATA
 0002:0000fc00 000001f4H .rdata$r                DATA
 0002:0000fdf4 00000064H .rdata$voltmd           DATA
 0002:0000fe58 00000310H .rdata$zzzdbg           DATA
 0002:00010168 00000008H .rtc$IAA                DATA
 0002:00010170 00000008H .rtc$IZZ                DATA
 0002:00010178 00000008H .rtc$TAA                DATA
 0002:00010180 00000008H .rtc$TZZ                DATA
 0002:00010188 00000480H .xdata                  DATA
 0002:00010608 000000f8H .xdata$x                DATA
 0002:00010700 00000a00H .edata                  DATA
 0002:00011100 000000b4H .idata$2                DATA
 0002:000111b4 00000014H .idata$3                DATA
 0002:000111c8 00000258H .idata$4                DATA
 0002:00011420 000005baH .idata$6                DATA
 0003:00000000 00000038H .data                   DATA
 0003:00000038 00000080H .data$r                 DATA
 0003:000000b8 00000028H .data$rs                DATA
 0003:000000e0 00000640H .bss                    DATA
 0004:00000000 000009e4H .pdata                  DATA
 0005:00000000 00000120H .rsrc$01                DATA
 0005:00000120 00000620H .rsrc$02                DATA

  Address         Publics by Value              Rva+Base               Lib:Object

 0000:00000000       __AbsoluteZero             0000000000000000     <absolute>
 0000:00000000       ___safe_se_handler_count   0000000000000000     <absolute>
 0000:00000000       ___safe_se_handler_table   0000000000000000     <absolute>
 0000:00000000       __arm64x_extra_rfe_table   0000000000000000     <absolute>
 0000:00000000       __arm64x_extra_rfe_table_size 0000000000000000     <absolute>
 0000:00000000       __arm64x_native_entrypoint 0000000000000000     <absolute>
 0000:00000000       __arm64x_redirection_metadata 0000000000000000     <absolute>
 0000:00000000       __arm64x_redirection_metadata_count 0000000000000000     <absolute>
 0000:00000000       __dynamic_value_reloc_table 0000000000000000     <absolute>
 0000:00000000       __enclave_config           0000000000000000     <absolute>
 0000:00000000       __guard_check_icall_a64n_fptr 0000000000000000     <absolute>
 0000:00000000       __guard_eh_cont_count      0000000000000000     <absolute>
 0000:00000000       __guard_eh_cont_table      0000000000000000     <absolute>
 0000:00000000       __guard_fids_count         0000000000000000     <absolute>
 0000:00000000       __guard_fids_table         0000000000000000     <absolute>
 0000:00000000       __guard_iat_count          0000000000000000     <absolute>
 0000:00000000       __guard_iat_table          0000000000000000     <absolute>
 0000:00000000       __guard_longjmp_count      0000000000000000     <absolute>
 0000:00000000       __guard_longjmp_table      0000000000000000     <absolute>
 0000:00000000       __hybrid_auxiliary_delayload_iat 0000000000000000     <absolute>
 0000:00000000       __hybrid_auxiliary_delayload_iat_copy 0000000000000000     <absolute>
 0000:00000000       __hybrid_auxiliary_iat     0000000000000000     <absolute>
 0000:00000000       __hybrid_auxiliary_iat_copy 0000000000000000     <absolute>
 0000:00000000       __hybrid_code_map          0000000000000000     <absolute>
 0000:00000000       __hybrid_code_map_count    0000000000000000     <absolute>
 0000:00000000       __hybrid_image_info_bitfield 0000000000000000     <absolute>
 0000:00000000       __x64_code_ranges_to_entry_points 0000000000000000     <absolute>
 0000:00000000       __x64_code_ranges_to_entry_points_count 0000000000000000     <absolute>
 0000:00000100       __guard_flags              0000000000000100     <absolute>
 0000:00000000       __ImageBase                0000000180000000     <linker-defined>
 0001:00000000       ??0AccessBridgeATInstance@@QEAA@PEAUHWND__@@0PEADPEAV0@@Z 0000000180001000 f   AccessBridgeATInstance.obj
 0001:00000040       ??1AccessBridgeATInstance@@QEAA@XZ 0000000180001040 f   AccessBridgeATInstance.obj
 0001:0000020c       ?findABATInstanceFromATHWND@AccessBridgeATInstance@@QEAAPEAV1@PEAUHWND__@@@Z 000000018000120c f   AccessBridgeATInstance.obj
 0001:0000022c       ?initiateIPC@AccessBridgeATInstance@@QEAA_JXZ 000000018000122c f   AccessBridgeATInstance.obj
 0001:00000324       ?sendAccessibilityEventPackage@AccessBridgeATInstance@@QEAA_JPEADHJ@Z 0000000180001324 f   AccessBridgeATInstance.obj
 0001:00000388       ?sendJavaEventPackage@AccessBridgeATInstance@@QEAA_JPEADHJ@Z 0000000180001388 f   AccessBridgeATInstance.obj
 0001:000003fc       PrintDebugString           00000001800013fc f   AccessBridgeDebug.obj
 0001:0000047c       __local_stdio_printf_options 000000018000147c f i AccessBridgeDebug.obj
 0001:00000484       finalizeFileLogger         0000000180001484 f   AccessBridgeDebug.obj
 0001:000004a8       fprintf                    00000001800014a8 f i AccessBridgeDebug.obj
 0001:000004ec       getTimeStamp               00000001800014ec f   AccessBridgeDebug.obj
 0001:00000524       initializeFileLogger       0000000180001524 f   AccessBridgeDebug.obj
 0001:00000634       printf                     0000000180001634 f i AccessBridgeDebug.obj
 0001:00000688       wPrintDebugString          0000000180001688 f   AccessBridgeDebug.obj
 0001:00000688       wPrintJavaDebugString      0000000180001688 f   AccessBridgeDebug.obj
 0001:00000708       ??0AccessBridgeJavaEntryPoints@@QEAA@PEAUJNIEnv_@@PEAV_jobject@@@Z 0000000180001708 f   AccessBridgeJavaEntryPoints.obj
 0001:00000730       ?BuildJavaEntryPoints@AccessBridgeJavaEntryPoints@@QEAAHXZ 0000000180001730 f   AccessBridgeJavaEntryPoints.obj
 0001:000026a8       ?CallBooleanMethod@JNIEnv_@@QEAAEPEAV_jobject@@PEAU_jmethodID@@ZZ 00000001800036a8 f i AccessBridgeJavaEntryPoints.obj
 0001:000026cc       ?CallCharMethod@JNIEnv_@@QEAAGPEAV_jobject@@PEAU_jmethodID@@ZZ 00000001800036cc f i AccessBridgeJavaEntryPoints.obj
 0001:000026f0       ?CallFloatMethod@JNIEnv_@@QEAAMPEAV_jobject@@PEAU_jmethodID@@ZZ 00000001800036f0 f i AccessBridgeJavaEntryPoints.obj
 0001:00002714       ?CallIntMethod@JNIEnv_@@QEAAJPEAV_jobject@@PEAU_jmethodID@@ZZ 0000000180003714 f i AccessBridgeJavaEntryPoints.obj
 0001:00002738       ?CallObjectMethod@JNIEnv_@@QEAAPEAV_jobject@@PEAV2@PEAU_jmethodID@@ZZ 0000000180003738 f i AccessBridgeJavaEntryPoints.obj
 0001:0000275c       ?CallVoidMethod@JNIEnv_@@QEAAXPEAV_jobject@@PEAU_jmethodID@@ZZ 000000018000375c f i AccessBridgeJavaEntryPoints.obj
 0001:00002780       ?activateAccessibleHyperlink@AccessBridgeJavaEntryPoints@@QEAAHPEAV_jobject@@0@Z 0000000180003780 f   AccessBridgeJavaEntryPoints.obj
 0001:00002828       ?addAccessibilityEventNotification@AccessBridgeJavaEntryPoints@@QEAAH_J@Z 0000000180003828 f   AccessBridgeJavaEntryPoints.obj
 0001:000028e0       ?addAccessibleSelectionFromContext@AccessBridgeJavaEntryPoints@@QEAAXPEAV_jobject@@H@Z 00000001800038e0 f   AccessBridgeJavaEntryPoints.obj
 0001:00002984       ?addJavaEventNotification@AccessBridgeJavaEntryPoints@@QEAAH_J@Z 0000000180003984 f   AccessBridgeJavaEntryPoints.obj
 0001:00002a1c       ?clearAccessibleSelectionFromContext@AccessBridgeJavaEntryPoints@@QEAAXPEAV_jobject@@@Z 0000000180003a1c f   AccessBridgeJavaEntryPoints.obj
 0001:00002ab0       ?doAccessibleActions@AccessBridgeJavaEntryPoints@@QEAAHPEAV_jobject@@PEAUAccessibleActionsToDoTag@@PEAJ@Z 0000000180003ab0 f   AccessBridgeJavaEntryPoints.obj
 0001:00002c34       ?getAccessibleActions@AccessBridgeJavaEntryPoints@@QEAAHPEAV_jobject@@PEAUAccessibleActionsTag@@@Z 0000000180003c34 f   AccessBridgeJavaEntryPoints.obj
 0001:00002ee4       ?getAccessibleChildFromContext@AccessBridgeJavaEntryPoints@@QEAAPEAV_jobject@@PEAV2@J@Z 0000000180003ee4 f   AccessBridgeJavaEntryPoints.obj
 0001:00002ff0       ?getAccessibleContextAt@AccessBridgeJavaEntryPoints@@QEAAPEAV_jobject@@JJPEAV2@@Z 0000000180003ff0 f   AccessBridgeJavaEntryPoints.obj
 0001:000030e4       ?getAccessibleContextFromHWND@AccessBridgeJavaEntryPoints@@QEAAPEAV_jobject@@J@Z 00000001800040e4 f   AccessBridgeJavaEntryPoints.obj
 0001:00003198       ?getAccessibleContextInfo@AccessBridgeJavaEntryPoints@@QEAAHPEAV_jobject@@PEAUAccessibleContextInfoTag@@@Z 0000000180004198 f   AccessBridgeJavaEntryPoints.obj
 0001:00004230       ?getAccessibleContextWithFocus@AccessBridgeJavaEntryPoints@@QEAAPEAV_jobject@@XZ 0000000180005230 f   AccessBridgeJavaEntryPoints.obj
 0001:00004308       ?getAccessibleHyperlink@AccessBridgeJavaEntryPoints@@QEAAHQEAV_jobject@@JPEAUAccessibleHyperlinkInfoTag@@@Z 0000000180005308 f   AccessBridgeJavaEntryPoints.obj
 0001:00004614       ?getAccessibleHyperlinkCount@AccessBridgeJavaEntryPoints@@QEAAJQEAV_jobject@@@Z 0000000180005614 f   AccessBridgeJavaEntryPoints.obj
 0001:000046ac       ?getAccessibleHypertext@AccessBridgeJavaEntryPoints@@QEAAHPEAV_jobject@@PEAUAccessibleHypertextInfoTag@@@Z 00000001800056ac f   AccessBridgeJavaEntryPoints.obj
 0001:00004afc       ?getAccessibleHypertextExt@AccessBridgeJavaEntryPoints@@QEAAHQEAV_jobject@@JPEAUAccessibleHypertextInfoTag@@@Z 0000000180005afc f   AccessBridgeJavaEntryPoints.obj
 0001:00004f70       ?getAccessibleHypertextLinkIndex@AccessBridgeJavaEntryPoints@@QEAAJQEAV_jobject@@J@Z 0000000180005f70 f   AccessBridgeJavaEntryPoints.obj
 0001:0000501c       ?getAccessibleIcons@AccessBridgeJavaEntryPoints@@QEAAHPEAV_jobject@@PEAUAccessibleIconsTag@@@Z 000000018000601c f   AccessBridgeJavaEntryPoints.obj
 0001:00005388       ?getAccessibleKeyBindings@AccessBridgeJavaEntryPoints@@QEAAHPEAV_jobject@@PEAUAccessibleKeyBindingsTag@@@Z 0000000180006388 f   AccessBridgeJavaEntryPoints.obj
 0001:00005514       ?getAccessibleParentFromContext@AccessBridgeJavaEntryPoints@@QEAAPEAV_jobject@@PEAV2@@Z 0000000180006514 f   AccessBridgeJavaEntryPoints.obj
 0001:0000561c       ?getAccessibleRelationSet@AccessBridgeJavaEntryPoints@@QEAAHPEAV_jobject@@PEAUAccessibleRelationSetInfoTag@@@Z 000000018000661c f   AccessBridgeJavaEntryPoints.obj
 0001:000059e0       ?getAccessibleSelectionCountFromContext@AccessBridgeJavaEntryPoints@@QEAAHPEAV_jobject@@@Z 00000001800069e0 f   AccessBridgeJavaEntryPoints.obj
 0001:00005a84       ?getAccessibleSelectionFromContext@AccessBridgeJavaEntryPoints@@QEAAPEAV_jobject@@PEAV2@H@Z 0000000180006a84 f   AccessBridgeJavaEntryPoints.obj
 0001:00005b90       ?getAccessibleTableCellInfo@AccessBridgeJavaEntryPoints@@QEAAHPEAV_jobject@@JJPEAUAccessibleTableCellInfoTag@@@Z 0000000180006b90 f   AccessBridgeJavaEntryPoints.obj
 0001:00005e30       ?getAccessibleTableColumn@AccessBridgeJavaEntryPoints@@QEAAJPEAV_jobject@@J@Z 0000000180006e30 f   AccessBridgeJavaEntryPoints.obj
 0001:00005ee8       ?getAccessibleTableColumnDescription@AccessBridgeJavaEntryPoints@@QEAAPEAV_jobject@@PEAV2@J@Z 0000000180006ee8 f   AccessBridgeJavaEntryPoints.obj
 0001:00005ff4       ?getAccessibleTableColumnHeader@AccessBridgeJavaEntryPoints@@QEAAHPEAV_jobject@@PEAUAccessibleTableInfoTag@@@Z 0000000180006ff4 f   AccessBridgeJavaEntryPoints.obj
 0001:000061a0       ?getAccessibleTableColumnSelectionCount@AccessBridgeJavaEntryPoints@@QEAAJPEAV_jobject@@@Z 00000001800071a0 f   AccessBridgeJavaEntryPoints.obj
 0001:00006244       ?getAccessibleTableColumnSelections@AccessBridgeJavaEntryPoints@@QEAAHPEAV_jobject@@JPEAJ@Z 0000000180007244 f   AccessBridgeJavaEntryPoints.obj
 0001:00006330       ?getAccessibleTableIndex@AccessBridgeJavaEntryPoints@@QEAAJPEAV_jobject@@JJ@Z 0000000180007330 f   AccessBridgeJavaEntryPoints.obj
 0001:000063f8       ?getAccessibleTableInfo@AccessBridgeJavaEntryPoints@@QEAAHPEAV_jobject@@PEAUAccessibleTableInfoTag@@@Z 00000001800073f8 f   AccessBridgeJavaEntryPoints.obj
 0001:00006658       ?getAccessibleTableRow@AccessBridgeJavaEntryPoints@@QEAAJPEAV_jobject@@J@Z 0000000180007658 f   AccessBridgeJavaEntryPoints.obj
 0001:00006710       ?getAccessibleTableRowDescription@AccessBridgeJavaEntryPoints@@QEAAPEAV_jobject@@PEAV2@J@Z 0000000180007710 f   AccessBridgeJavaEntryPoints.obj
 0001:0000681c       ?getAccessibleTableRowHeader@AccessBridgeJavaEntryPoints@@QEAAHPEAV_jobject@@PEAUAccessibleTableInfoTag@@@Z 000000018000781c f   AccessBridgeJavaEntryPoints.obj
 0001:000069c8       ?getAccessibleTableRowSelectionCount@AccessBridgeJavaEntryPoints@@QEAAJPEAV_jobject@@@Z 00000001800079c8 f   AccessBridgeJavaEntryPoints.obj
 0001:00006a6c       ?getAccessibleTableRowSelections@AccessBridgeJavaEntryPoints@@QEAAHPEAV_jobject@@JPEAJ@Z 0000000180007a6c f   AccessBridgeJavaEntryPoints.obj
 0001:00006b58       ?getAccessibleTextAttributes@AccessBridgeJavaEntryPoints@@QEAAHPEAV_jobject@@JPEAUAccessibleTextAttributesInfoTag@@@Z 0000000180007b58 f   AccessBridgeJavaEntryPoints.obj
 0001:00007ff0       ?getAccessibleTextInfo@AccessBridgeJavaEntryPoints@@QEAAHPEAV_jobject@@PEAUAccessibleTextInfoTag@@JJ@Z 0000000180008ff0 f   AccessBridgeJavaEntryPoints.obj
 0001:00008194       ?getAccessibleTextItems@AccessBridgeJavaEntryPoints@@QEAAHPEAV_jobject@@PEAUAccessibleTextItemsInfoTag@@J@Z 0000000180009194 f   AccessBridgeJavaEntryPoints.obj
 0001:000086f0       ?getAccessibleTextLineBounds@AccessBridgeJavaEntryPoints@@QEAAHPEAV_jobject@@JPEAJ1@Z 00000001800096f0 f   AccessBridgeJavaEntryPoints.obj
 0001:00008820       ?getAccessibleTextRange@AccessBridgeJavaEntryPoints@@QEAAHPEAV_jobject@@JJPEAGF@Z 0000000180009820 f   AccessBridgeJavaEntryPoints.obj
 0001:00008ad4       ?getAccessibleTextRect@AccessBridgeJavaEntryPoints@@QEAAHPEAV_jobject@@PEAUAccessibleTextRectInfoTag@@J@Z 0000000180009ad4 f   AccessBridgeJavaEntryPoints.obj
 0001:00008cb8       ?getAccessibleTextSelectionInfo@AccessBridgeJavaEntryPoints@@QEAAHPEAV_jobject@@PEAUAccessibleTextSelectionInfoTag@@@Z 0000000180009cb8 f   AccessBridgeJavaEntryPoints.obj
 0001:00008fb0       ?getActiveDescendent@AccessBridgeJavaEntryPoints@@QEAAPEAV_jobject@@QEAV2@@Z 0000000180009fb0 f   AccessBridgeJavaEntryPoints.obj
 0001:000090a0       ?getCaretLocation@AccessBridgeJavaEntryPoints@@QEAAHPEAV_jobject@@PEAUAccessibleTextRectInfoTag@@J@Z 000000018000a0a0 f   AccessBridgeJavaEntryPoints.obj
 0001:00009284       ?getCurrentAccessibleValueFromContext@AccessBridgeJavaEntryPoints@@QEAAHPEAV_jobject@@PEAGF@Z 000000018000a284 f   AccessBridgeJavaEntryPoints.obj
 0001:000094bc       ?getHWNDFromAccessibleContext@AccessBridgeJavaEntryPoints@@QEAAPEAUHWND__@@PEAV_jobject@@@Z 000000018000a4bc f   AccessBridgeJavaEntryPoints.obj
 0001:00009560       ?getMaximumAccessibleValueFromContext@AccessBridgeJavaEntryPoints@@QEAAHPEAV_jobject@@PEAGF@Z 000000018000a560 f   AccessBridgeJavaEntryPoints.obj
 0001:00009798       ?getMinimumAccessibleValueFromContext@AccessBridgeJavaEntryPoints@@QEAAHPEAV_jobject@@PEAGF@Z 000000018000a798 f   AccessBridgeJavaEntryPoints.obj
 0001:000099d0       ?getObjectDepth@AccessBridgeJavaEntryPoints@@QEAAJQEAV_jobject@@@Z 000000018000a9d0 f   AccessBridgeJavaEntryPoints.obj
 0001:00009a74       ?getParentWithRole@AccessBridgeJavaEntryPoints@@QEAAPEAV_jobject@@QEAV2@PEBG@Z 000000018000aa74 f   AccessBridgeJavaEntryPoints.obj
 0001:00009b9c       ?getParentWithRoleElseRoot@AccessBridgeJavaEntryPoints@@QEAAPEAV_jobject@@QEAV2@PEBG@Z 000000018000ab9c f   AccessBridgeJavaEntryPoints.obj
 0001:00009cc4       ?getTextAttributesInRange@AccessBridgeJavaEntryPoints@@QEAAHQEAV_jobject@@HHPEAUAccessibleTextAttributesInfoTag@@PEAF@Z 000000018000acc4 f   AccessBridgeJavaEntryPoints.obj
 0001:00009fbc       ?getTopLevelObject@AccessBridgeJavaEntryPoints@@QEAAPEAV_jobject@@QEAV2@@Z 000000018000afbc f   AccessBridgeJavaEntryPoints.obj
 0001:0000a0ac       ?getVersionInfo@AccessBridgeJavaEntryPoints@@QEAAHPEAUAccessBridgeVersionInfoTag@@@Z 000000018000b0ac f   AccessBridgeJavaEntryPoints.obj
 0001:0000a2f8       ?getVirtualAccessibleName@AccessBridgeJavaEntryPoints@@QEAAHQEAV_jobject@@PEAGH@Z 000000018000b2f8 f   AccessBridgeJavaEntryPoints.obj
 0001:0000a53c       ?getVisibleChildren@AccessBridgeJavaEntryPoints@@QEAAHQEAV_jobject@@HPEAUVisibleChildenInfoTag@@@Z 000000018000b53c f   AccessBridgeJavaEntryPoints.obj
 0001:0000a6c8       ?getVisibleChildrenCount@AccessBridgeJavaEntryPoints@@QEAAHQEAV_jobject@@@Z 000000018000b6c8 f   AccessBridgeJavaEntryPoints.obj
 0001:0000a758       ?isAccessibleChildSelectedFromContext@AccessBridgeJavaEntryPoints@@QEAAHPEAV_jobject@@H@Z 000000018000b758 f   AccessBridgeJavaEntryPoints.obj
 0001:0000a814       ?isAccessibleTableColumnSelected@AccessBridgeJavaEntryPoints@@QEAAHPEAV_jobject@@J@Z 000000018000b814 f   AccessBridgeJavaEntryPoints.obj
 0001:0000a8c8       ?isAccessibleTableRowSelected@AccessBridgeJavaEntryPoints@@QEAAHPEAV_jobject@@J@Z 000000018000b8c8 f   AccessBridgeJavaEntryPoints.obj
 0001:0000a97c       ?isJavaWindow@AccessBridgeJavaEntryPoints@@QEAAHJ@Z 000000018000b97c f   AccessBridgeJavaEntryPoints.obj
 0001:0000aa10       ?isSameObject@AccessBridgeJavaEntryPoints@@QEAAHPEAV_jobject@@0@Z 000000018000ba10 f   AccessBridgeJavaEntryPoints.obj
 0001:0000aaac       ?removeAccessibilityEventNotification@AccessBridgeJavaEntryPoints@@QEAAH_J@Z 000000018000baac f   AccessBridgeJavaEntryPoints.obj
 0001:0000ab44       ?removeAccessibleSelectionFromContext@AccessBridgeJavaEntryPoints@@QEAAXPEAV_jobject@@H@Z 000000018000bb44 f   AccessBridgeJavaEntryPoints.obj
 0001:0000abe8       ?removeJavaEventNotification@AccessBridgeJavaEntryPoints@@QEAAH_J@Z 000000018000bbe8 f   AccessBridgeJavaEntryPoints.obj
 0001:0000ac80       ?requestFocus@AccessBridgeJavaEntryPoints@@QEAAHQEAV_jobject@@@Z 000000018000bc80 f   AccessBridgeJavaEntryPoints.obj
 0001:0000ad24       ?selectAllAccessibleSelectionFromContext@AccessBridgeJavaEntryPoints@@QEAAXPEAV_jobject@@@Z 000000018000bd24 f   AccessBridgeJavaEntryPoints.obj
 0001:0000adb8       ?selectTextRange@AccessBridgeJavaEntryPoints@@QEAAHQEAV_jobject@@HH@Z 000000018000bdb8 f   AccessBridgeJavaEntryPoints.obj
 0001:0000ae80       ?setCaretPosition@AccessBridgeJavaEntryPoints@@QEAAHQEAV_jobject@@H@Z 000000018000be80 f   AccessBridgeJavaEntryPoints.obj
 0001:0000af34       ?setTextContents@AccessBridgeJavaEntryPoints@@QEAAHQEAV_jobject@@PEBG@Z 000000018000bf34 f   AccessBridgeJavaEntryPoints.obj
 0001:0000b01c       ?verifyAccessibleText@AccessBridgeJavaEntryPoints@@QEAAHPEAV_jobject@@@Z 000000018000c01c f   AccessBridgeJavaEntryPoints.obj
 0001:0000b140       ?initBroadcastMessageIDs@@YAHXZ 000000018000c140 f   AccessBridgeMessages.obj
 0001:0000b180       ??0JavaAccessBridge@@QEAA@PEAUHINSTANCE__@@@Z 000000018000c180 f   JavaAccessBridge.obj
 0001:0000b1ac       ??1JavaAccessBridge@@QEAA@XZ 000000018000c1ac f   JavaAccessBridge.obj
 0001:0000b27c       ?MemoryMappedFileCreated@JavaAccessBridge@@QEAA_JPEAUHWND__@@PEAD@Z 000000018000c27c f   JavaAccessBridge.obj
 0001:0000b320       ?WindowsATDestroyed@JavaAccessBridge@@QEAAXPEAUHWND__@@@Z 000000018000c320 f   JavaAccessBridge.obj
 0001:0000b3d4       ?addAccessibilityEventNotification@JavaAccessBridge@@QEAAX_JPEAUHWND__@@@Z 000000018000c3d4 f   JavaAccessBridge.obj
 0001:0000b47c       ?addJavaEventNotification@JavaAccessBridge@@QEAAX_JPEAUHWND__@@@Z 000000018000c47c f   JavaAccessBridge.obj
 0001:0000b524       ?fireCaretUpdate@JavaAccessBridge@@QEAAXPEAUJNIEnv_@@PEAV_jobject@@11@Z 000000018000c524 f   JavaAccessBridge.obj
 0001:0000b650       ?fireFocusGained@JavaAccessBridge@@QEAAXPEAUJNIEnv_@@PEAV_jobject@@11@Z 000000018000c650 f   JavaAccessBridge.obj
 0001:0000b77c       ?fireFocusLost@JavaAccessBridge@@QEAAXPEAUJNIEnv_@@PEAV_jobject@@11@Z 000000018000c77c f   JavaAccessBridge.obj
 0001:0000b8a8       ?fireMenuCanceled@JavaAccessBridge@@QEAAXPEAUJNIEnv_@@PEAV_jobject@@11@Z 000000018000c8a8 f   JavaAccessBridge.obj
 0001:0000b9d8       ?fireMenuDeselected@JavaAccessBridge@@QEAAXPEAUJNIEnv_@@PEAV_jobject@@11@Z 000000018000c9d8 f   JavaAccessBridge.obj
 0001:0000bb08       ?fireMenuSelected@JavaAccessBridge@@QEAAXPEAUJNIEnv_@@PEAV_jobject@@11@Z 000000018000cb08 f   JavaAccessBridge.obj
 0001:0000bc38       ?fireMouseClicked@JavaAccessBridge@@QEAAXPEAUJNIEnv_@@PEAV_jobject@@11@Z 000000018000cc38 f   JavaAccessBridge.obj
 0001:0000bd64       ?fireMouseEntered@JavaAccessBridge@@QEAAXPEAUJNIEnv_@@PEAV_jobject@@11@Z 000000018000cd64 f   JavaAccessBridge.obj
 0001:0000be90       ?fireMouseExited@JavaAccessBridge@@QEAAXPEAUJNIEnv_@@PEAV_jobject@@11@Z 000000018000ce90 f   JavaAccessBridge.obj
 0001:0000bfbc       ?fireMousePressed@JavaAccessBridge@@QEAAXPEAUJNIEnv_@@PEAV_jobject@@11@Z 000000018000cfbc f   JavaAccessBridge.obj
 0001:0000c0e8       ?fireMouseReleased@JavaAccessBridge@@QEAAXPEAUJNIEnv_@@PEAV_jobject@@11@Z 000000018000d0e8 f   JavaAccessBridge.obj
 0001:0000c218       ?firePopupMenuCanceled@JavaAccessBridge@@QEAAXPEAUJNIEnv_@@PEAV_jobject@@11@Z 000000018000d218 f   JavaAccessBridge.obj
 0001:0000c348       ?firePopupMenuWillBecomeInvisible@JavaAccessBridge@@QEAAXPEAUJNIEnv_@@PEAV_jobject@@11@Z 000000018000d348 f   JavaAccessBridge.obj
 0001:0000c478       ?firePopupMenuWillBecomeVisible@JavaAccessBridge@@QEAAXPEAUJNIEnv_@@PEAV_jobject@@11@Z 000000018000d478 f   JavaAccessBridge.obj
 0001:0000c5a8       ?firePropertyActiveDescendentChange@JavaAccessBridge@@QEAAXPEAUJNIEnv_@@PEAV_jobject@@1111@Z 000000018000d5a8 f   JavaAccessBridge.obj
 0001:0000c700       ?firePropertyCaretChange@JavaAccessBridge@@QEAAXPEAUJNIEnv_@@PEAV_jobject@@11JJ@Z 000000018000d700 f   JavaAccessBridge.obj
 0001:0000c820       ?firePropertyChildChange@JavaAccessBridge@@QEAAXPEAUJNIEnv_@@PEAV_jobject@@1111@Z 000000018000d820 f   JavaAccessBridge.obj
 0001:0000c978       ?firePropertyDescriptionChange@JavaAccessBridge@@QEAAXPEAUJNIEnv_@@PEAV_jobject@@11PEAV_jstring@@2@Z 000000018000d978 f   JavaAccessBridge.obj
 0001:0000cba4       ?firePropertyNameChange@JavaAccessBridge@@QEAAXPEAUJNIEnv_@@PEAV_jobject@@11PEAV_jstring@@2@Z 000000018000dba4 f   JavaAccessBridge.obj
 0001:0000cdd0       ?firePropertySelectionChange@JavaAccessBridge@@QEAAXPEAUJNIEnv_@@PEAV_jobject@@11@Z 000000018000ddd0 f   JavaAccessBridge.obj
 0001:0000cec4       ?firePropertyStateChange@JavaAccessBridge@@QEAAXPEAUJNIEnv_@@PEAV_jobject@@11PEAV_jstring@@2@Z 000000018000dec4 f   JavaAccessBridge.obj
 0001:0000d0f0       ?firePropertyTableModelChange@JavaAccessBridge@@QEAAXPEAUJNIEnv_@@PEAV_jobject@@11PEAV_jstring@@2@Z 000000018000e0f0 f   JavaAccessBridge.obj
 0001:0000d320       ?firePropertyTextChange@JavaAccessBridge@@QEAAXPEAUJNIEnv_@@PEAV_jobject@@11@Z 000000018000e320 f   JavaAccessBridge.obj
 0001:0000d414       ?firePropertyValueChange@JavaAccessBridge@@QEAAXPEAUJNIEnv_@@PEAV_jobject@@11PEAV_jstring@@2@Z 000000018000e414 f   JavaAccessBridge.obj
 0001:0000d640       ?firePropertyVisibleDataChange@JavaAccessBridge@@QEAAXPEAUJNIEnv_@@PEAV_jobject@@11@Z 000000018000e640 f   JavaAccessBridge.obj
 0001:0000d734       ?initWindow@JavaAccessBridge@@QEAAHXZ 000000018000e734 f   JavaAccessBridge.obj
 0001:0000d778       ?javaRun@JavaAccessBridge@@QEAAXPEAUJNIEnv_@@PEAV_jobject@@@Z 000000018000e778 f   JavaAccessBridge.obj
 0001:0000d924       ?javaShutdown@JavaAccessBridge@@QEAAXPEAUJNIEnv_@@PEAV_jobject@@@Z 000000018000e924 f   JavaAccessBridge.obj
 0001:0000d9dc       ?postHelloToWindowsDLLMsg@JavaAccessBridge@@QEAAXPEAUHWND__@@@Z 000000018000e9dc f   JavaAccessBridge.obj
 0001:0000da38       ?processPackage@JavaAccessBridge@@QEAA_JPEADH@Z 000000018000ea38 f   JavaAccessBridge.obj
 0001:0000ec20       ?receiveMemoryPackage@JavaAccessBridge@@QEAAHPEAUHWND__@@J@Z 000000018000fc20 f   JavaAccessBridge.obj
 0001:0000ecbc       ?releaseJavaObject@JavaAccessBridge@@QEAAXPEAV_jobject@@@Z 000000018000fcbc f   JavaAccessBridge.obj
 0001:0000ed24       ?removeAccessibilityEventNotification@JavaAccessBridge@@QEAAX_JPEAUHWND__@@@Z 000000018000fd24 f   JavaAccessBridge.obj
 0001:0000edcc       ?removeJavaEventNotification@JavaAccessBridge@@QEAAX_JPEAUHWND__@@@Z 000000018000fdcc f   JavaAccessBridge.obj
 0001:0000ee74       AccessBridgeDialogProc     000000018000fe74 f   JavaAccessBridge.obj
 0001:0000ef94       DllMain                    000000018000ff94 f   JavaAccessBridge.obj
 0001:0000f01c       Java_com_sun_java_accessibility_internal_AccessBridge_caretUpdate 000000018001001c f   JavaAccessBridge.obj
 0001:0000f040       Java_com_sun_java_accessibility_internal_AccessBridge_focusGained 0000000180010040 f   JavaAccessBridge.obj
 0001:0000f064       Java_com_sun_java_accessibility_internal_AccessBridge_focusLost 0000000180010064 f   JavaAccessBridge.obj
 0001:0000f088       Java_com_sun_java_accessibility_internal_AccessBridge_javaShutdown 0000000180010088 f   JavaAccessBridge.obj
 0001:0000f09c       Java_com_sun_java_accessibility_internal_AccessBridge_jawtGetComponentFromNativeWindowHandle 000000018001009c f   JavaAccessBridge.obj
 0001:0000f0e0       Java_com_sun_java_accessibility_internal_AccessBridge_jawtGetNativeWindowHandleFromComponent 00000001800100e0 f   JavaAccessBridge.obj
 0001:0000f148       Java_com_sun_java_accessibility_internal_AccessBridge_menuCanceled 0000000180010148 f   JavaAccessBridge.obj
 0001:0000f16c       Java_com_sun_java_accessibility_internal_AccessBridge_menuDeselected 000000018001016c f   JavaAccessBridge.obj
 0001:0000f190       Java_com_sun_java_accessibility_internal_AccessBridge_menuSelected 0000000180010190 f   JavaAccessBridge.obj
 0001:0000f1b4       Java_com_sun_java_accessibility_internal_AccessBridge_mouseClicked 00000001800101b4 f   JavaAccessBridge.obj
 0001:0000f1d8       Java_com_sun_java_accessibility_internal_AccessBridge_mouseEntered 00000001800101d8 f   JavaAccessBridge.obj
 0001:0000f1fc       Java_com_sun_java_accessibility_internal_AccessBridge_mouseExited 00000001800101fc f   JavaAccessBridge.obj
 0001:0000f220       Java_com_sun_java_accessibility_internal_AccessBridge_mousePressed 0000000180010220 f   JavaAccessBridge.obj
 0001:0000f244       Java_com_sun_java_accessibility_internal_AccessBridge_mouseReleased 0000000180010244 f   JavaAccessBridge.obj
 0001:0000f268       Java_com_sun_java_accessibility_internal_AccessBridge_popupMenuCanceled 0000000180010268 f   JavaAccessBridge.obj
 0001:0000f28c       Java_com_sun_java_accessibility_internal_AccessBridge_popupMenuWillBecomeInvisible 000000018001028c f   JavaAccessBridge.obj
 0001:0000f2b0       Java_com_sun_java_accessibility_internal_AccessBridge_popupMenuWillBecomeVisible 00000001800102b0 f   JavaAccessBridge.obj
 0001:0000f2d4       Java_com_sun_java_accessibility_internal_AccessBridge_propertyActiveDescendentChange 00000001800102d4 f   JavaAccessBridge.obj
 0001:0000f30c       Java_com_sun_java_accessibility_internal_AccessBridge_propertyCaretChange 000000018001030c f   JavaAccessBridge.obj
 0001:0000f340       Java_com_sun_java_accessibility_internal_AccessBridge_propertyChildChange 0000000180010340 f   JavaAccessBridge.obj
 0001:0000f378       Java_com_sun_java_accessibility_internal_AccessBridge_propertyDescriptionChange 0000000180010378 f   JavaAccessBridge.obj
 0001:0000f3b0       Java_com_sun_java_accessibility_internal_AccessBridge_propertyNameChange 00000001800103b0 f   JavaAccessBridge.obj
 0001:0000f3e8       Java_com_sun_java_accessibility_internal_AccessBridge_propertySelectionChange 00000001800103e8 f   JavaAccessBridge.obj
 0001:0000f40c       Java_com_sun_java_accessibility_internal_AccessBridge_propertyStateChange 000000018001040c f   JavaAccessBridge.obj
 0001:0000f444       Java_com_sun_java_accessibility_internal_AccessBridge_propertyTableModelChange 0000000180010444 f   JavaAccessBridge.obj
 0001:0000f47c       Java_com_sun_java_accessibility_internal_AccessBridge_propertyTextChange 000000018001047c f   JavaAccessBridge.obj
 0001:0000f4a0       Java_com_sun_java_accessibility_internal_AccessBridge_propertyValueChange 00000001800104a0 f   JavaAccessBridge.obj
 0001:0000f4d8       Java_com_sun_java_accessibility_internal_AccessBridge_propertyVisibleDataChange 00000001800104d8 f   JavaAccessBridge.obj
 0001:0000f4fc       Java_com_sun_java_accessibility_internal_AccessBridge_runDLL 00000001800104fc f   JavaAccessBridge.obj
 0001:0000f534       Java_com_sun_java_accessibility_internal_AccessBridge_sendDebugString 0000000180010534 f   JavaAccessBridge.obj
 0001:0000f5c8       ??2@YAPEAX_K@Z             00000001800105c8 f   MSVCRT:new_scalar.obj
 0001:0000f604       ??3@YAXPEAX_K@Z            0000000180010604 f   MSVCRT:delete_scalar_size.obj
 0001:0000f604       ??_V@YAXPEAX@Z             0000000180010604 f   MSVCRT:delete_array.obj
 0001:0000f60c       ??_U@YAPEAX_K@Z            000000018001060c f   MSVCRT:new_array.obj
 0001:0000f614       __GSHandlerCheck           0000000180010614 f   MSVCRT:gshandler.obj
 0001:0000f634       __GSHandlerCheckCommon     0000000180010634 f   MSVCRT:gshandler.obj
 0001:0000f6a0       __security_check_cookie    00000001800106a0 f   MSVCRT:amdsecgs.obj
 0001:0000f9e0       _DllMainCRTStartup         00000001800109e0 f   MSVCRT:dll_dllmain.obj
 0001:0000fa20       ??0bad_alloc@std@@QEAA@AEBV01@@Z 0000000180010a20 f i MSVCRT:throw_bad_alloc.obj
 0001:0000fa5c       ??0bad_alloc@std@@QEAA@XZ  0000000180010a5c f i MSVCRT:throw_bad_alloc.obj
 0001:0000fa7c       ??0bad_array_new_length@std@@QEAA@AEBV01@@Z 0000000180010a7c f i MSVCRT:throw_bad_alloc.obj
 0001:0000fab8       ??0bad_array_new_length@std@@QEAA@XZ 0000000180010ab8 f i MSVCRT:throw_bad_alloc.obj
 0001:0000fad8       ??0exception@std@@QEAA@AEBV01@@Z 0000000180010ad8 f i MSVCRT:throw_bad_alloc.obj
 0001:0000fb0c       ??1bad_alloc@std@@UEAA@XZ  0000000180010b0c f i MSVCRT:throw_bad_alloc.obj
 0001:0000fb0c       ??1bad_array_new_length@std@@UEAA@XZ 0000000180010b0c f i MSVCRT:throw_bad_alloc.obj
 0001:0000fb20       ??_Ebad_alloc@std@@UEAAPEAXI@Z 0000000180010b20 f i MSVCRT:throw_bad_alloc.obj
 0001:0000fb20       ??_Ebad_array_new_length@std@@UEAAPEAXI@Z 0000000180010b20 f i MSVCRT:throw_bad_alloc.obj
 0001:0000fb20       ??_Eexception@std@@UEAAPEAXI@Z 0000000180010b20 f i MSVCRT:throw_bad_alloc.obj
 0001:0000fb20       ??_Gbad_alloc@std@@UEAAPEAXI@Z 0000000180010b20 f i MSVCRT:throw_bad_alloc.obj
 0001:0000fb20       ??_Gbad_array_new_length@std@@UEAAPEAXI@Z 0000000180010b20 f i MSVCRT:throw_bad_alloc.obj
 0001:0000fb20       ??_Gexception@std@@UEAAPEAXI@Z 0000000180010b20 f i MSVCRT:throw_bad_alloc.obj
 0001:0000fb64       ?__scrt_throw_std_bad_alloc@@YAXXZ 0000000180010b64 f   MSVCRT:throw_bad_alloc.obj
 0001:0000fb84       ?__scrt_throw_std_bad_array_new_length@@YAXXZ 0000000180010b84 f   MSVCRT:throw_bad_alloc.obj
 0001:0000fba4       ?what@exception@std@@UEBAPEBDXZ 0000000180010ba4 f i MSVCRT:throw_bad_alloc.obj
 0001:0000fbb8       ??3@YAXPEAX@Z              0000000180010bb8 f   MSVCRT:delete_scalar.obj
 0001:0000fbc0       __raise_securityfailure    0000000180010bc0 f   MSVCRT:gs_report.obj
 0001:0000fbf4       __report_gsfailure         0000000180010bf4 f   MSVCRT:gs_report.obj
 0001:0000fd3c       __security_init_cookie     0000000180010d3c f   MSVCRT:gs_support.obj
 0001:0000fde8       ?__scrt_initialize_type_info@@YAXXZ 0000000180010de8 f   MSVCRT:tncleanup.obj
 0001:0000fdf8       ?__scrt_uninitialize_type_info@@YAXXZ 0000000180010df8 f   MSVCRT:tncleanup.obj
 0001:0000fe04       __local_stdio_scanf_options 0000000180010e04 f i MSVCRT:default_local_stdio_options.obj
 0001:0000fe0c       __scrt_initialize_default_local_stdio_options 0000000180010e0c f   MSVCRT:default_local_stdio_options.obj
 0001:0000fe28       __scrt_acquire_startup_lock 0000000180010e28 f   MSVCRT:utility.obj
 0001:0000fe64       __scrt_dllmain_after_initialize_c 0000000180010e64 f   MSVCRT:utility.obj
 0001:0000fe98       __scrt_dllmain_before_initialize_c 0000000180010e98 f   MSVCRT:utility.obj
 0001:0000feb0       __scrt_dllmain_crt_thread_attach 0000000180010eb0 f   MSVCRT:utility.obj
 0001:0000fed8       __scrt_dllmain_crt_thread_detach 0000000180010ed8 f   MSVCRT:utility.obj
 0001:0000fef0       __scrt_dllmain_exception_filter 0000000180010ef0 f   MSVCRT:utility.obj
 0001:0000ff50       __scrt_dllmain_uninitialize_c 0000000180010f50 f   MSVCRT:utility.obj
 0001:0000ff80       __scrt_dllmain_uninitialize_critical 0000000180010f80 f   MSVCRT:utility.obj
 0001:0000ff94       __scrt_initialize_crt      0000000180010f94 f   MSVCRT:utility.obj
 0001:0000ffe0       __scrt_initialize_onexit_tables 0000000180010fe0 f   MSVCRT:utility.obj
 0001:0001006c       __scrt_is_nonwritable_in_current_image 000000018001106c f   MSVCRT:utility.obj
 0001:00010104       __scrt_release_startup_lock 0000000180011104 f   MSVCRT:utility.obj
 0001:00010128       __scrt_uninitialize_crt    0000000180011128 f   MSVCRT:utility.obj
 0001:00010154       __scrt_get_dyn_tls_init_callback 0000000180011154 f   MSVCRT:dyn_tls_init.obj
 0001:0001015c       __crt_debugger_hook        000000018001115c f   MSVCRT:utility_desktop.obj
 0001:00010164       __scrt_fastfail            0000000180011164 f   MSVCRT:utility_desktop.obj
 0001:000102b0       _RTC_Initialize            00000001800112b0 f   MSVCRT:initsect.obj
 0001:000102ec       _RTC_Terminate             00000001800112ec f   MSVCRT:initsect.obj
 0001:00010328       _guard_check_icall_nop     0000000180011328 f i MSVCRT:guard_support.obj
 0001:0001032c       ??_Etype_info@@UEAAPEAXI@Z 000000018001132c f i MSVCRT:std_type_info_static.obj
 0001:0001032c       ??_Gtype_info@@UEAAPEAXI@Z 000000018001132c f i MSVCRT:std_type_info_static.obj
 0001:00010358       __isa_available_init       0000000180011358 f   MSVCRT:cpu_disp.obj
 0001:00010504       _get_startup_argv_mode     0000000180011504 f   MSVCRT:argv_mode.obj
 0001:0001050c       __scrt_is_ucrt_dll_in_use  000000018001150c f   MSVCRT:ucrt_detection.obj
 0001:00010520       memcpy                     0000000180011520 f   vcruntime:VCRUNTIME140.dll
 0001:00010526       memset                     0000000180011526 f   vcruntime:VCRUNTIME140.dll
 0001:0001052c       __C_specific_handler       000000018001152c f   vcruntime:VCRUNTIME140.dll
 0001:00010532       __std_exception_copy       0000000180011532 f   vcruntime:VCRUNTIME140.dll
 0001:00010538       __std_exception_destroy    0000000180011538 f   vcruntime:VCRUNTIME140.dll
 0001:0001053e       _CxxThrowException         000000018001153e f   vcruntime:VCRUNTIME140.dll
 0001:00010544       __std_type_info_destroy_list 0000000180011544 f   vcruntime:VCRUNTIME140.dll
 0001:0001054a       strcmp                     000000018001154a f   ucrt:api-ms-win-crt-string-l1-1-0.dll
 0001:00010550       strcpy                     0000000180011550 f   ucrt:api-ms-win-crt-string-l1-1-0.dll
 0001:00010556       strlen                     0000000180011556 f   ucrt:api-ms-win-crt-string-l1-1-0.dll
 0001:0001055c       _callnewh                  000000018001155c f   ucrt:api-ms-win-crt-heap-l1-1-0.dll
 0001:00010562       malloc                     0000000180011562 f   ucrt:api-ms-win-crt-heap-l1-1-0.dll
 0001:00010568       _initterm                  0000000180011568 f   ucrt:api-ms-win-crt-runtime-l1-1-0.dll
 0001:0001056e       _initterm_e                000000018001156e f   ucrt:api-ms-win-crt-runtime-l1-1-0.dll
 0001:00010574       free                       0000000180011574 f   ucrt:api-ms-win-crt-heap-l1-1-0.dll
 0001:0001057a       _seh_filter_dll            000000018001157a f   ucrt:api-ms-win-crt-runtime-l1-1-0.dll
 0001:00010580       _configure_narrow_argv     0000000180011580 f   ucrt:api-ms-win-crt-runtime-l1-1-0.dll
 0001:00010586       _initialize_narrow_environment 0000000180011586 f   ucrt:api-ms-win-crt-runtime-l1-1-0.dll
 0001:0001058c       _initialize_onexit_table   000000018001158c f   ucrt:api-ms-win-crt-runtime-l1-1-0.dll
 0001:00010592       _execute_onexit_table      0000000180011592 f   ucrt:api-ms-win-crt-runtime-l1-1-0.dll
 0001:00010598       _cexit                     0000000180011598 f   ucrt:api-ms-win-crt-runtime-l1-1-0.dll
 0001:000105a0       __acrt_initialize          00000001800115a0 f   MSVCRT:ucrt_stubs.obj
 0001:000105a0       __acrt_thread_attach       00000001800115a0 f   MSVCRT:ucrt_stubs.obj
 0001:000105a0       __acrt_thread_detach       00000001800115a0 f   MSVCRT:ucrt_stubs.obj
 0001:000105a0       __acrt_uninitialize        00000001800115a0 f   MSVCRT:ucrt_stubs.obj
 0001:000105a0       __acrt_uninitialize_critical 00000001800115a0 f   MSVCRT:ucrt_stubs.obj
 0001:000105a0       __scrt_stub_for_acrt_initialize 00000001800115a0 f   MSVCRT:ucrt_stubs.obj
 0001:000105a0       __scrt_stub_for_acrt_thread_attach 00000001800115a0 f   MSVCRT:ucrt_stubs.obj
 0001:000105a0       __scrt_stub_for_acrt_thread_detach 00000001800115a0 f   MSVCRT:ucrt_stubs.obj
 0001:000105a0       __scrt_stub_for_acrt_uninitialize 00000001800115a0 f   MSVCRT:ucrt_stubs.obj
 0001:000105a0       __scrt_stub_for_acrt_uninitialize_critical 00000001800115a0 f   MSVCRT:ucrt_stubs.obj
 0001:000105a0       __vcrt_initialize          00000001800115a0 f   MSVCRT:ucrt_stubs.obj
 0001:000105a0       __vcrt_thread_attach       00000001800115a0 f   MSVCRT:ucrt_stubs.obj
 0001:000105a0       __vcrt_thread_detach       00000001800115a0 f   MSVCRT:ucrt_stubs.obj
 0001:000105a0       __vcrt_uninitialize        00000001800115a0 f   MSVCRT:ucrt_stubs.obj
 0001:000105a0       __vcrt_uninitialize_critical 00000001800115a0 f   MSVCRT:ucrt_stubs.obj
 0001:000105a4       __scrt_stub_for_is_c_termination_complete 00000001800115a4 f   MSVCRT:ucrt_stubs.obj
 0001:000105a4       _is_c_termination_complete 00000001800115a4 f   MSVCRT:ucrt_stubs.obj
 0001:000105c0       _guard_dispatch_icall_nop  00000001800115c0 f   MSVCRT:guard_dispatch.obj
 0001:000105e0       _guard_xfg_dispatch_icall_nop 00000001800115e0 f   MSVCRT:guard_xfg_dispatch.obj
 0002:00000000       __imp_CloseHandle          0000000180012000     kernel32:KERNEL32.dll
 0002:00000008       __imp_GetLastError         0000000180012008     kernel32:KERNEL32.dll
 0002:00000010       __imp_MapViewOfFile        0000000180012010     kernel32:KERNEL32.dll
 0002:00000018       __imp_UnmapViewOfFile      0000000180012018     kernel32:KERNEL32.dll
 0002:00000020       __imp_OpenFileMappingA     0000000180012020     kernel32:KERNEL32.dll
 0002:00000028       __imp_GetSystemTimeAsFileTime 0000000180012028     kernel32:KERNEL32.dll
 0002:00000030       __imp_InitializeCriticalSection 0000000180012030     kernel32:KERNEL32.dll
 0002:00000038       __imp_EnterCriticalSection 0000000180012038     kernel32:KERNEL32.dll
 0002:00000040       __imp_LeaveCriticalSection 0000000180012040     kernel32:KERNEL32.dll
 0002:00000048       __imp_DeleteCriticalSection 0000000180012048     kernel32:KERNEL32.dll
 0002:00000050       __imp_Sleep                0000000180012050     kernel32:KERNEL32.dll
 0002:00000058       __imp_IsDebuggerPresent    0000000180012058     kernel32:KERNEL32.dll
 0002:00000060       __imp_InitializeSListHead  0000000180012060     kernel32:KERNEL32.dll
 0002:00000068       __imp_GetCurrentThreadId   0000000180012068     kernel32:KERNEL32.dll
 0002:00000070       __imp_GetCurrentProcessId  0000000180012070     kernel32:KERNEL32.dll
 0002:00000078       __imp_QueryPerformanceCounter 0000000180012078     kernel32:KERNEL32.dll
 0002:00000080       __imp_IsProcessorFeaturePresent 0000000180012080     kernel32:KERNEL32.dll
 0002:00000088       __imp_TerminateProcess     0000000180012088     kernel32:KERNEL32.dll
 0002:00000090       __imp_GetCurrentProcess    0000000180012090     kernel32:KERNEL32.dll
 0002:00000098       __imp_SetUnhandledExceptionFilter 0000000180012098     kernel32:KERNEL32.dll
 0002:000000a0       __imp_UnhandledExceptionFilter 00000001800120a0     kernel32:KERNEL32.dll
 0002:000000a8       __imp_RtlVirtualUnwind     00000001800120a8     kernel32:KERNEL32.dll
 0002:000000b0       __imp_RtlLookupFunctionEntry 00000001800120b0     kernel32:KERNEL32.dll
 0002:000000b8       __imp_RtlCaptureContext    00000001800120b8     kernel32:KERNEL32.dll
 0002:000000c0       \177KERNEL32_NULL_THUNK_DATA 00000001800120c0     kernel32:KERNEL32.dll
 0002:000000c8       __imp_DispatchMessageA     00000001800120c8     user32:USER32.dll
 0002:000000d0       __imp_TranslateMessage     00000001800120d0     user32:USER32.dll
 0002:000000d8       __imp_RegisterWindowMessageA 00000001800120d8     user32:USER32.dll
 0002:000000e0       __imp_PostQuitMessage      00000001800120e0     user32:USER32.dll
 0002:000000e8       __imp_PostThreadMessageA   00000001800120e8     user32:USER32.dll
 0002:000000f0       __imp_SendMessageA         00000001800120f0     user32:USER32.dll
 0002:000000f8       __imp_GetMessageA          00000001800120f8     user32:USER32.dll
 0002:00000100       __imp_CreateDialogParamA   0000000180012100     user32:USER32.dll
 0002:00000108       __imp_PostMessageA         0000000180012108     user32:USER32.dll
 0002:00000110       \177USER32_NULL_THUNK_DATA 0000000180012110     user32:USER32.dll
 0002:00000118       __imp___std_type_info_destroy_list 0000000180012118     vcruntime:VCRUNTIME140.dll
 0002:00000120       __imp__CxxThrowException   0000000180012120     vcruntime:VCRUNTIME140.dll
 0002:00000128       __imp_memset               0000000180012128     vcruntime:VCRUNTIME140.dll
 0002:00000130       __imp___std_exception_destroy 0000000180012130     vcruntime:VCRUNTIME140.dll
 0002:00000138       __imp___std_exception_copy 0000000180012138     vcruntime:VCRUNTIME140.dll
 0002:00000140       __imp_memcpy               0000000180012140     vcruntime:VCRUNTIME140.dll
 0002:00000148       __imp___C_specific_handler 0000000180012148     vcruntime:VCRUNTIME140.dll
 0002:00000150       \177VCRUNTIME140_NULL_THUNK_DATA 0000000180012150     vcruntime:VCRUNTIME140.dll
 0002:00000158       __imp_getenv               0000000180012158     ucrt:api-ms-win-crt-environment-l1-1-0.dll
 0002:00000160       \177api-ms-win-crt-environment-l1-1-0_NULL_THUNK_DATA 0000000180012160     ucrt:api-ms-win-crt-environment-l1-1-0.dll
 0002:00000168       __imp_malloc               0000000180012168     ucrt:api-ms-win-crt-heap-l1-1-0.dll
 0002:00000170       __imp_free                 0000000180012170     ucrt:api-ms-win-crt-heap-l1-1-0.dll
 0002:00000178       __imp__callnewh            0000000180012178     ucrt:api-ms-win-crt-heap-l1-1-0.dll
 0002:00000180       \177api-ms-win-crt-heap-l1-1-0_NULL_THUNK_DATA 0000000180012180     ucrt:api-ms-win-crt-heap-l1-1-0.dll
 0002:00000188       __imp__initterm_e          0000000180012188     ucrt:api-ms-win-crt-runtime-l1-1-0.dll
 0002:00000190       __imp__seh_filter_dll      0000000180012190     ucrt:api-ms-win-crt-runtime-l1-1-0.dll
 0002:00000198       __imp__configure_narrow_argv 0000000180012198     ucrt:api-ms-win-crt-runtime-l1-1-0.dll
 0002:000001a0       __imp__beginthreadex       00000001800121a0     ucrt:api-ms-win-crt-runtime-l1-1-0.dll
 0002:000001a8       __imp__initterm            00000001800121a8     ucrt:api-ms-win-crt-runtime-l1-1-0.dll
 0002:000001b0       __imp__execute_onexit_table 00000001800121b0     ucrt:api-ms-win-crt-runtime-l1-1-0.dll
 0002:000001b8       __imp__cexit               00000001800121b8     ucrt:api-ms-win-crt-runtime-l1-1-0.dll
 0002:000001c0       __imp__initialize_onexit_table 00000001800121c0     ucrt:api-ms-win-crt-runtime-l1-1-0.dll
 0002:000001c8       __imp__initialize_narrow_environment 00000001800121c8     ucrt:api-ms-win-crt-runtime-l1-1-0.dll
 0002:000001d0       \177api-ms-win-crt-runtime-l1-1-0_NULL_THUNK_DATA 00000001800121d0     ucrt:api-ms-win-crt-runtime-l1-1-0.dll
 0002:000001d8       __imp_fopen                00000001800121d8     ucrt:api-ms-win-crt-stdio-l1-1-0.dll
 0002:000001e0       __imp___acrt_iob_func      00000001800121e0     ucrt:api-ms-win-crt-stdio-l1-1-0.dll
 0002:000001e8       __imp_fclose               00000001800121e8     ucrt:api-ms-win-crt-stdio-l1-1-0.dll
 0002:000001f0       __imp___stdio_common_vfwprintf 00000001800121f0     ucrt:api-ms-win-crt-stdio-l1-1-0.dll
 0002:000001f8       __imp___stdio_common_vfprintf 00000001800121f8     ucrt:api-ms-win-crt-stdio-l1-1-0.dll
 0002:00000200       \177api-ms-win-crt-stdio-l1-1-0_NULL_THUNK_DATA 0000000180012200     ucrt:api-ms-win-crt-stdio-l1-1-0.dll
 0002:00000208       __imp_wcscmp               0000000180012208     ucrt:api-ms-win-crt-string-l1-1-0.dll
 0002:00000210       __imp_strcmp               0000000180012210     ucrt:api-ms-win-crt-string-l1-1-0.dll
 0002:00000218       __imp_strcpy               0000000180012218     ucrt:api-ms-win-crt-string-l1-1-0.dll
 0002:00000220       __imp_wcsncpy              0000000180012220     ucrt:api-ms-win-crt-string-l1-1-0.dll
 0002:00000228       __imp_strncpy              0000000180012228     ucrt:api-ms-win-crt-string-l1-1-0.dll
 0002:00000230       __imp_strlen               0000000180012230     ucrt:api-ms-win-crt-string-l1-1-0.dll
 0002:00000238       __imp_wcslen               0000000180012238     ucrt:api-ms-win-crt-string-l1-1-0.dll
 0002:00000240       \177api-ms-win-crt-string-l1-1-0_NULL_THUNK_DATA 0000000180012240     ucrt:api-ms-win-crt-string-l1-1-0.dll
 0002:00000248       __imp_JAWT_GetAWT          0000000180012248     jawt:jawt.dll
 0002:00000250       \177jawt_NULL_THUNK_DATA   0000000180012250     jawt:jawt.dll
 0002:00000258       __guard_check_icall_fptr   0000000180012258     MSVCRT:guard_support.obj
 0002:00000260       __guard_xfg_check_icall_fptr 0000000180012260     MSVCRT:guard_support.obj
 0002:00000268       __guard_dispatch_icall_fptr 0000000180012268     MSVCRT:guard_support.obj
 0002:00000270       __guard_xfg_dispatch_icall_fptr 0000000180012270     MSVCRT:guard_support.obj
 0002:00000278       __guard_xfg_table_dispatch_icall_fptr 0000000180012278     MSVCRT:guard_support.obj
 0002:00000280       __castguard_check_failure_os_handled_fptr 0000000180012280     MSVCRT:guard_support.obj
 0002:00000288       __guard_memcpy_fptr        0000000180012288     vcruntime:softmemtag.obj
 0002:00000290       __xc_a                     0000000180012290     MSVCRT:initializers.obj
 0002:00000298       __xc_z                     0000000180012298     MSVCRT:initializers.obj
 0002:000002a0       __xi_a                     00000001800122a0     MSVCRT:initializers.obj
 0002:000002a8       __xi_z                     00000001800122a8     MSVCRT:initializers.obj
 0002:000002b0       __xp_a                     00000001800122b0     MSVCRT:initializers.obj
 0002:000002b8       __xp_z                     00000001800122b8     MSVCRT:initializers.obj
 0002:000002c0       __xt_a                     00000001800122c0     MSVCRT:initializers.obj
 0002:000002c8       __xt_z                     00000001800122c8     MSVCRT:initializers.obj
 0002:000002d0       ??_C@_0DL@PNCLIPJM@?$FLINFO?$FN?3?5in?5AccessBridgeATInstan@ 00000001800122d0     AccessBridgeATInstance.obj
 0002:00000310       ??_C@_0DA@ILNDDPNA@?$FLINFO?$FN?3?5?5?5unmapping?5memoryMappe@ 0000000180012310     AccessBridgeATInstance.obj
 0002:00000340       ??_C@_0DJ@FCAPEKK@?$FLINFO?$FN?3?5?5?5closing?5memoryMappedF@ 0000000180012340     AccessBridgeATInstance.obj
 0002:00000380       ??_C@_0DB@BBBKEEOJ@?$FLINFO?$FN?3?5In?5AccessBridgeATInstan@ 0000000180012380     AccessBridgeATInstance.obj
 0002:000003b8       ??_C@_0DJ@HCNGCGLH@?$FLERROR?$FN?3?5?5?5Failed?5to?5CreateFile@ 00000001800123b8     AccessBridgeATInstance.obj
 0002:000003f8       ??_C@_0DC@INNGAKAO@?$FLINFO?$FN?3?5?5?5CreateFileMapping?5wor@ 00000001800123f8     AccessBridgeATInstance.obj
 0002:00000430       ??_C@_0DF@EKLGABNF@?$FLERROR?$FN?3?5?5?5Failed?5to?5MapViewOfF@ 0000000180012430     AccessBridgeATInstance.obj
 0002:00000468       ??_C@_0CK@LMLFEIHL@?$FLINFO?$FN?3?5?5?5MapViewOfFile?5worked?5@ 0000000180012468     AccessBridgeATInstance.obj
 0002:00000494       ??_C@_03DJNNCAJF@OK?$DP@   0000000180012494     AccessBridgeATInstance.obj
 0002:00000498       ??_C@_0DL@FPNEIEFH@?$FLERROR?$FN?3?5?5?5JavaVM?5failed?5to?5wri@ 0000000180012498     AccessBridgeATInstance.obj
 0002:000004d8       ??_C@_0CN@CCHCHAPN@?$FLINFO?$FN?3?5?5?5JavaVM?5successfully?5w@ 00000001800124d8     AccessBridgeATInstance.obj
 0002:00000508       ??_C@_03ONJMBPEK@OK?$CB@   0000000180012508     AccessBridgeATInstance.obj
 0002:00000510       ??_C@_0EE@MNPDBEBN@?$FLINFO?$FN?3?5AccessBridgeATInstance?3@ 0000000180012510     AccessBridgeATInstance.obj
 0002:00000560       ??_C@_0FI@KACFLKHC@?$FLINFO?$FN?3?5AccessBridgeATInstance?3@ 0000000180012560     AccessBridgeATInstance.obj
 0002:000005c0       ??_C@_0EN@DDCKACNO@?$FLINFO?$FN?3?5AccessBridgeATInstance?3@ 00000001800125c0     AccessBridgeATInstance.obj
 0002:00000610       ??_C@_0BJ@FKCDJFDK@JAVA_ACCESSBRIDGE_LOGDIR@ 0000000180012610     AccessBridgeDebug.obj
 0002:0000062c       ??_C@_04FPOLKAEB@?4log@    000000018001262c     AccessBridgeDebug.obj
 0002:00000634       ??_C@_01NOFIACDB@w@        0000000180012634     AccessBridgeDebug.obj
 0002:00000638       ??_C@_04EINJHBMM@?6?$CFs?6@ 0000000180012638     AccessBridgeDebug.obj
 0002:00000640       ??_C@_0BH@PPBGFLKL@Could?5not?5open?5file?5?$CFs@ 0000000180012640     AccessBridgeDebug.obj
 0002:00000658       ??_C@_07IBOBEFLP@?$FL?$CFllu?$FN?5@ 0000000180012658     AccessBridgeDebug.obj
 0002:00000660       ??_C@_02PCIJFNDE@?$AN?6@   0000000180012660     AccessBridgeDebug.obj
 0002:00000668       ??_C@_0DD@HABIDLLD@?$FLINFO?$FN?3?5AccessBridgeJavaEntryPo@ 0000000180012668     AccessBridgeJavaEntryPoints.obj
 0002:000006a0       ??_C@_0CI@FJHGEAOO@?$FLINFO?$FN?3?5Calling?5BuildJavaEntryP@ 00000001800126a0     AccessBridgeJavaEntryPoints.obj
 0002:000006c8       ??_C@_0DB@PHGNIPBB@com?1sun?1java?1accessibility?1inte@ 00000001800126c8     AccessBridgeJavaEntryPoints.obj
 0002:00000700       ??_C@_0CP@OJHOIDNH@?$FLERROR?$FN?3?5?5FindClass?$CI?$CFs?$CJ?5failed?$CB@ 0000000180012700     AccessBridgeJavaEntryPoints.obj
 0002:00000730       ??_C@_0DE@FJPDGHPE@?$FLERROR?$FN?3?5FindClass?$CI?$CFs?$CJ?5failed?$CB?5@ 0000000180012730     AccessBridgeJavaEntryPoints.obj
 0002:00000768       ??_C@_0BG@JLFLBLJI@?$CILjava?1lang?1Object?$DL?$CJV@ 0000000180012768     AccessBridgeJavaEntryPoints.obj
 0002:00000780       ??_C@_0BD@PAIEAHIF@decrementReference@ 0000000180012780     AccessBridgeJavaEntryPoints.obj
 0002:00000798       ??_C@_0DP@BBIEPKKN@?$FLERROR?$FN?3?5GetMethodID?$CI?$CFs?$CJ?5failed@ 0000000180012798     AccessBridgeJavaEntryPoints.obj
 0002:000007d8       ??_C@_0BF@FOHFOJOB@?$CI?$CJLjava?1lang?1String?$DL@ 00000001800127d8     AccessBridgeJavaEntryPoints.obj
 0002:000007f0       ??_C@_0BH@KKNMIJGK@getJavaVersionProperty@ 00000001800127f0     AccessBridgeJavaEntryPoints.obj
 0002:00000808       ??_C@_04FJLILDCB@?$CII?$CJZ@ 0000000180012808     AccessBridgeJavaEntryPoints.obj
 0002:00000810       ??_C@_0N@MHDJENGP@isJavaWindow@ 0000000180012810     AccessBridgeJavaEntryPoints.obj
 0002:00000820       ??_C@_0CL@DDDHKJEI@?$CII?$CJLjavax?1accessibility?1Accessi@ 0000000180012820     AccessBridgeJavaEntryPoints.obj
 0002:00000850       ??_C@_0CB@JPFPCEPL@getContextFromNativeWindowHandl@ 0000000180012850     AccessBridgeJavaEntryPoints.obj
 0002:00000878       ??_C@_0CL@LNFAHLDN@?$CILjavax?1accessibility?1Accessibl@ 0000000180012878     AccessBridgeJavaEntryPoints.obj
 0002:000008a8       ??_C@_0CB@OGDNEJKI@getNativeWindowHandleFromContex@ 00000001800128a8     AccessBridgeJavaEntryPoints.obj
 0002:000008d0       ??_C@_0FB@EAOFMHCM@?$CILjavax?1accessibility?1Accessibl@ 00000001800128d0     AccessBridgeJavaEntryPoints.obj
 0002:00000928       ??_C@_0BP@OKMFCEDC@getAccessibleParentFromContext@ 0000000180012928     AccessBridgeJavaEntryPoints.obj
 0002:00000948       ??_C@_0DN@EHCPLCMJ@?$CILjavax?1accessibility?1Accessibl@ 0000000180012948     AccessBridgeJavaEntryPoints.obj
 0002:00000988       ??_C@_0BA@NNDOMDNC@setTextContents@ 0000000180012988     AccessBridgeJavaEntryPoints.obj
 0002:000009a0       ??_C@_0GD@DBHMDOGO@?$CILjavax?1accessibility?1Accessibl@ 00000001800129a0     AccessBridgeJavaEntryPoints.obj
 0002:00000a08       ??_C@_0BC@EHMJEOIE@getParentWithRole@ 0000000180012a08     AccessBridgeJavaEntryPoints.obj
 0002:00000a20       ??_C@_0BC@CBIPDOMM@getTopLevelObject@ 0000000180012a20     AccessBridgeJavaEntryPoints.obj
 0002:00000a38       ??_C@_0BK@KAMHKCND@getParentWithRoleElseRoot@ 0000000180012a38     AccessBridgeJavaEntryPoints.obj
 0002:00000a58       ??_C@_0P@POFHEAF@getObjectDepth@ 0000000180012a58     AccessBridgeJavaEntryPoints.obj
 0002:00000a68       ??_C@_0BE@CDLLPKAM@getActiveDescendent@ 0000000180012a68     AccessBridgeJavaEntryPoints.obj
 0002:00000a80       ??_C@_0FD@CINPJKCJ@?$CIIILjavax?1accessibility?1Accessi@ 0000000180012a80     AccessBridgeJavaEntryPoints.obj
 0002:00000ad8       ??_C@_0BH@BIEKBJIN@getAccessibleContextAt@ 0000000180012ad8     AccessBridgeJavaEntryPoints.obj
 0002:00000af0       ??_C@_0CK@DOBCJGDO@?$CI?$CJLjavax?1accessibility?1Accessib@ 0000000180012af0     AccessBridgeJavaEntryPoints.obj
 0002:00000b20       ??_C@_0BO@BAFCPPBG@getAccessibleContextWithFocus@ 0000000180012b20     AccessBridgeJavaEntryPoints.obj
 0002:00000b40       ??_C@_0DM@JMIIJMDP@?$CILjavax?1accessibility?1Accessibl@ 0000000180012b40     AccessBridgeJavaEntryPoints.obj
 0002:00000b80       ??_C@_0BN@DPBDCOIO@getAccessibleNameFromContext@ 0000000180012b80     AccessBridgeJavaEntryPoints.obj
 0002:00000ba0       ??_C@_0CE@IOFJICIE@getAccessibleDescriptionFromCon@ 0000000180012ba0     AccessBridgeJavaEntryPoints.obj
 0002:00000bc8       ??_C@_0CD@DDGCACMP@getAccessibleRoleStringFromCont@ 0000000180012bc8     AccessBridgeJavaEntryPoints.obj
 0002:00000bf0       ??_C@_0CJ@OOFFKIOD@getAccessibleRoleStringFromCont@ 0000000180012bf0     AccessBridgeJavaEntryPoints.obj
 0002:00000c20       ??_C@_0CF@JIKEBCCK@getAccessibleStatesStringFromCo@ 0000000180012c20     AccessBridgeJavaEntryPoints.obj
 0002:00000c48       ??_C@_0CL@EODHLGAL@getAccessibleStatesStringFromCo@ 0000000180012c48     AccessBridgeJavaEntryPoints.obj
 0002:00000c78       ??_C@_0CG@LAIPJCLP@getAccessibleIndexInParentFromC@ 0000000180012c78     AccessBridgeJavaEntryPoints.obj
 0002:00000ca0       ??_C@_0CG@KMCKGMOL@getAccessibleChildrenCountFromC@ 0000000180012ca0     AccessBridgeJavaEntryPoints.obj
 0002:00000cd0       ??_C@_0FC@MAPACPFB@?$CILjavax?1accessibility?1Accessibl@ 0000000180012cd0     AccessBridgeJavaEntryPoints.obj
 0002:00000d28       ??_C@_0BO@BJCAFAFF@getAccessibleChildFromContext@ 0000000180012d28     AccessBridgeJavaEntryPoints.obj
 0002:00000d48       ??_C@_0DO@DCCADJME@?$CILjavax?1accessibility?1Accessibl@ 0000000180012d48     AccessBridgeJavaEntryPoints.obj
 0002:00000d88       ??_C@_0CH@EEFIDNHA@getAccessibleBoundsOnScreenFrom@ 0000000180012d88     AccessBridgeJavaEntryPoints.obj
 0002:00000db0       ??_C@_0BP@FJIKBALD@getAccessibleXcoordFromContext@ 0000000180012db0     AccessBridgeJavaEntryPoints.obj
 0002:00000dd0       ??_C@_0BP@LGNIKGFC@getAccessibleYcoordFromContext@ 0000000180012dd0     AccessBridgeJavaEntryPoints.obj
 0002:00000df0       ??_C@_0BP@EMIHBOON@getAccessibleHeightFromContext@ 0000000180012df0     AccessBridgeJavaEntryPoints.obj
 0002:00000e10       ??_C@_0BO@OAEOJGNL@getAccessibleWidthFromContext@ 0000000180012e10     AccessBridgeJavaEntryPoints.obj
 0002:00000e30       ??_C@_0FD@DOBAJOLJ@?$CILjavax?1accessibility?1Accessibl@ 0000000180012e30     AccessBridgeJavaEntryPoints.obj
 0002:00000e88       ??_C@_0CC@MHPILDJI@getAccessibleComponentFromConte@ 0000000180012e88     AccessBridgeJavaEntryPoints.obj
 0002:00000eb0       ??_C@_0FA@DEIINAGF@?$CILjavax?1accessibility?1Accessibl@ 0000000180012eb0     AccessBridgeJavaEntryPoints.obj
 0002:00000f00       ??_C@_0BP@PKDLLPIG@getAccessibleActionFromContext@ 0000000180012f00     AccessBridgeJavaEntryPoints.obj
 0002:00000f20       ??_C@_0FD@KNPEAGPM@?$CILjavax?1accessibility?1Accessibl@ 0000000180012f20     AccessBridgeJavaEntryPoints.obj
 0002:00000f78       ??_C@_0CC@BHJMNIGA@getAccessibleSelectionFromConte@ 0000000180012f78     AccessBridgeJavaEntryPoints.obj
 0002:00000fa0       ??_C@_0EO@JMGLFFGI@?$CILjavax?1accessibility?1Accessibl@ 0000000180012fa0     AccessBridgeJavaEntryPoints.obj
 0002:00000ff0       ??_C@_0BN@CMHLOCAB@getAccessibleTextFromContext@ 0000000180012ff0     AccessBridgeJavaEntryPoints.obj
 0002:00001010       ??_C@_0EP@DILHGLKF@?$CILjavax?1accessibility?1Accessibl@ 0000000180013010     AccessBridgeJavaEntryPoints.obj
 0002:00001060       ??_C@_0BO@BFBIPFI@getAccessibleValueFromContext@ 0000000180013060     AccessBridgeJavaEntryPoints.obj
 0002:00001080       ??_C@_0EP@DNAJNMPI@?$CILjavax?1accessibility?1Accessibl@ 0000000180013080     AccessBridgeJavaEntryPoints.obj
 0002:000010d0       ??_C@_0BO@PAPKMEMG@getAccessibleTableFromContext@ 00000001800130d0     AccessBridgeJavaEntryPoints.obj
 0002:000010f0       ??_C@_0EP@HGIIMPLK@?$CILjavax?1accessibility?1Accessibl@ 00000001800130f0     AccessBridgeJavaEntryPoints.obj
 0002:00001140       ??_C@_0BO@PDGALDAF@getContextFromAccessibleTable@ 0000000180013140     AccessBridgeJavaEntryPoints.obj
 0002:00001160       ??_C@_0BM@FOJGHDMD@getAccessibleTableRowHeader@ 0000000180013160     AccessBridgeJavaEntryPoints.obj
 0002:00001180       ??_C@_0BP@FNCIHNLO@getAccessibleTableColumnHeader@ 0000000180013180     AccessBridgeJavaEntryPoints.obj
 0002:000011a0       ??_C@_0BL@FHMDFDAE@getAccessibleTableRowCount@ 00000001800131a0     AccessBridgeJavaEntryPoints.obj
 0002:000011c0       ??_C@_0BO@FPCPCCIG@getAccessibleTableColumnCount@ 00000001800131c0     AccessBridgeJavaEntryPoints.obj
 0002:000011e0       ??_C@_0FB@MHAEKEPL@?$CILjavax?1accessibility?1Accessibl@ 00000001800131e0     AccessBridgeJavaEntryPoints.obj
 0002:00001238       ??_C@_0CI@CIBBMNLI@getAccessibleTableCellAccessibl@ 0000000180013238     AccessBridgeJavaEntryPoints.obj
 0002:00001260       ??_C@_0CL@HMHFCPKO@?$CILjavax?1accessibility?1Accessibl@ 0000000180013260     AccessBridgeJavaEntryPoints.obj
 0002:00001290       ??_C@_0BM@BBCGJJGP@getAccessibleTableCellIndex@ 0000000180013290     AccessBridgeJavaEntryPoints.obj
 0002:000012b0       ??_C@_0CA@MEOFLNBC@getAccessibleTableCellRowExtent@ 00000001800132b0     AccessBridgeJavaEntryPoints.obj
 0002:000012d0       ??_C@_0CD@GOAKABO@getAccessibleTableCellColumnExt@ 00000001800132d0     AccessBridgeJavaEntryPoints.obj
 0002:000012f8       ??_C@_0CL@BNJKGODM@?$CILjavax?1accessibility?1Accessibl@ 00000001800132f8     AccessBridgeJavaEntryPoints.obj
 0002:00001328       ??_C@_0BO@KIDDCDEB@isAccessibleTableCellSelected@ 0000000180013328     AccessBridgeJavaEntryPoints.obj
 0002:00001348       ??_C@_0CE@NOEAKJPM@getAccessibleTableRowHeaderRowC@ 0000000180013348     AccessBridgeJavaEntryPoints.obj
 0002:00001370       ??_C@_0CH@NOEKFODF@getAccessibleTableColumnHeaderR@ 0000000180013370     AccessBridgeJavaEntryPoints.obj
 0002:00001398       ??_C@_0CH@HOBKNLMK@getAccessibleTableRowHeaderColu@ 0000000180013398     AccessBridgeJavaEntryPoints.obj
 0002:000013c0       ??_C@_0CK@FLEMOIGB@getAccessibleTableColumnHeaderC@ 00000001800133c0     AccessBridgeJavaEntryPoints.obj
 0002:000013f0       ??_C@_0FA@NJKKHECI@?$CILjavax?1accessibility?1Accessibl@ 00000001800133f0     AccessBridgeJavaEntryPoints.obj
 0002:00001440       ??_C@_0CB@KCKFJBAJ@getAccessibleTableRowDescriptio@ 0000000180013440     AccessBridgeJavaEntryPoints.obj
 0002:00001468       ??_C@_0CE@KHNFECJN@getAccessibleTableColumnDescrip@ 0000000180013468     AccessBridgeJavaEntryPoints.obj
 0002:00001490       ??_C@_0CJ@HGNCMOOJ@?$CILjavax?1accessibility?1Accessibl@ 0000000180013490     AccessBridgeJavaEntryPoints.obj
 0002:000014c0       ??_C@_0CE@CDNGIBEK@getAccessibleTableRowSelectionC@ 00000001800134c0     AccessBridgeJavaEntryPoints.obj
 0002:000014e8       ??_C@_0CK@OKAFABOP@?$CILjavax?1accessibility?1Accessibl@ 00000001800134e8     AccessBridgeJavaEntryPoints.obj
 0002:00001518       ??_C@_0BN@PCLDBBIG@isAccessibleTableRowSelected@ 0000000180013518     AccessBridgeJavaEntryPoints.obj
 0002:00001538       ??_C@_0CK@ILOKEAHN@?$CILjavax?1accessibility?1Accessibl@ 0000000180013538     AccessBridgeJavaEntryPoints.obj
 0002:00001568       ??_C@_0CA@CNAAIKJJ@getAccessibleTableRowSelections@ 0000000180013568     AccessBridgeJavaEntryPoints.obj
 0002:00001588       ??_C@_0CH@CDNMHGID@getAccessibleTableColumnSelecti@ 0000000180013588     AccessBridgeJavaEntryPoints.obj
 0002:000015b0       ??_C@_0CA@NFOBJKJN@isAccessibleTableColumnSelected@ 00000001800135b0     AccessBridgeJavaEntryPoints.obj
 0002:000015d0       ??_C@_0CD@FNIEANFO@getAccessibleTableColumnSelecti@ 00000001800135d0     AccessBridgeJavaEntryPoints.obj
 0002:000015f8       ??_C@_0BG@JNIAKEE@getAccessibleTableRow@ 00000001800135f8     AccessBridgeJavaEntryPoints.obj
 0002:00001610       ??_C@_0BJ@DEHNOIGE@getAccessibleTableColumn@ 0000000180013610     AccessBridgeJavaEntryPoints.obj
 0002:00001630       ??_C@_0BI@MLOHLDGL@getAccessibleTableIndex@ 0000000180013630     AccessBridgeJavaEntryPoints.obj
 0002:00001648       ??_C@_0BL@NLFDIBPJ@getAccessibleRelationCount@ 0000000180013648     AccessBridgeJavaEntryPoints.obj
 0002:00001668       ??_C@_0DN@BLNOMAFI@?$CILjavax?1accessibility?1Accessibl@ 0000000180013668     AccessBridgeJavaEntryPoints.obj
 0002:000016a8       ??_C@_0BJ@DOGHLHFJ@getAccessibleRelationKey@ 00000001800136a8     AccessBridgeJavaEntryPoints.obj
 0002:000016c8       ??_C@_0CM@KJPNEAF@?$CILjavax?1accessibility?1Accessibl@ 00000001800136c8     AccessBridgeJavaEntryPoints.obj
 0002:000016f8       ??_C@_0CB@ONJFHOJM@getAccessibleRelationTargetCoun@ 00000001800136f8     AccessBridgeJavaEntryPoints.obj
 0002:00001720       ??_C@_0FD@OOMEDHDI@?$CILjavax?1accessibility?1Accessibl@ 0000000180013720     AccessBridgeJavaEntryPoints.obj
 0002:00001778       ??_C@_0BM@MFFGDMCG@getAccessibleRelationTarget@ 0000000180013778     AccessBridgeJavaEntryPoints.obj
 0002:000017a0       ??_C@_0FD@IPGDKGIL@?$CILjavax?1accessibility?1Accessibl@ 00000001800137a0     AccessBridgeJavaEntryPoints.obj
 0002:000017f8       ??_C@_0BH@IPNEFMCF@getAccessibleHypertext@ 00000001800137f8     AccessBridgeJavaEntryPoints.obj
 0002:00001810       ??_C@_0FE@PMDDAMJI@?$CILjavax?1accessibility?1Accessibl@ 0000000180013810     AccessBridgeJavaEntryPoints.obj
 0002:00001868       ??_C@_0BM@JMCFFMCN@activateAccessibleHyperlink@ 0000000180013868     AccessBridgeJavaEntryPoints.obj
 0002:00001888       ??_C@_0BM@IADLHNKN@getAccessibleHyperlinkCount@ 0000000180013888     AccessBridgeJavaEntryPoints.obj
 0002:000018b0       ??_C@_0FG@JAOELFOA@?$CILjavax?1accessibility?1Accessibl@ 00000001800138b0     AccessBridgeJavaEntryPoints.obj
 0002:00001908       ??_C@_0BH@EAGDOOIC@getAccessibleHyperlink@ 0000000180013908     AccessBridgeJavaEntryPoints.obj
 0002:00001920       ??_C@_0DO@OBGKICOI@?$CILjavax?1accessibility?1Accessibl@ 0000000180013920     AccessBridgeJavaEntryPoints.obj
 0002:00001960       ??_C@_0BL@MPKBBMO@getAccessibleHyperlinkText@ 0000000180013960     AccessBridgeJavaEntryPoints.obj
 0002:00001980       ??_C@_0BK@DJNACEGJ@getAccessibleHyperlinkURL@ 0000000180013980     AccessBridgeJavaEntryPoints.obj
 0002:000019a0       ??_C@_0CN@CAHDBMA@?$CILjavax?1accessibility?1Accessibl@ 00000001800139a0     AccessBridgeJavaEntryPoints.obj
 0002:000019d0       ??_C@_0CB@LKDEDAHI@getAccessibleHyperlinkStartInde@ 00000001800139d0     AccessBridgeJavaEntryPoints.obj
 0002:000019f8       ??_C@_0BP@KJGEOOIO@getAccessibleHyperlinkEndIndex@ 00000001800139f8     AccessBridgeJavaEntryPoints.obj
 0002:00001a18       ??_C@_0CO@HPBFOBHC@?$CILjavax?1accessibility?1Accessibl@ 0000000180013a18     AccessBridgeJavaEntryPoints.obj
 0002:00001a48       ??_C@_0CA@FBPINCJA@getAccessibleHypertextLinkIndex@ 0000000180013a48     AccessBridgeJavaEntryPoints.obj
 0002:00001a68       ??_C@_0BO@KGNEMCMH@getAccessibleKeyBindingsCount@ 0000000180013a68     AccessBridgeJavaEntryPoints.obj
 0002:00001a88       ??_C@_0CM@PAHADMIP@?$CILjavax?1accessibility?1Accessibl@ 0000000180013a88     AccessBridgeJavaEntryPoints.obj
 0002:00001ab8       ??_C@_0BM@HBNEDKIN@getAccessibleKeyBindingChar@ 0000000180013ab8     AccessBridgeJavaEntryPoints.obj
 0002:00001ad8       ??_C@_0CB@CIMFEKNG@getAccessibleKeyBindingModifier@ 0000000180013ad8     AccessBridgeJavaEntryPoints.obj
 0002:00001b00       ??_C@_0BI@MJKKDJIF@getAccessibleIconsCount@ 0000000180013b00     AccessBridgeJavaEntryPoints.obj
 0002:00001b18       ??_C@_0BN@CJEBMOD@getAccessibleIconDescription@ 0000000180013b18     AccessBridgeJavaEntryPoints.obj
 0002:00001b38       ??_C@_0BI@MDOGDIAA@getAccessibleIconHeight@ 0000000180013b38     AccessBridgeJavaEntryPoints.obj
 0002:00001b50       ??_C@_0BH@GGKEIMGD@getAccessibleIconWidth@ 0000000180013b50     AccessBridgeJavaEntryPoints.obj
 0002:00001b68       ??_C@_0BK@PKOFGGNC@getAccessibleActionsCount@ 0000000180013b68     AccessBridgeJavaEntryPoints.obj
 0002:00001b88       ??_C@_0BI@DODALGBC@getAccessibleActionName@ 0000000180013b88     AccessBridgeJavaEntryPoints.obj
 0002:00001ba0       ??_C@_0BE@CCPKEBNJ@doAccessibleActions@ 0000000180013ba0     AccessBridgeJavaEntryPoints.obj
 0002:00001bb8       ??_C@_0CC@JCBADKJK@getAccessibleCharCountFromConte@ 0000000180013bb8     AccessBridgeJavaEntryPoints.obj
 0002:00001be0       ??_C@_0CG@KPDPNIKI@getAccessibleCaretPositionFromC@ 0000000180013be0     AccessBridgeJavaEntryPoints.obj
 0002:00001c08       ??_C@_0CN@CCCKKDDE@?$CILjavax?1accessibility?1Accessibl@ 0000000180013c08     AccessBridgeJavaEntryPoints.obj
 0002:00001c38       ??_C@_0CF@IPJFBKEC@getAccessibleIndexAtPointFromCo@ 0000000180013c38     AccessBridgeJavaEntryPoints.obj
 0002:00001c60       ??_C@_0CG@CGEAMPNI@getAccessibleLetterAtIndexFromC@ 0000000180013c60     AccessBridgeJavaEntryPoints.obj
 0002:00001c88       ??_C@_0CE@CLNANFEE@getAccessibleWordAtIndexFromCon@ 0000000180013c88     AccessBridgeJavaEntryPoints.obj
 0002:00001cb0       ??_C@_0CI@BJNPGKMI@getAccessibleSentenceAtIndexFro@ 0000000180013cb0     AccessBridgeJavaEntryPoints.obj
 0002:00001cd8       ??_C@_0CL@HGHPNDH@getAccessibleTextSelectionStart@ 0000000180013cd8     AccessBridgeJavaEntryPoints.obj
 0002:00001d08       ??_C@_0CJ@IPEBCNBB@getAccessibleTextSelectionEndFr@ 0000000180013d08     AccessBridgeJavaEntryPoints.obj
 0002:00001d38       ??_C@_0CJ@IBCLFAFA@getAccessibleTextSelectedTextFr@ 0000000180013d38     AccessBridgeJavaEntryPoints.obj
 0002:00001d68       ??_C@_0CK@JLPCFBLN@getAccessibleAttributesAtIndexF@ 0000000180013d68     AccessBridgeJavaEntryPoints.obj
 0002:00001da0       ??_C@_0EK@JEPLCIJI@?$CILjavax?1accessibility?1Accessibl@ 0000000180013da0     AccessBridgeJavaEntryPoints.obj
 0002:00001df0       ??_C@_0CM@LKNKHCB@getAccessibleAttributeSetAtInde@ 0000000180013df0     AccessBridgeJavaEntryPoints.obj
 0002:00001e20       ??_C@_0DP@HKEBFOCN@?$CILjavax?1accessibility?1Accessibl@ 0000000180013e20     AccessBridgeJavaEntryPoints.obj
 0002:00001e60       ??_C@_0CI@IIHCGONP@getAccessibleTextRectAtIndexFro@ 0000000180013e60     AccessBridgeJavaEntryPoints.obj
 0002:00001e88       ??_C@_0CO@OMLKOFDL@getAccessibleXcoordTextRectAtIn@ 0000000180013e88     AccessBridgeJavaEntryPoints.obj
 0002:00001eb8       ??_C@_0CO@NKEIHFMI@getAccessibleYcoordTextRectAtIn@ 0000000180013eb8     AccessBridgeJavaEntryPoints.obj
 0002:00001ee8       ??_C@_0CO@JHFMLGGO@getAccessibleHeightTextRectAtIn@ 0000000180013ee8     AccessBridgeJavaEntryPoints.obj
 0002:00001f18       ??_C@_0CN@COKFHFFE@getAccessibleWidthTextRectAtInd@ 0000000180013f18     AccessBridgeJavaEntryPoints.obj
 0002:00001f48       ??_C@_0BC@NPONPPPN@getCaretLocationX@ 0000000180013f48     AccessBridgeJavaEntryPoints.obj
 0002:00001f60       ??_C@_0BC@MGPGMOLM@getCaretLocationY@ 0000000180013f60     AccessBridgeJavaEntryPoints.obj
 0002:00001f78       ??_C@_0BH@MJJIPGPF@getCaretLocationHeight@ 0000000180013f78     AccessBridgeJavaEntryPoints.obj
 0002:00001f90       ??_C@_0BG@BIMEFOON@getCaretLocationWidth@ 0000000180013f90     AccessBridgeJavaEntryPoints.obj
 0002:00001fa8       ??_C@_0CL@JPPFAPAC@getAccessibleTextLineLeftBounds@ 0000000180013fa8     AccessBridgeJavaEntryPoints.obj
 0002:00001fd8       ??_C@_0CM@IBNKHADJ@getAccessibleTextLineRightBound@ 0000000180013fd8     AccessBridgeJavaEntryPoints.obj
 0002:00002008       ??_C@_0DO@MIIPGCPP@?$CILjavax?1accessibility?1Accessibl@ 0000000180014008     AccessBridgeJavaEntryPoints.obj
 0002:00002048       ??_C@_0CC@CIBLKPOK@getAccessibleTextRangeFromConte@ 0000000180014048     AccessBridgeJavaEntryPoints.obj
 0002:00002070       ??_C@_0CF@CJIJHKPD@getCurrentAccessibleValueFromCo@ 0000000180014070     AccessBridgeJavaEntryPoints.obj
 0002:00002098       ??_C@_0CF@PMHBGBIN@getMaximumAccessibleValueFromCo@ 0000000180014098     AccessBridgeJavaEntryPoints.obj
 0002:000020c0       ??_C@_0CF@MEICJJIC@getMinimumAccessibleValueFromCo@ 00000001800140c0     AccessBridgeJavaEntryPoints.obj
 0002:000020e8       ??_C@_0CM@MHMFNKJL@?$CILjavax?1accessibility?1Accessibl@ 00000001800140e8     AccessBridgeJavaEntryPoints.obj
 0002:00002118       ??_C@_0CC@OHDKMAMO@addAccessibleSelectionFromConte@ 0000000180014118     AccessBridgeJavaEntryPoints.obj
 0002:00002140       ??_C@_0CL@HAAKHFKD@?$CILjavax?1accessibility?1Accessibl@ 0000000180014140     AccessBridgeJavaEntryPoints.obj
 0002:00002170       ??_C@_0CE@JAJNKBKJ@clearAccessibleSelectionFromCon@ 0000000180014170     AccessBridgeJavaEntryPoints.obj
 0002:00002198       ??_C@_0CH@GOOENNPE@getAccessibleSelectionCountFrom@ 0000000180014198     AccessBridgeJavaEntryPoints.obj
 0002:000021c0       ??_C@_0CM@GLHAJFJH@?$CILjavax?1accessibility?1Accessibl@ 00000001800141c0     AccessBridgeJavaEntryPoints.obj
 0002:000021f0       ??_C@_0CF@PFGNJKHP@isAccessibleChildSelectedFromCo@ 00000001800141f0     AccessBridgeJavaEntryPoints.obj
 0002:00002218       ??_C@_0CF@LNEMJFKL@removeAccessibleSelectionFromCo@ 0000000180014218     AccessBridgeJavaEntryPoints.obj
 0002:00002240       ??_C@_0CI@GIPFHPKO@selectAllAccessibleSelectionFro@ 0000000180014240     AccessBridgeJavaEntryPoints.obj
 0002:00002268       ??_C@_04OHLIFDMD@?$CIJ?$CJV@ 0000000180014268     AccessBridgeJavaEntryPoints.obj
 0002:00002270       ??_C@_0BJ@MPIBKFAO@addJavaEventNotification@ 0000000180014270     AccessBridgeJavaEntryPoints.obj
 0002:00002290       ??_C@_0BM@FNBBPCEJ@removeJavaEventNotification@ 0000000180014290     AccessBridgeJavaEntryPoints.obj
 0002:000022b0       ??_C@_0CC@MPLKGCBM@addAccessibilityEventNotificati@ 00000001800142b0     AccessBridgeJavaEntryPoints.obj
 0002:000022d8       ??_C@_0CF@JFMMDHHJ@removeAccessibilityEventNotific@ 00000001800142d8     AccessBridgeJavaEntryPoints.obj
 0002:00002300       ??_C@_0CD@PFBLKFGD@?$CILjavax?1swing?1text?1AttributeSet@ 0000000180014300     AccessBridgeJavaEntryPoints.obj
 0002:00002328       ??_C@_0BI@PMOBPKB@getBoldFromAttributeSet@ 0000000180014328     AccessBridgeJavaEntryPoints.obj
 0002:00002340       ??_C@_0BK@HMLEJNMA@getItalicFromAttributeSet@ 0000000180014340     AccessBridgeJavaEntryPoints.obj
 0002:00002360       ??_C@_0BN@BGEODKID@getUnderlineFromAttributeSet@ 0000000180014360     AccessBridgeJavaEntryPoints.obj
 0002:00002380       ??_C@_0CB@BICMGOJK@getStrikethroughFromAttributeSe@ 0000000180014380     AccessBridgeJavaEntryPoints.obj
 0002:000023a8       ??_C@_0BP@BNLEAGAN@getSuperscriptFromAttributeSet@ 00000001800143a8     AccessBridgeJavaEntryPoints.obj
 0002:000023c8       ??_C@_0BN@FENOLEGG@getSubscriptFromAttributeSet@ 00000001800143c8     AccessBridgeJavaEntryPoints.obj
 0002:000023e8       ??_C@_0DE@PFGGMCPM@?$CILjavax?1swing?1text?1AttributeSet@ 00000001800143e8     AccessBridgeJavaEntryPoints.obj
 0002:00002420       ??_C@_0CD@MGNACFJA@getBackgroundColorFromAttribute@ 0000000180014420     AccessBridgeJavaEntryPoints.obj
 0002:00002448       ??_C@_0CD@JFAEMBOF@getForegroundColorFromAttribute@ 0000000180014448     AccessBridgeJavaEntryPoints.obj
 0002:00002470       ??_C@_0BO@JFHBDDGD@getFontFamilyFromAttributeSet@ 0000000180014470     AccessBridgeJavaEntryPoints.obj
 0002:00002490       ??_C@_0CD@JEPEOEPB@?$CILjavax?1swing?1text?1AttributeSet@ 0000000180014490     AccessBridgeJavaEntryPoints.obj
 0002:000024b8       ??_C@_0BM@OMIOBJPB@getFontSizeFromAttributeSet@ 00000001800144b8     AccessBridgeJavaEntryPoints.obj
 0002:000024d8       ??_C@_0BN@BAFOGOJK@getAlignmentFromAttributeSet@ 00000001800144d8     AccessBridgeJavaEntryPoints.obj
 0002:000024f8       ??_C@_0BN@DEDFHCOP@getBidiLevelFromAttributeSet@ 00000001800144f8     AccessBridgeJavaEntryPoints.obj
 0002:00002518       ??_C@_0CD@BDGMPIDO@?$CILjavax?1swing?1text?1AttributeSet@ 0000000180014518     AccessBridgeJavaEntryPoints.obj
 0002:00002540       ??_C@_0CD@EJOOBJDB@getFirstLineIndentFromAttribute@ 0000000180014540     AccessBridgeJavaEntryPoints.obj
 0002:00002568       ??_C@_0BO@KCBIJLNO@getLeftIndentFromAttributeSet@ 0000000180014568     AccessBridgeJavaEntryPoints.obj
 0002:00002588       ??_C@_0BP@KEIFBKEA@getRightIndentFromAttributeSet@ 0000000180014588     AccessBridgeJavaEntryPoints.obj
 0002:000025a8       ??_C@_0BP@ICDNCHPN@getLineSpacingFromAttributeSet@ 00000001800145a8     AccessBridgeJavaEntryPoints.obj
 0002:000025c8       ??_C@_0BO@CHPMHCHE@getSpaceAboveFromAttributeSet@ 00000001800145c8     AccessBridgeJavaEntryPoints.obj
 0002:000025e8       ??_C@_0BO@DOLMIFOK@getSpaceBelowFromAttributeSet@ 00000001800145e8     AccessBridgeJavaEntryPoints.obj
 0002:00002608       ??_C@_0CL@NMLPDKKP@?$CILjavax?1accessibility?1Accessibl@ 0000000180014608     AccessBridgeJavaEntryPoints.obj
 0002:00002638       ??_C@_0N@CEMKNPGL@requestFocus@ 0000000180014638     AccessBridgeJavaEntryPoints.obj
 0002:00002648       ??_C@_0CN@EDMFOCKG@?$CILjavax?1accessibility?1Accessibl@ 0000000180014648     AccessBridgeJavaEntryPoints.obj
 0002:00002678       ??_C@_0BA@JKPGAJFL@selectTextRange@ 0000000180014678     AccessBridgeJavaEntryPoints.obj
 0002:00002688       ??_C@_0BI@IIOLCPFK@getVisibleChildrenCount@ 0000000180014688     AccessBridgeJavaEntryPoints.obj
 0002:000026a0       ??_C@_0BA@JIDLMKH@getVisibleChild@ 00000001800146a0     AccessBridgeJavaEntryPoints.obj
 0002:000026b0       ??_C@_0BB@ENIAPGBO@setCaretPosition@ 00000001800146b0     AccessBridgeJavaEntryPoints.obj
 0002:000026c8       ??_C@_0CE@MELACKPN@getVirtualAccessibleNameFromCon@ 00000001800146c8     AccessBridgeJavaEntryPoints.obj
 0002:000026f0       ??_C@_0DP@ODHDIMGL@?$FLINFO?$FN?3?5Calling?5AccessBridgeJav@ 00000001800146f0     AccessBridgeJavaEntryPoints.obj
 0002:00002730       ??_C@_0DD@INJPOCHE@Getting?5isJavaWindow?5?9?5call?5to?5@ 0000000180014730     AccessBridgeJavaEntryPoints.obj
 0002:00002768       ??_C@_0DN@ENCLOLFG@?$FLERROR?$FN?3?5?$CK?$CK?$CK?5Exception?5occured?5@ 0000000180014768     AccessBridgeJavaEntryPoints.obj
 0002:000027a8       ??_C@_0DH@DHJJKMLN@?$FLERROR?$FN?3?5either?5jniEnv?5?$DN?$DN?50?5or?5@ 00000001800147a8     AccessBridgeJavaEntryPoints.obj
 0002:000027e0       ??_C@_0DN@GKGIBPBO@?$FLINFO?$FN?3?5In?5AccessBridgeJavaEntr@ 00000001800147e0     AccessBridgeJavaEntryPoints.obj
 0002:00002820       ??_C@_0BF@LOIOEBHF@Calling?5IsSameObject@ 0000000180014820     AccessBridgeJavaEntryPoints.obj
 0002:00002838       ??_C@_0CE@PJOLBDKG@?$FLINFO?$FN?3?5?5?5isSameObject?5returnin@ 0000000180014838     AccessBridgeJavaEntryPoints.obj
 0002:00002860       ??_C@_0EK@MPPKLDGH@?$FLINFO?$FN?3?5In?5AccessBridgeJavaEntr@ 0000000180014860     AccessBridgeJavaEntryPoints.obj
 0002:000028b0       ??_C@_0DP@INBKCEII@Getting?5AccessibleContextFromHW@ 00000001800148b0     AccessBridgeJavaEntryPoints.obj
 0002:000028f0       ??_C@_0EI@POHJNOIF@?$FLERROR?$FN?3?5?5either?5jniEnv?5?$DN?$DN?50?5or@ 00000001800148f0     AccessBridgeJavaEntryPoints.obj
 0002:00002940       ??_C@_0EK@KGPHBKLN@?$FLINFO?$FN?3?5In?5AccessBridgeJavaEntr@ 0000000180014940     AccessBridgeJavaEntryPoints.obj
 0002:00002990       ??_C@_0DM@OPKABADC@Getting?5HWNDFromAccessibleConte@ 0000000180014990     AccessBridgeJavaEntryPoints.obj
 0002:000029d0       ??_C@_0BD@NKFEMHLM@?$FLINFO?$FN?3?5rHWND?5?$DN?5?$CFX@ 00000001800149d0     AccessBridgeJavaEntryPoints.obj
 0002:000029f0       ??_C@_0EH@MFPOIGJN@?$FLERROR?$FN?3?5either?5jniEnv?5?$DN?$DN?50?5or?5@ 00000001800149f0     AccessBridgeJavaEntryPoints.obj
 0002:00002a40       ??_C@_0EC@BPPANMDJ@?$FLINFO?$FN?3?5In?5AccessBridgeJavaEntr@ 0000000180014a40     AccessBridgeJavaEntryPoints.obj
 0002:00002a88       ??_C@_0BN@LGGMDMGD@?$FLERROR?$FN?3?5?5?5?5NewString?5failed@ 0000000180014a88     AccessBridgeJavaEntryPoints.obj
 0002:00002aa8       ??_C@_0CO@NCDGKPGB@setTextContents?5?9?5call?5to?5CallB@ 0000000180014aa8     AccessBridgeJavaEntryPoints.obj
 0002:00002ad8       ??_C@_0BI@IMHMFAIB@?$FLINFO?$FN?3?5?5?5?5?5result?5?$DN?5?$CFd@ 0000000180014ad8     AccessBridgeJavaEntryPoints.obj
 0002:00002af0       ??_C@_0DK@MGDAPF@?$FLERROR?$FN?3?5either?5jniEnv?5?$DN?$DN?50?5or?5@ 0000000180014af0     AccessBridgeJavaEntryPoints.obj
 0002:00002b30       ??_C@_0DP@LHNNHOD@?$FLINFO?$FN?3?5In?5AccessBridgeJavaEntr@ 0000000180014b30     AccessBridgeJavaEntryPoints.obj
 0002:00002b70       ??_C@_0BO@LLFKIHLA@?$FLERROR?$FN?3?5?5?5?5?5NewString?5failed@ 0000000180014b70     AccessBridgeJavaEntryPoints.obj
 0002:00002b90       ??_C@_0DE@KBFMBJPI@Getting?5ParentWithRole?5?9?5call?5t@ 0000000180014b90     AccessBridgeJavaEntryPoints.obj
 0002:00002bc8       ??_C@_0CE@LNEDINGM@?$FLINFO?$FN?3?5?5?5?5?5rAccessibleContext?5@ 0000000180014bc8     AccessBridgeJavaEntryPoints.obj
 0002:00002bf0       ??_C@_0DA@OMNPGENP@Getting?5ParentWithRole?5?9?5call?5t@ 0000000180014bf0     AccessBridgeJavaEntryPoints.obj
 0002:00002c20       ??_C@_0EF@LHAMKGPK@?$FLINFO?$FN?3?5?5?5Returning?5?9?5returnedA@ 0000000180014c20     AccessBridgeJavaEntryPoints.obj
 0002:00002c68       ??_C@_0DM@OLEIFDLG@?$FLERROR?$FN?3?5either?5jniEnv?5?$DN?$DN?50?5or?5@ 0000000180014c68     AccessBridgeJavaEntryPoints.obj
 0002:00002ca8       ??_C@_0DP@EPHBFJKE@?$FLINFO?$FN?3?5In?5AccessBridgeJavaEntr@ 0000000180014ca8     AccessBridgeJavaEntryPoints.obj
 0002:00002ce8       ??_C@_0DE@FDIFCLEM@Getting?5TopLevelObject?5?9?5call?5t@ 0000000180014ce8     AccessBridgeJavaEntryPoints.obj
 0002:00002d20       ??_C@_0CB@GDMCCFCK@?$FLINFO?$FN?3?5?5rAccessibleContext?5?$DN?5?$CF@ 0000000180014d20     AccessBridgeJavaEntryPoints.obj
 0002:00002d48       ??_C@_0DA@ELIJHKN@Getting?5TopLevelObject?5?9?5call?5t@ 0000000180014d48     AccessBridgeJavaEntryPoints.obj
 0002:00002d78       ??_C@_0DM@MKIGPNDF@?$FLERROR?$FN?3?5either?5jniEnv?5?$DN?$DN?50?5or?5@ 0000000180014d78     AccessBridgeJavaEntryPoints.obj
 0002:00002dc0       ??_C@_0EH@MCHGGFNF@?$FLINFO?$FN?3?5In?5AccessBridgeJavaEntr@ 0000000180014dc0     AccessBridgeJavaEntryPoints.obj
 0002:00002e08       ??_C@_0DM@IKNMPPHI@Getting?5ParentWithRoleElseRoot?5@ 0000000180014e08     AccessBridgeJavaEntryPoints.obj
 0002:00002e48       ??_C@_0DI@CDJCPAOF@Getting?5ParentWithRoleElseRoot?5@ 0000000180014e48     AccessBridgeJavaEntryPoints.obj
 0002:00002e80       ??_C@_0EF@MODADMKL@?$FLERROR?$FN?3?5?5either?5jniEnv?5?$DN?$DN?50?5or@ 0000000180014e80     AccessBridgeJavaEntryPoints.obj
 0002:00002ec8       ??_C@_0DM@EBONPKNN@?$FLINFO?$FN?3?5In?5AccessBridgeJavaEntr@ 0000000180014ec8     AccessBridgeJavaEntryPoints.obj
 0002:00002f08       ??_C@_0CO@CCBFEFG@Getting?5ObjectDepth?5?9?5call?5to?5C@ 0000000180014f08     AccessBridgeJavaEntryPoints.obj
 0002:00002f38       ??_C@_0BJ@KJFHIGKC@?$FLINFO?$FN?3?5?5?5?5?5rResult?5?$DN?5?$CFd@ 0000000180014f38     AccessBridgeJavaEntryPoints.obj
 0002:00002f58       ??_C@_0DJ@NCMDONA@?$FLERROR?$FN?3?5either?5jniEnv?5?$DN?$DN?50?5or?5@ 0000000180014f58     AccessBridgeJavaEntryPoints.obj
 0002:00002fa0       ??_C@_0EB@OJAHMNKI@?$FLINFO?$FN?3?5In?5AccessBridgeJavaEntr@ 0000000180014fa0     AccessBridgeJavaEntryPoints.obj
 0002:00002fe8       ??_C@_0DG@FKCKDOAD@Getting?5ActiveDescendent?5?9?5call@ 0000000180014fe8     AccessBridgeJavaEntryPoints.obj
 0002:00003020       ??_C@_0DC@DOJHNKHC@Getting?5ActiveDescendant?5?9?5call@ 0000000180015020     AccessBridgeJavaEntryPoints.obj
 0002:00003058       ??_C@_0DO@FBKMCPK@?$FLERROR?$FN?3?5either?5jniEnv?5?$DN?$DN?50?5or?5@ 0000000180015058     AccessBridgeJavaEntryPoints.obj
 0002:00003098       ??_C@_0CK@IFAHAOG@?$FLINFO?$FN?3?5?5getVirtualAccessibleNa@ 0000000180015098     AccessBridgeJavaEntryPoints.obj
 0002:000030c8       ??_C@_0DE@GLGPLDPG@Getting?5AccessibleName?5?9?5call?5t@ 00000001800150c8     AccessBridgeJavaEntryPoints.obj
 0002:00003100       ??_C@_0DC@LMABNHGH@Getting?5AccessibleName?5?9?5call?5t@ 0000000180015100     AccessBridgeJavaEntryPoints.obj
 0002:00003138       ??_C@_0BH@PDDJGLOG@Getting?5AccessibleName@ 0000000180015138     AccessBridgeJavaEntryPoints.obj
 0002:00003150       ??_C@_0FH@LIIILLEC@?$FLERROR?$FN?3?5?$CK?$CK?$CK?5Exception?5occured?5@ 0000000180015150     AccessBridgeJavaEntryPoints.obj
 0002:000031b0       ??_C@_0FK@LMDLLNDA@?$FLERROR?$FN?3?5?$CK?$CK?$CK?5Exception?5occured?5@ 00000001800151b0     AccessBridgeJavaEntryPoints.obj
 0002:00003210       ??_C@_0DC@MBCPGFEL@Getting?5AccessibleName?5?9?5call?5t@ 0000000180015210     AccessBridgeJavaEntryPoints.obj
 0002:00003248       ??_C@_1DA@BACBNKJB@?$AA?5?$AA?5?$AAA?$AAc?$AAc?$AAe?$AAs?$AAs?$AAi?$AAb?$AAl?$AAe?$AA?5?$AAN?$AAa@ 0000000180015248     AccessBridgeJavaEntryPoints.obj
 0002:00003278       ??_C@_0DC@HCPEBFPJ@Getting?5AccessibleName?5?9?5call?5t@ 0000000180015278     AccessBridgeJavaEntryPoints.obj
 0002:000032b0       ??_C@_0CD@JNOMKFNM@?$FLINFO?$FN?3?5?5?5Accessible?5Name?5is?5nu@ 00000001800152b0     AccessBridgeJavaEntryPoints.obj
 0002:000032e0       ??_C@_0EN@LBGKPBFG@?$FLINFO?$FN?3?5either?5jniEnv?5?$DN?$DN?50?5or?5g@ 00000001800152e0     AccessBridgeJavaEntryPoints.obj
 0002:00003330       ??_C@_0DK@COLMCNJL@?$FLINFO?$FN?3?5In?5AccessBridgeJavaEntr@ 0000000180015330     AccessBridgeJavaEntryPoints.obj
 0002:00003370       ??_C@_0CL@OHFNFEAE@requestFocus?5?9?5call?5to?5CallBool@ 0000000180015370     AccessBridgeJavaEntryPoints.obj
 0002:000033a0       ??_C@_0BH@JOKEJIHH@?$FLINFO?$FN?3?5?5?5?5result?5?$DN?5?$CFd@ 00000001800153a0     AccessBridgeJavaEntryPoints.obj
 0002:000033b8       ??_C@_0DH@OADKFKDG@?$FLERROR?$FN?3?5either?5jniEnv?5?$DN?$DN?50?5or?5@ 00000001800153b8     AccessBridgeJavaEntryPoints.obj
 0002:000033f0       ??_C@_0FB@HEEEBDKB@?$FLINFO?$FN?3?5In?5AccessBridgeJavaEntr@ 00000001800153f0     AccessBridgeJavaEntryPoints.obj
 0002:00003448       ??_C@_0CO@NOPLEGNC@selectTextRange?5?9?5call?5to?5CallB@ 0000000180015448     AccessBridgeJavaEntryPoints.obj
 0002:00003478       ??_C@_0DK@EDLAMPCD@?$FLERROR?$FN?3?5either?5jniEnv?5?$DN?$DN?50?5or?5@ 0000000180015478     AccessBridgeJavaEntryPoints.obj
 0002:000034c0       ??_C@_0FK@CBBPCLFD@?$FLINFO?$FN?3?5In?5AccessBridgeJavaEntr@ 00000001800154c0     AccessBridgeJavaEntryPoints.obj
 0002:00003520       ??_C@_0DN@CIOOGMLK@?$FLINFO?$FN?3?5?5Getting?5full?5test_attr@ 0000000180015520     AccessBridgeJavaEntryPoints.obj
 0002:00003560       ??_C@_0EB@FNOCJLAN@Getting?5AccessibleAttributesAtI@ 0000000180015560     AccessBridgeJavaEntryPoints.obj
 0002:000035a8       ??_C@_0DE@NPIJKEOK@?$FLINFO?$FN?3?5?5?5returned?5from?5CallObj@ 00000001800155a8     AccessBridgeJavaEntryPoints.obj
 0002:000035e0       ??_C@_0DP@GAODIEPK@Getting?5AccessibleAttributesAtI@ 00000001800155e0     AccessBridgeJavaEntryPoints.obj
 0002:00003620       ??_C@_0CE@KAHCBNHC@Getting?5AccessibleAttributesAtI@ 0000000180015620     AccessBridgeJavaEntryPoints.obj
 0002:00003648       ??_C@_0DP@BNMNDGNG@Getting?5AccessibleAttributesAtI@ 0000000180015648     AccessBridgeJavaEntryPoints.obj
 0002:00003690       ??_C@_1FE@NAFGNNMA@?$AA?$FL?$AAI?$AAN?$AAF?$AAO?$AA?$FN?$AA?3?$AA?5?$AA?5?$AAA?$AAc?$AAc?$AAe?$AAs?$AAs@ 0000000180015690     AccessBridgeJavaEntryPoints.obj
 0002:000036e8       ??_C@_0DP@KOBGEGGE@Getting?5AccessibleAttributesAtI@ 00000001800156e8     AccessBridgeJavaEntryPoints.obj
 0002:00003728       ??_C@_0CO@GBFCDBDB@?$FLWARN?$FN?3?5?5?5Accessible?5Text?5attri@ 0000000180015728     AccessBridgeJavaEntryPoints.obj
 0002:00003760       ??_C@_0FB@DKHOICMI@?$FLERROR?$FN?3?5either?5env?5?$DN?$DN?50?5or?5get@ 0000000180015760     AccessBridgeJavaEntryPoints.obj
 0002:000037c0       ??_C@_0EH@KKFBHMJC@?$FLINFO?$FN?3?5?$CD?$CD?$CD?$CD?$CD?5AccessBridgeJavaE@ 00000001800157c0     AccessBridgeJavaEntryPoints.obj
 0002:00003808       ??_C@_0DP@MHLDKAGF@?$CD?$CD?$CD?$CD?$CD?5Getting?5visible?5children?5@ 0000000180015808     AccessBridgeJavaEntryPoints.obj
 0002:00003848       ??_C@_0CM@JAPBNGLO@?$FLINFO?$FN?3?5?5?5?$CD?$CD?$CD?$CD?$CD?5visible?5childre@ 0000000180015848     AccessBridgeJavaEntryPoints.obj
 0002:00003880       ??_C@_0FD@GLIPOPHN@?$FLINFO?$FN?3?5?$CD?$CD?$CD?$CD?$CD?5AccessBridgeJavaE@ 0000000180015880     AccessBridgeJavaEntryPoints.obj
 0002:000038d8       ??_C@_0CH@ONKDDCMN@?$FLINFO?$FN?3?5?5?5getting?5visible?5child@ 00000001800158d8     AccessBridgeJavaEntryPoints.obj
 0002:00003900       ??_C@_0DJ@HGPLCHEB@?$CD?$CD?$CD?$CD?$CD?5getVisibleChildMethod?5?9?5c@ 0000000180015900     AccessBridgeJavaEntryPoints.obj
 0002:00003940       ??_C@_0DF@JHJIJJH@?$CD?$CD?$CD?$CD?$CD?5getVisibleChildMethod?5?9?5c@ 0000000180015940     AccessBridgeJavaEntryPoints.obj
 0002:00003978       ??_C@_0CD@ECMHOCH@?$FLINFO?$FN?3?5?5?5?$CD?$CD?$CD?$CD?$CD?5visible?5child?5?$DN@ 0000000180015978     AccessBridgeJavaEntryPoints.obj
 0002:000039a0       ??_C@_0EK@GNPPBBMN@?$FLINFO?$FN?3?5?5?5?$CD?$CD?$CD?$CD?$CD?5AccessBridgeJav@ 00000001800159a0     AccessBridgeJavaEntryPoints.obj
 0002:000039f0       ??_C@_0EL@OPKFGOFA@?$FLINFO?$FN?3?5In?5AccessBridgeJavaEntr@ 00000001800159f0     AccessBridgeJavaEntryPoints.obj
 0002:00003a40       ??_C@_0CO@BDNAFHGG@setCaretPostion?5?9?5call?5to?5CallB@ 0000000180015a40     AccessBridgeJavaEntryPoints.obj
 0002:00003a70       ??_C@_0BJ@PGHBDIPI@?$FLERROR?$FN?3?5?5?5?5?5result?5?$DN?5?$CFd@ 0000000180015a70     AccessBridgeJavaEntryPoints.obj
 0002:00003a90       ??_C@_0DL@CBEPMOL@?$FLERROR?$FN?3?5either?5jniEnv?5?$DN?$DN?50?5or?5@ 0000000180015a90     AccessBridgeJavaEntryPoints.obj
 0002:00003ad0       ??_C@_0DP@DPLDEGDE@?$FLINFO?$FN?3?5Calling?5AccessBridgeJav@ 0000000180015ad0     AccessBridgeJavaEntryPoints.obj
 0002:00003b10       ??_C@_0DJ@EBEOKJAG@Getting?5JavaVersionProperty?5?9?5c@ 0000000180015b10     AccessBridgeJavaEntryPoints.obj
 0002:00003b50       ??_C@_0FC@KFJABCDE@?$FLERROR?$FN?3?5?5?$CK?$CK?$CK?5Exception?5when?5ge@ 0000000180015b50     AccessBridgeJavaEntryPoints.obj
 0002:00003ba8       ??_C@_0DL@FDAICLOI@Getting?5JavaVersionProperty?5?9?5c@ 0000000180015ba8     AccessBridgeJavaEntryPoints.obj
 0002:00003be8       ??_C@_0DH@PEMIMKKJ@Getting?5JavaVersionProperty?5?9?5c@ 0000000180015be8     AccessBridgeJavaEntryPoints.obj
 0002:00003c20       ??_C@_1CK@PFPDBLJ@?$AA?5?$AA?5?$AAJ?$AAa?$AAv?$AAa?$AA?5?$AAv?$AAe?$AAr?$AAs?$AAi?$AAo?$AAn?$AA?5@ 0000000180015c20     AccessBridgeJavaEntryPoints.obj
 0002:00003c50       ??_C@_0DH@EHBDLKBL@Getting?5JavaVersionProperty?5?9?5c@ 0000000180015c50     AccessBridgeJavaEntryPoints.obj
 0002:00003c88       ??_C@_0CA@KOJKOLB@?$FLWARN?$FN?3?5?5?5Java?5version?5is?5null?4@ 0000000180015c88     AccessBridgeJavaEntryPoints.obj
 0002:00003ca8       ??_C@_0DP@FHBJPJDO@?$FLERROR?$FN?3?5?5either?5env?5?$DN?$DN?50?5or?5ge@ 0000000180015ca8     AccessBridgeJavaEntryPoints.obj
 0002:00003cf0       ??_C@_0EC@OAJCCJEK@?$FLINFO?$FN?3?5Calling?5AccessBridgeJav@ 0000000180015cf0     AccessBridgeJavaEntryPoints.obj
 0002:00003d38       ??_C@_0BF@MJCCCBHB@?$FLERROR?$FN?3?5?5No?5Java?5VM@ 0000000180015d38     AccessBridgeJavaEntryPoints.obj
 0002:00003d50       ??_C@_0BH@PCLEJECO@?$FLERROR?$FN?3?5?5Null?5jobject@ 0000000180015d50     AccessBridgeJavaEntryPoints.obj
 0002:00003d68       ??_C@_0DE@FOOENAKM@Getting?5AccessibleText?5?9?5call?5t@ 0000000180015d68     AccessBridgeJavaEntryPoints.obj
 0002:00003da0       ??_C@_0BP@NHKMDDHI@?$FLERROR?$FN?3?5?5?5AccessibleText?5?$DN?5?$CFp@ 0000000180015da0     AccessBridgeJavaEntryPoints.obj
 0002:00003dc0       ??_C@_0DC@NHCDOGBO@Getting?5AccessibleText?5?9?5call?5t@ 0000000180015dc0     AccessBridgeJavaEntryPoints.obj
 0002:00003e00       ??_C@_0EF@KPMHECBJ@?$FLERROR?$FN?3?5?5either?5env?5?$DN?$DN?50?5or?5ge@ 0000000180015e00     AccessBridgeJavaEntryPoints.obj
 0002:00003e48       ??_C@_0CL@OMBEMJIM@?$FLERROR?$FN?3?5?5jobject?5is?5not?5an?5Acc@ 0000000180015e48     AccessBridgeJavaEntryPoints.obj
 0002:00003e80       ??_C@_0FB@IMPDGAOD@?$FLINFO?$FN?3?5Calling?5AccessBridgeJav@ 0000000180015e80     AccessBridgeJavaEntryPoints.obj
 0002:00003ed8       ??_C@_0DJ@CBKJGOIB@Getting?5AccessibleContextAt?5?9?5c@ 0000000180015ed8     AccessBridgeJavaEntryPoints.obj
 0002:00003f18       ??_C@_0DF@PJCJKGPI@Getting?5AccessibleContextAt?5?9?5c@ 0000000180015f18     AccessBridgeJavaEntryPoints.obj
 0002:00003f50       ??_C@_0DP@LFOACNJN@?$FLERROR?$FN?3?5?5either?5env?5?$DN?$DN?50?5or?5ge@ 0000000180015f50     AccessBridgeJavaEntryPoints.obj
 0002:00003f90       ??_C@_0EN@LHFHLFOC@?$FLINFO?$FN?3?5Calling?5AccessBridgeJav@ 0000000180015f90     AccessBridgeJavaEntryPoints.obj
 0002:00003fe0       ??_C@_0EA@NLINILPH@Getting?5AccessibleContextWithFo@ 0000000180015fe0     AccessBridgeJavaEntryPoints.obj
 0002:00004020       ??_C@_0DM@IJDJLPBO@Getting?5AccessibleContextWithFo@ 0000000180016020     AccessBridgeJavaEntryPoints.obj
 0002:00004060       ??_C@_0EJ@KBIILIHA@?$FLERROR?$FN?3?5?5either?5jniEnv?5?$DN?$DN?50?5or@ 0000000180016060     AccessBridgeJavaEntryPoints.obj
 0002:000040b0       ??_C@_0FB@NNGDGCK@?$FLINFO?$FN?3?5?$CD?$CD?$CD?$CD?$CD?5Calling?5AccessBri@ 00000001800160b0     AccessBridgeJavaEntryPoints.obj
 0002:00004108       ??_C@_0DF@BABIDEMG@?$FLWARN?$FN?3?5?5passed?5in?5AccessibleCo@ 0000000180016108     AccessBridgeJavaEntryPoints.obj
 0002:00004140       ??_C@_1EA@IPHAHEJA@?$AA?$FL?$AAI?$AAN?$AAF?$AAO?$AA?$FN?$AA?3?$AA?5?$AA?5?$AA?5?$AAA?$AAc?$AAc?$AAe?$AAs@ 0000000180016140     AccessBridgeJavaEntryPoints.obj
 0002:00004180       ??_C@_0CD@BCDIDKCI@?$FLWARN?$FN?3?5?5?5Accessible?5Name?5is?5nu@ 0000000180016180     AccessBridgeJavaEntryPoints.obj
 0002:000041b0       ??_C@_0EF@DMNCHIBL@?$FLERROR?$FN?3?5?5either?5env?5?$DN?$DN?50?5or?5ge@ 00000001800161b0     AccessBridgeJavaEntryPoints.obj
 0002:000041f8       ??_C@_0DL@IPNAGHCP@Getting?5AccessibleDescription?5?9@ 00000001800161f8     AccessBridgeJavaEntryPoints.obj
 0002:00004240       ??_C@_1EO@NBFBPIFN@?$AA?$FL?$AAI?$AAN?$AAF?$AAO?$AA?$FN?$AA?3?$AA?5?$AA?5?$AA?5?$AAA?$AAc?$AAc?$AAe?$AAs@ 0000000180016240     AccessBridgeJavaEntryPoints.obj
 0002:00004290       ??_C@_0CK@KNEKOBNE@?$FLWARN?$FN?3?5?5?5Accessible?5Descriptio@ 0000000180016290     AccessBridgeJavaEntryPoints.obj
 0002:000042c0       ??_C@_0EM@LPILGNDD@?$FLERROR?$FN?3?5?5either?5env?5?$DN?$DN?50?5or?5ge@ 00000001800162c0     AccessBridgeJavaEntryPoints.obj
 0002:00004310       ??_C@_0DE@IKDIHCF@Getting?5AccessibleRole?5?9?5call?5t@ 0000000180016310     AccessBridgeJavaEntryPoints.obj
 0002:00004348       ??_C@_0DC@FOMJEAJG@Getting?5AccessibleRole?5?9?5call?5t@ 0000000180016348     AccessBridgeJavaEntryPoints.obj
 0002:00004380       ??_C@_0BH@LHDEAMGB@Getting?5AccessibleRole@ 0000000180016380     AccessBridgeJavaEntryPoints.obj
 0002:00004398       ??_C@_0DC@CDOHPCLK@Getting?5AccessibleRole?5?9?5call?5t@ 0000000180016398     AccessBridgeJavaEntryPoints.obj
 0002:000043d0       ??_C@_1EA@DFMPHGFH@?$AA?$FL?$AAI?$AAN?$AAF?$AAO?$AA?$FN?$AA?3?$AA?5?$AA?5?$AA?5?$AAA?$AAc?$AAc?$AAe?$AAs@ 00000001800163d0     AccessBridgeJavaEntryPoints.obj
 0002:00004410       ??_C@_0DC@JADMICAI@Getting?5AccessibleRole?5?9?5call?5t@ 0000000180016410     AccessBridgeJavaEntryPoints.obj
 0002:00004448       ??_C@_0CD@DPDMNHLG@?$FLWARN?$FN?3?5?5?5Accessible?5Role?5is?5nu@ 0000000180016448     AccessBridgeJavaEntryPoints.obj
 0002:00004470       ??_C@_0EL@ENOHPPLP@?$FLERROR?$FN?3?5?5either?5env?5?$DN?$DN?50?5or?5ge@ 0000000180016470     AccessBridgeJavaEntryPoints.obj
 0002:000044c0       ??_C@_0DK@OPAANMJH@Getting?5AccessibleRole_en_US?5?9?5@ 00000001800164c0     AccessBridgeJavaEntryPoints.obj
 0002:00004500       ??_C@_0DI@CJNJDFMD@Getting?5AccessibleRole_en_US?5?9?5@ 0000000180016500     AccessBridgeJavaEntryPoints.obj
 0002:00004538       ??_C@_0BN@HKCJIFDO@Getting?5AccessibleRole_en_US@ 0000000180016538     AccessBridgeJavaEntryPoints.obj
 0002:00004558       ??_C@_0DI@FEPHIHOP@Getting?5AccessibleRole_en_US?5?9?5@ 0000000180016558     AccessBridgeJavaEntryPoints.obj
 0002:00004590       ??_C@_1EM@ICLLIBMO@?$AA?$FL?$AAI?$AAN?$AAF?$AAO?$AA?$FN?$AA?3?$AA?5?$AA?5?$AA?5?$AAA?$AAc?$AAc?$AAe?$AAs@ 0000000180016590     AccessBridgeJavaEntryPoints.obj
 0002:000045e0       ??_C@_0DI@OHCMPHFN@Getting?5AccessibleRole_en_US?5?9?5@ 00000001800165e0     AccessBridgeJavaEntryPoints.obj
 0002:00004618       ??_C@_0CJ@JHFOCCMF@?$FLWARN?$FN?3?5?5?5Accessible?5Role?5en_US@ 0000000180016618     AccessBridgeJavaEntryPoints.obj
 0002:00004650       ??_C@_0FA@EDCBAJIO@?$FLERROR?$FN?3?5either?5env?5?$DN?$DN?50?5or?5get@ 0000000180016650     AccessBridgeJavaEntryPoints.obj
 0002:000046a0       ??_C@_0DF@HNCNCNCA@Getting?5AccessibleState?5?9?5call?5@ 00000001800166a0     AccessBridgeJavaEntryPoints.obj
 0002:000046d8       ??_C@_0DD@FJJPIJBK@Getting?5AccessibleState?5?9?5call?5@ 00000001800166d8     AccessBridgeJavaEntryPoints.obj
 0002:00004710       ??_C@_0BI@BBGKJOIM@Getting?5AccessibleState@ 0000000180016710     AccessBridgeJavaEntryPoints.obj
 0002:00004728       ??_C@_0DD@CELBDLDG@Getting?5AccessibleState?5?9?5call?5@ 0000000180016728     AccessBridgeJavaEntryPoints.obj
 0002:00004760       ??_C@_1EE@DCJFHGCM@?$AA?$FL?$AAI?$AAN?$AAF?$AAO?$AA?$FN?$AA?3?$AA?5?$AA?5?$AA?5?$AAA?$AAc?$AAc?$AAe?$AAs@ 0000000180016760     AccessBridgeJavaEntryPoints.obj
 0002:000047a8       ??_C@_0DD@JHGKELIE@Getting?5AccessibleState?5?9?5call?5@ 00000001800167a8     AccessBridgeJavaEntryPoints.obj
 0002:000047e0       ??_C@_0CF@EJIKBPCF@?$FLWARN?$FN?3?5?5?5Accessible?5States?5is?5@ 00000001800167e0     AccessBridgeJavaEntryPoints.obj
 0002:00004810       ??_C@_0EN@PLJCLDAI@?$FLERROR?$FN?3?5?5either?5env?5?$DN?$DN?50?5or?5ge@ 0000000180016810     AccessBridgeJavaEntryPoints.obj
 0002:00004860       ??_C@_0DL@NKOGKBKA@Getting?5AccessibleState_en_US?5?9@ 0000000180016860     AccessBridgeJavaEntryPoints.obj
 0002:000048a0       ??_C@_0DJ@EPIHCNDB@Getting?5AccessibleState_en_US?5?9@ 00000001800168a0     AccessBridgeJavaEntryPoints.obj
 0002:000048e0       ??_C@_0BO@INBCKAFB@Getting?5AccessibleState_en_US@ 00000001800168e0     AccessBridgeJavaEntryPoints.obj
 0002:00004900       ??_C@_0DJ@DCKJJPBN@Getting?5AccessibleState_en_US?5?9@ 0000000180016900     AccessBridgeJavaEntryPoints.obj
 0002:00004940       ??_C@_1FA@BNDENPHM@?$AA?$FL?$AAI?$AAN?$AAF?$AAO?$AA?$FN?$AA?3?$AA?5?$AA?5?$AA?5?$AAA?$AAc?$AAc?$AAe?$AAs@ 0000000180016940     AccessBridgeJavaEntryPoints.obj
 0002:00004990       ??_C@_0DJ@IBHCOPKP@Getting?5AccessibleState_en_US?5?9@ 0000000180016990     AccessBridgeJavaEntryPoints.obj
 0002:000049d0       ??_C@_0CL@LNKMOAJG@?$FLWARN?$FN?3?5?5?5Accessible?5States?5en_@ 00000001800169d0     AccessBridgeJavaEntryPoints.obj
 0002:00004a00       ??_C@_0FC@KNGBOCJI@?$FLERROR?$FN?3?5either?5env?5?$DN?$DN?50?5or?5get@ 0000000180016a00     AccessBridgeJavaEntryPoints.obj
 0002:00004a58       ??_C@_0DK@NAACLIEE@Getting?5AccessibleIndexInParent@ 0000000180016a58     AccessBridgeJavaEntryPoints.obj
 0002:00004a98       ??_C@_0BP@LDKDBFNM@?$FLINFO?$FN?3?5?5?5Index?5in?5Parent?5?$DN?5?$CFd@ 0000000180016a98     AccessBridgeJavaEntryPoints.obj
 0002:00004ac0       ??_C@_0EO@FMBHNIPI@?$FLERROR?$FN?3?5?5either?5env?5?$DN?$DN?50?5or?5ge@ 0000000180016ac0     AccessBridgeJavaEntryPoints.obj
 0002:00004b10       ??_C@_0EK@BLALEJAL@?$FLINFO?$FN?3?5?$CK?$CK?$CK?5jniEnv?3?5?$CFp?$DL?5accessB@ 0000000180016b10     AccessBridgeJavaEntryPoints.obj
 0002:00004b60       ??_C@_0DK@HBEJENLO@Getting?5AccessibleChildrenCount@ 0000000180016b60     AccessBridgeJavaEntryPoints.obj
 0002:00004ba0       ??_C@_0BO@INNKBLPE@?$FLINFO?$FN?3?5?5?5Children?5count?5?$DN?5?$CFd@ 0000000180016ba0     AccessBridgeJavaEntryPoints.obj
 0002:00004bc0       ??_C@_0EO@BPNCCJLD@?$FLERROR?$FN?3?5?5either?5env?5?$DN?$DN?50?5or?5ge@ 0000000180016bc0     AccessBridgeJavaEntryPoints.obj
 0002:00004c10       ??_C@_0EK@PAPEMOFA@?$FLINFO?$FN?3?5?$CK?$CK?$CK?5jniEnv?3?5?$CFp?$DL?5accessB@ 0000000180016c10     AccessBridgeJavaEntryPoints.obj
 0002:00004c60       ??_C@_0DD@EIHALEFK@Getting?5AccessibleXcoord?5?9?5call@ 0000000180016c60     AccessBridgeJavaEntryPoints.obj
 0002:00004c98       ??_C@_0BH@EMDFCPBA@?$FLINFO?$FN?3?5?5?5X?5coord?5?$DN?5?$CFd@ 0000000180016c98     AccessBridgeJavaEntryPoints.obj
 0002:00004cb0       ??_C@_0EH@EAAFBPMN@?$FLERROR?$FN?3?5?5either?5env?5?$DN?$DN?50?5or?5ge@ 0000000180016cb0     AccessBridgeJavaEntryPoints.obj
 0002:00004d00       ??_C@_0EK@PIPPCCAB@?$FLINFO?$FN?3?5?$CK?$CK?$CK?5jniEnv?3?5?$CFX?$DL?5accessB@ 0000000180016d00     AccessBridgeJavaEntryPoints.obj
 0002:00004d50       ??_C@_0DD@HOICCEKJ@Getting?5AccessibleYcoord?5?9?5call@ 0000000180016d50     AccessBridgeJavaEntryPoints.obj
 0002:00004d88       ??_C@_0BH@JBKDPGJF@?$FLINFO?$FN?3?5?5?5Y?5coord?5?$DN?5?$CFd@ 0000000180016d88     AccessBridgeJavaEntryPoints.obj
 0002:00004da0       ??_C@_0EH@CDACMGOJ@?$FLERROR?$FN?3?5?5either?5env?5?$DN?$DN?50?5or?5ge@ 0000000180016da0     AccessBridgeJavaEntryPoints.obj
 0002:00004de8       ??_C@_0DC@IECDLNHB@Getting?5AccessibleWidth?5?9?5call?5@ 0000000180016de8     AccessBridgeJavaEntryPoints.obj
 0002:00004e20       ??_C@_0BF@EEAFCLIB@?$FLINFO?$FN?3?5?5?5Width?5?$DN?5?$CFd@ 0000000180016e20     AccessBridgeJavaEntryPoints.obj
 0002:00004e40       ??_C@_0EG@HOHNFBDJ@?$FLERROR?$FN?3?5?5either?5env?5?$DN?$DN?50?5or?5ge@ 0000000180016e40     AccessBridgeJavaEntryPoints.obj
 0002:00004e88       ??_C@_0DD@DDJGOHAP@Getting?5AccessibleHeight?5?9?5call@ 0000000180016e88     AccessBridgeJavaEntryPoints.obj
 0002:00004ec0       ??_C@_0BG@DJGLJFGH@?$FLINFO?$FN?3?5?5?5Height?5?$DN?5?$CFd@ 0000000180016ec0     AccessBridgeJavaEntryPoints.obj
 0002:00004ee0       ??_C@_0EH@LBBAABEE@?$FLERROR?$FN?3?5?5either?5env?5?$DN?$DN?50?5or?5ge@ 0000000180016ee0     AccessBridgeJavaEntryPoints.obj
 0002:00004f28       ??_C@_0DJ@LNCBBGOH@Getting?5AccessibleComponent?5?9?5c@ 0000000180016f28     AccessBridgeJavaEntryPoints.obj
 0002:00004f68       ??_C@_0CD@PFGFGKFI@?$FLINFO?$FN?3?5?5?5AccessibleComponent?5?$DN@ 0000000180016f68     AccessBridgeJavaEntryPoints.obj
 0002:00004f90       ??_C@_0DH@KGCNAJLL@Getting?5AccessibleComponent?5?9?5c@ 0000000180016f90     AccessBridgeJavaEntryPoints.obj
 0002:00004fd0       ??_C@_0EK@MOFEFKAP@?$FLERROR?$FN?3?5?5either?5env?5?$DN?$DN?50?5or?5ge@ 0000000180016fd0     AccessBridgeJavaEntryPoints.obj
 0002:00005020       ??_C@_0DG@DACOODAE@Getting?5AccessibleAction?5?9?5call@ 0000000180017020     AccessBridgeJavaEntryPoints.obj
 0002:00005058       ??_C@_0CA@PJFDOLN@?$FLINFO?$FN?3?5?5?5AccessibleAction?5?$DN?5?$CFp@ 0000000180017058     AccessBridgeJavaEntryPoints.obj
 0002:00005078       ??_C@_0DE@DDPPAPLP@Getting?5AccessibleAction?5?9?5call@ 0000000180017078     AccessBridgeJavaEntryPoints.obj
 0002:000050b0       ??_C@_0EH@DKLGJNHO@?$FLERROR?$FN?3?5?5either?5env?5?$DN?$DN?50?5or?5ge@ 00000001800170b0     AccessBridgeJavaEntryPoints.obj
 0002:000050f8       ??_C@_0DJ@CGHCFMLP@Getting?5AccessibleSelection?5?9?5c@ 00000001800170f8     AccessBridgeJavaEntryPoints.obj
 0002:00005138       ??_C@_0CD@PJLLNPAJ@?$FLINFO?$FN?3?5?5?5AccessibleSelection?5?$DN@ 0000000180017138     AccessBridgeJavaEntryPoints.obj
 0002:00005160       ??_C@_0DH@PGPODJFA@Getting?5AccessibleSelection?5?9?5c@ 0000000180017160     AccessBridgeJavaEntryPoints.obj
 0002:000051a0       ??_C@_0EK@NDMBIFBF@?$FLERROR?$FN?3?5?5either?5env?5?$DN?$DN?50?5or?5ge@ 00000001800171a0     AccessBridgeJavaEntryPoints.obj
 0002:000051f0       ??_C@_0DO@EELLKHNA@?$FLINFO?$FN?3?5?$CD?$CD?$CD?$CD?$CD?5Calling?5getAccess@ 00000001800171f0     AccessBridgeJavaEntryPoints.obj
 0002:00005230       ??_C@_0EE@BBNKAGDP@?$FLINFO?$FN?3?5?$CD?$CD?$CD?$CD?$CD?5?4?4?4?5Returned?5from@ 0000000180017230     AccessBridgeJavaEntryPoints.obj
 0002:00005278       ??_C@_0DL@DIOKBKHD@?$CD?$CD?$CD?$CD?$CD?5Getting?5AccessibleTable?5?9@ 0000000180017278     AccessBridgeJavaEntryPoints.obj
 0002:000052b8       ??_C@_0CF@KFOMFGJG@?$FLINFO?$FN?3?5?5?5?$CD?$CD?$CD?$CD?$CD?5AccessibleTable@ 00000001800172b8     AccessBridgeJavaEntryPoints.obj
 0002:000052e0       ??_C@_0DJ@ELALBBFD@?$CD?$CD?$CD?$CD?$CD?5Getting?5AccessibleTable?5?9@ 00000001800172e0     AccessBridgeJavaEntryPoints.obj
 0002:00005320       ??_C@_0EF@MKDIKDJP@?$FLERROR?$FN?3?5either?5env?5?$DN?$DN?50?5or?5get@ 0000000180017320     AccessBridgeJavaEntryPoints.obj
 0002:00005368       ??_C@_0BO@PJMPGGKG@?$FLINFO?$FN?3?5?5?5AccessibleText?5?$DN?5?$CFp@ 0000000180017368     AccessBridgeJavaEntryPoints.obj
 0002:00005388       ??_C@_0DF@NJBDDCEL@Getting?5AccessibleValue?5?9?5call?5@ 0000000180017388     AccessBridgeJavaEntryPoints.obj
 0002:000053c0       ??_C@_0BP@BANALONE@?$FLINFO?$FN?3?5?5?5AccessibleValue?5?$DN?5?$CFp@ 00000001800173c0     AccessBridgeJavaEntryPoints.obj
 0002:000053e0       ??_C@_0DD@JJHMAHMH@Getting?5AccessibleValue?5?9?5call?5@ 00000001800173e0     AccessBridgeJavaEntryPoints.obj
 0002:00005420       ??_C@_0EG@HHMGAANK@?$FLERROR?$FN?3?5?5either?5env?5?$DN?$DN?50?5or?5ge@ 0000000180017420     AccessBridgeJavaEntryPoints.obj
 0002:00005468       ??_C@_0DJ@EACHBMMF@Getting?5AccessibleHypertext?5?9?5c@ 0000000180017468     AccessBridgeJavaEntryPoints.obj
 0002:000054a8       ??_C@_0CD@DNELEHHF@?$FLINFO?$FN?3?5?5?5AccessibleHypertext?5?$DN@ 00000001800174a8     AccessBridgeJavaEntryPoints.obj
 0002:000054d0       ??_C@_0DH@DONNNDKC@Getting?5AccessibleHypertext?5?9?5c@ 00000001800174d0     AccessBridgeJavaEntryPoints.obj
 0002:00005510       ??_C@_0FA@DGBOEHHP@?$FLINFO?$FN?3?5Calling?5AccessBridgeJav@ 0000000180017510     AccessBridgeJavaEntryPoints.obj
 0002:00005560       ??_C@_0DF@OGEEIIFE@Getting?5AccessibleChild?5?9?5call?5@ 0000000180017560     AccessBridgeJavaEntryPoints.obj
 0002:00005598       ??_C@_0DB@OOCPCHE@Getting?5AccessibleChild?5?9?5call?5@ 0000000180017598     AccessBridgeJavaEntryPoints.obj
 0002:000055d0       ??_C@_0DD@JNMELFAO@Getting?5AccessibleChild?5?9?5call?5@ 00000001800175d0     AccessBridgeJavaEntryPoints.obj
 0002:00005610       ??_C@_0EC@MDNHELGM@?$FLERROR?$FN?3?5?5either?5env?5?$DN?$DN?50?5or?5ge@ 0000000180017610     AccessBridgeJavaEntryPoints.obj
 0002:00005660       ??_C@_0FB@PNLEIBEF@?$FLINFO?$FN?3?5Calling?5AccessBridgeJav@ 0000000180017660     AccessBridgeJavaEntryPoints.obj
 0002:000056b8       ??_C@_0DG@BJCEEHCN@Getting?5AccessibleParent?5?9?5call@ 00000001800176b8     AccessBridgeJavaEntryPoints.obj
 0002:000056f0       ??_C@_0DC@MKLJMCBC@Getting?5AccessibleParent?5?9?5call@ 00000001800176f0     AccessBridgeJavaEntryPoints.obj
 0002:00005728       ??_C@_0DE@IILKINNI@Getting?5AccessibleParent?5?9?5call@ 0000000180017728     AccessBridgeJavaEntryPoints.obj
 0002:00005760       ??_C@_0EH@MOCAMKEC@?$FLERROR?$FN?3?5?5either?5env?5?$DN?$DN?50?5or?5ge@ 0000000180017760     AccessBridgeJavaEntryPoints.obj
 0002:000057b0       ??_C@_0EP@IDGNPODK@?$FLINFO?$FN?3?5?$CD?$CD?$CD?$CD?$CD?5Calling?5AccessBri@ 00000001800177b0     AccessBridgeJavaEntryPoints.obj
 0002:00005800       ??_C@_0EA@HDPDLION@?$CD?$CD?$CD?$CD?$CD?5Getting?5AccessibleTableRo@ 0000000180017800     AccessBridgeJavaEntryPoints.obj
 0002:00005840       ??_C@_0CF@OMEBMMOI@?$FLINFO?$FN?3?5?5?5?$CD?$CD?$CD?$CD?$CD?5table?5row?5count@ 0000000180017840     AccessBridgeJavaEntryPoints.obj
 0002:00005868       ??_C@_0DN@MNMKPHBJ@?$FLERROR?$FN?3?5either?5env?5?$DN?$DN?50?5or?5get@ 0000000180017868     AccessBridgeJavaEntryPoints.obj
 0002:000058a8       ??_C@_0DN@LHDBHOOP@Getting?5AccessibleTableColumnCo@ 00000001800178a8     AccessBridgeJavaEntryPoints.obj
 0002:000058e8       ??_C@_0CI@GJGENPPF@?$FLINFO?$FN?3?5?5?5?$CD?$CD?$CD?$CD?$CD?5table?5column?5co@ 00000001800178e8     AccessBridgeJavaEntryPoints.obj
 0002:00005910       ??_C@_0EF@LHBDGBA@?$FLERROR?$FN?3?5either?5env?5?$DN?$DN?50?5or?5get@ 0000000180017910     AccessBridgeJavaEntryPoints.obj
 0002:00005958       ??_C@_0DH@GFGBCDOC@?$CD?$CD?$CD?$CD?$CD?5Getting?5AccessibleTable?5?9@ 0000000180017958     AccessBridgeJavaEntryPoints.obj
 0002:00005990       ??_C@_0CF@DCCEHDEO@?$FLINFO?$FN?3?5?5?5?$CD?$CD?$CD?$CD?$CD?5accessibleTable@ 0000000180017990     AccessBridgeJavaEntryPoints.obj
 0002:000059b8       ??_C@_0DP@FLHLIILD@?$FLINFO?$FN?3?5?$CD?$CD?$CD?$CD?$CD?5Calling?5getContex@ 00000001800179b8     AccessBridgeJavaEntryPoints.obj
 0002:00005a00       ??_C@_0EF@JOJDMPNM@?$FLINFO?$FN?3?5?$CD?$CD?$CD?$CD?$CD?5?4?4?4?5Returned?5from@ 0000000180017a00     AccessBridgeJavaEntryPoints.obj
 0002:00005a48       ??_C@_0CH@GEKEKGKL@?$FLINFO?$FN?3?5?5?5?$CD?$CD?$CD?$CD?$CD?5accessibleConte@ 0000000180017a48     AccessBridgeJavaEntryPoints.obj
 0002:00005a70       ??_C@_0EG@CNEBJJDJ@?$FLERROR?$FN?3?5either?5env?5?$DN?$DN?50?5or?5get@ 0000000180017a70     AccessBridgeJavaEntryPoints.obj
 0002:00005ac0       ??_C@_0FE@GFOFNDOE@?$FLINFO?$FN?3?5?$CD?$CD?$CD?$CD?$CD?5Calling?5AccessBri@ 0000000180017ac0     AccessBridgeJavaEntryPoints.obj
 0002:00005b20       ??_C@_0GF@GDALOMIB@?$FLINFO?$FN?3?5?$CD?$CD?$CD?$CD?$CD?5Calling?5AccessBri@ 0000000180017b20     AccessBridgeJavaEntryPoints.obj
 0002:00005b90       ??_C@_0EB@IFJOCDDE@?$CD?$CD?$CD?$CD?$CD?5Getting?5AccessibleTableCe@ 0000000180017b90     AccessBridgeJavaEntryPoints.obj
 0002:00005bd8       ??_C@_0CG@KKOMOEPJ@?$FLINFO?$FN?3?5?5?5?$CD?$CD?$CD?$CD?$CD?5table?5cell?5inde@ 0000000180017bd8     AccessBridgeJavaEntryPoints.obj
 0002:00005c00       ??_C@_0ED@MJPDAFIJ@?$FLERROR?$FN?3?5either?5env?5?$DN?$DN?50?5or?5get@ 0000000180017c00     AccessBridgeJavaEntryPoints.obj
 0002:00005c50       ??_C@_0EK@HFAIKGKI@?$CD?$CD?$CD?$CD?$CD?5Getting?5AccessibleTableCe@ 0000000180017c50     AccessBridgeJavaEntryPoints.obj
 0002:00005ca0       ??_C@_0CL@CDCOGIJD@?$FLINFO?$FN?3?5?5?5?$CD?$CD?$CD?$CD?$CD?5table?5cell?5row?5@ 0000000180017ca0     AccessBridgeJavaEntryPoints.obj
 0002:00005cd0       ??_C@_0EH@MFABNFMJ@?$FLERROR?$FN?3?5either?5env?5?$DN?$DN?50?5or?5get@ 0000000180017cd0     AccessBridgeJavaEntryPoints.obj
 0002:00005d20       ??_C@_0EN@GIPGNDGO@?$CD?$CD?$CD?$CD?$CD?5Getting?5AccessibleTableCe@ 0000000180017d20     AccessBridgeJavaEntryPoints.obj
 0002:00005d70       ??_C@_0CN@JHPAHOLB@?$FLINFO?$FN?3?5?5?$CD?$CD?$CD?$CD?$CD?5table?5cell?5colum@ 0000000180017d70     AccessBridgeJavaEntryPoints.obj
 0002:00005da0       ??_C@_0EK@MCJJFMIG@?$FLERROR?$FN?3?5either?5env?5?$DN?$DN?50?5or?5get@ 0000000180017da0     AccessBridgeJavaEntryPoints.obj
 0002:00005df0       ??_C@_0EK@OAKDMNFI@?$CD?$CD?$CD?$CD?$CD?5Getting?5isAccessibleTable@ 0000000180017df0     AccessBridgeJavaEntryPoints.obj
 0002:00005e40       ??_C@_0CL@FGJJGBAG@?$FLINFO?$FN?3?5?5?5?$CD?$CD?$CD?$CD?$CD?5table?5cell?5isSe@ 0000000180017e40     AccessBridgeJavaEntryPoints.obj
 0002:00005e70       ??_C@_0EF@NDHLMIOL@?$FLERROR?$FN?3?5either?5env?5?$DN?$DN?50?5or?5isA@ 0000000180017e70     AccessBridgeJavaEntryPoints.obj
 0002:00005ec0       ??_C@_0FA@PNFLEDNO@?$CD?$CD?$CD?$CD?$CD?5Getting?5AccessibleTableCe@ 0000000180017ec0     AccessBridgeJavaEntryPoints.obj
 0002:00005f10       ??_C@_0EM@CCOLAKIM@?$CD?$CD?$CD?$CD?$CD?5Getting?5AccessibleTableCe@ 0000000180017f10     AccessBridgeJavaEntryPoints.obj
 0002:00005f60       ??_C@_0DC@NHIEBBHC@?$FLINFO?$FN?3?5?5?5?$CD?$CD?$CD?$CD?$CD?5table?5cell?5Acce@ 0000000180017f60     AccessBridgeJavaEntryPoints.obj
 0002:00005fa0       ??_C@_0EP@BAKELAEL@?$FLERROR?$FN?3?5either?5env?5?$DN?$DN?50?5or?5get@ 0000000180017fa0     AccessBridgeJavaEntryPoints.obj
 0002:00005ff0       ??_C@_0FJ@JCFFKNHH@?$FLINFO?$FN?3?5?5?$CD?$CD?$CD?$CD?$CD?5Calling?5AccessBr@ 0000000180017ff0     AccessBridgeJavaEntryPoints.obj
 0002:00006050       ??_C@_0FE@DGILOPPB@?$FLINFO?$FN?3?5?$CD?$CD?$CD?$CD?$CD?5Calling?5AccessBri@ 0000000180018050     AccessBridgeJavaEntryPoints.obj
 0002:000060b0       ??_C@_0EJ@OONHAJKO@?$CD?$CD?$CD?$CD?$CD?5Getting?5AccessibleTableRo@ 00000001800180b0     AccessBridgeJavaEntryPoints.obj
 0002:00006100       ??_C@_0EG@NDBCAEFO@?$FLERROR?$FN?3?5either?5env?5?$DN?$DN?50?5or?5get@ 0000000180018100     AccessBridgeJavaEntryPoints.obj
 0002:00006150       ??_C@_0EG@DALLPPNJ@Getting?5AccessibleTableRowHeade@ 0000000180018150     AccessBridgeJavaEntryPoints.obj
 0002:000061a0       ??_C@_0EO@OOHGOEEK@?$FLERROR?$FN?3?5either?5env?5?$DN?$DN?50?5or?5get@ 00000001800181a0     AccessBridgeJavaEntryPoints.obj
 0002:000061f0       ??_C@_0EE@GCIECGJK@?$CD?$CD?$CD?$CD?$CD?5Getting?5AccessibleTableRo@ 00000001800181f0     AccessBridgeJavaEntryPoints.obj
 0002:00006240       ??_C@_0EA@OEOKKCMN@?$CD?$CD?$CD?$CD?$CD?5Getting?5AccessibleTableRo@ 0000000180018240     AccessBridgeJavaEntryPoints.obj
 0002:00006280       ??_C@_0DA@BEAKBEEG@?$FLINFO?$FN?3?5?5?5?$CD?$CD?$CD?$CD?$CD?5row?5header?5Acce@ 0000000180018280     AccessBridgeJavaEntryPoints.obj
 0002:000062b0       ??_C@_0ED@KKINKAGC@?$FLERROR?$FN?3?5either?5env?5?$DN?$DN?50?5or?5get@ 00000001800182b0     AccessBridgeJavaEntryPoints.obj
 0002:00006300       ??_C@_0FL@PPBJDPIL@?$FLINFO?$FN?3?5?5?5?$CD?$CD?$CD?$CD?$CD?5Calling?5AccessB@ 0000000180018300     AccessBridgeJavaEntryPoints.obj
 0002:00006360       ??_C@_0FH@EJOHBEGH@?$FLINFO?$FN?3?5?$CD?$CD?$CD?$CD?$CD?5Calling?5AccessBri@ 0000000180018360     AccessBridgeJavaEntryPoints.obj
 0002:000063c0       ??_C@_0EM@ILKGOFLG@?$CD?$CD?$CD?$CD?$CD?5Getting?5AccessibleTableCo@ 00000001800183c0     AccessBridgeJavaEntryPoints.obj
 0002:00006410       ??_C@_0EK@LPGMLANE@?$FLERROR?$FN?3?5?5either?5env?5?$DN?$DN?50?5or?5ge@ 0000000180018410     AccessBridgeJavaEntryPoints.obj
 0002:00006460       ??_C@_0EJ@CKEIFDID@Getting?5AccessibleTableColumnHe@ 0000000180018460     AccessBridgeJavaEntryPoints.obj
 0002:000064b0       ??_C@_0FB@LHNIAEHP@?$FLERROR?$FN?3?5either?5env?5?$DN?$DN?50?5or?5get@ 00000001800184b0     AccessBridgeJavaEntryPoints.obj
 0002:00006510       ??_C@_0EH@JIOGAIC@?$CD?$CD?$CD?$CD?$CD?5Getting?5AccessibleTableCo@ 0000000180018510     AccessBridgeJavaEntryPoints.obj
 0002:00006560       ??_C@_0ED@DCBGPFPL@?$CD?$CD?$CD?$CD?$CD?5Getting?5AccessibleTableCo@ 0000000180018560     AccessBridgeJavaEntryPoints.obj
 0002:000065a8       ??_C@_0DD@JPNBDACB@?$FLINFO?$FN?3?5?5?5?$CD?$CD?$CD?$CD?$CD?5column?5header?5A@ 00000001800185a8     AccessBridgeJavaEntryPoints.obj
 0002:000065e0       ??_C@_0EG@EHCJNLHA@?$FLERROR?$FN?3?5either?5env?5?$DN?$DN?50?5or?5get@ 00000001800185e0     AccessBridgeJavaEntryPoints.obj
 0002:00006630       ??_C@_0FO@DKAHOFOA@?$FLINFO?$FN?3?5?5?5?$CD?$CD?$CD?$CD?$CD?5Calling?5AccessB@ 0000000180018630     AccessBridgeJavaEntryPoints.obj
 0002:00006690       ??_C@_0FJ@IPEPPO@?$FLINFO?$FN?3?5?$CD?$CD?$CD?$CD?$CD?5Calling?5AccessBri@ 0000000180018690     AccessBridgeJavaEntryPoints.obj
 0002:000066f0       ??_C@_0ED@ECGPKBKB@Getting?5AccessibleTableRowDescr@ 00000001800186f0     AccessBridgeJavaEntryPoints.obj
 0002:00006738       ??_C@_0DP@MGPIFPGE@Getting?5AccessibleTableRowDescr@ 0000000180018738     AccessBridgeJavaEntryPoints.obj
 0002:00006780       ??_C@_0EB@HPGBLABA@Getting?5AccessibleTableRowDescr@ 0000000180018780     AccessBridgeJavaEntryPoints.obj
 0002:000067d0       ??_C@_0EI@FALMFIJI@?$FLERROR?$FN?3?5either?5env?5?$DN?$DN?50?5or?5get@ 00000001800187d0     AccessBridgeJavaEntryPoints.obj
 0002:00006820       ??_C@_0FM@OGMEFLJF@?$FLINFO?$FN?3?5?$CD?$CD?$CD?$CD?$CD?5Calling?5AccessBri@ 0000000180018820     AccessBridgeJavaEntryPoints.obj
 0002:00006880       ??_C@_0EG@HNHAKGAA@Getting?5AccessibleTableColumnDe@ 0000000180018880     AccessBridgeJavaEntryPoints.obj
 0002:000068d0       ??_C@_0EC@OOIBKPKB@Getting?5AccessibleTableColumnDe@ 00000001800188d0     AccessBridgeJavaEntryPoints.obj
 0002:00006920       ??_C@_0EE@HEFBEJHO@Getting?5AccessibleTableColumnDe@ 0000000180018920     AccessBridgeJavaEntryPoints.obj
 0002:00006970       ??_C@_0EL@MDADMDPK@?$FLERROR?$FN?3?5either?5env?5?$DN?$DN?50?5or?5get@ 0000000180018970     AccessBridgeJavaEntryPoints.obj
 0002:000069c0       ??_C@_0FD@NONCILOI@?$FLINFO?$FN?3?5?$CD?$CD?$CD?$CD?$CD?5AccessBridgeJavaE@ 00000001800189c0     AccessBridgeJavaEntryPoints.obj
 0002:00006a20       ??_C@_0EJ@CONOFLFI@?$CD?$CD?$CD?$CD?$CD?5Getting?5AccessibleTableRo@ 0000000180018a20     AccessBridgeJavaEntryPoints.obj
 0002:00006a70       ??_C@_0CP@GJAEEGNO@?$FLINFO?$FN?3?5?5?5?$CD?$CD?$CD?$CD?$CD?5table?5row?5selec@ 0000000180018a70     AccessBridgeJavaEntryPoints.obj
 0002:00006aa0       ??_C@_0EL@JIBDDMIF@?$FLERROR?$FN?3?5either?5env?5?$DN?$DN?50?5or?5get@ 0000000180018aa0     AccessBridgeJavaEntryPoints.obj
 0002:00006af0       ??_C@_0FA@LAKDEELL@?$FLINFO?$FN?3?5?$CD?$CD?$CD?$CD?$CD?5AccessBridgeJavaE@ 0000000180018af0     AccessBridgeJavaEntryPoints.obj
 0002:00006b40       ??_C@_0EJ@PAIANDP@?$CD?$CD?$CD?$CD?$CD?5Getting?5isAccessibleTable@ 0000000180018b40     AccessBridgeJavaEntryPoints.obj
 0002:00006b90       ??_C@_0CK@ENCKDAKJ@?$FLINFO?$FN?3?5?5?5?$CD?$CD?$CD?$CD?$CD?5table?5row?5isSel@ 0000000180018b90     AccessBridgeJavaEntryPoints.obj
 0002:00006bc0       ??_C@_0EE@OPDECGCG@?$FLERROR?$FN?3?5either?5env?5?$DN?$DN?50?5or?5isA@ 0000000180018bc0     AccessBridgeJavaEntryPoints.obj
 0002:00006c10       ??_C@_0FG@BNGDNOAB@?$FLINFO?$FN?3?5?$CD?$CD?$CD?$CD?$CD?5AccessBridgeJavaE@ 0000000180018c10     AccessBridgeJavaEntryPoints.obj
 0002:00006c70       ??_C@_0EF@MANEDMPN@?$CD?$CD?$CD?$CD?$CD?5Getting?5AccessibleTableRo@ 0000000180018c70     AccessBridgeJavaEntryPoints.obj
 0002:00006cb8       ??_C@_0CN@EGDPALEC@?$FLINFO?$FN?3?5?5?5?$CD?$CD?$CD?$CD?$CD?5table?5row?5selec@ 0000000180018cb8     AccessBridgeJavaEntryPoints.obj
 0002:00006cf0       ??_C@_0FH@IBIGBELL@?$FLINFO?$FN?3?5?5?5?$CD?$CD?$CD?$CD?$CD?5AccessBridgeJav@ 0000000180018cf0     AccessBridgeJavaEntryPoints.obj
 0002:00006d50       ??_C@_0FG@LAILABJF@?$FLINFO?$FN?3?5?$CD?$CD?$CD?$CD?$CD?5AccessBridgeJavaE@ 0000000180018d50     AccessBridgeJavaEntryPoints.obj
 0002:00006db0       ??_C@_0EM@ELKPLHEA@?$CD?$CD?$CD?$CD?$CD?5Getting?5AccessibleTableCo@ 0000000180018db0     AccessBridgeJavaEntryPoints.obj
 0002:00006e00       ??_C@_0DC@EFKBJLFF@?$FLINFO?$FN?3?5?5?5?$CD?$CD?$CD?$CD?$CD?5table?5column?5se@ 0000000180018e00     AccessBridgeJavaEntryPoints.obj
 0002:00006e40       ??_C@_0FD@ODFPPIDD@?$FLINFO?$FN?3?5?$CD?$CD?$CD?$CD?$CD?5AccessBridgeJavaE@ 0000000180018e40     AccessBridgeJavaEntryPoints.obj
 0002:00006ea0       ??_C@_0EM@HPIPAKED@?$CD?$CD?$CD?$CD?$CD?5Getting?5isAccessibleTable@ 0000000180018ea0     AccessBridgeJavaEntryPoints.obj
 0002:00006ef0       ??_C@_0CN@OPIEHDOO@?$FLINFO?$FN?3?5?5?5?$CD?$CD?$CD?$CD?$CD?5table?5column?5is@ 0000000180018ef0     AccessBridgeJavaEntryPoints.obj
 0002:00006f20       ??_C@_0EI@CBBNNOEE@?$FLERROR?$FN?3?5?5either?5env?5?$DN?$DN?50?5or?5is@ 0000000180018f20     AccessBridgeJavaEntryPoints.obj
 0002:00006f70       ??_C@_0FK@KHEECFFC@?$FLINFO?$FN?3?5?$CD?$CD?$CD?$CD?$CD?5AccessBridgeJavaE@ 0000000180018f70     AccessBridgeJavaEntryPoints.obj
 0002:00006fd0       ??_C@_0EI@NDNDKOON@?$CD?$CD?$CD?$CD?$CD?5Getting?5AccessibleTableCo@ 0000000180018fd0     AccessBridgeJavaEntryPoints.obj
 0002:00007018       ??_C@_0DA@FGAFLCDN@?$FLINFO?$FN?3?5?5?5?$CD?$CD?$CD?$CD?$CD?5table?5Column?5se@ 0000000180019018     AccessBridgeJavaEntryPoints.obj
 0002:00007050       ??_C@_0FK@PECCMPIL@?$FLINFO?$FN?3?5?5?5?$CD?$CD?$CD?$CD?$CD?5AccessBridgeJav@ 0000000180019050     AccessBridgeJavaEntryPoints.obj
 0002:000070b0       ??_C@_0EP@DEKNIMFA@?$FLINFO?$FN?3?5?$CD?$CD?$CD?$CD?$CD?5AccessBridgeJavaE@ 00000001800190b0     AccessBridgeJavaEntryPoints.obj
 0002:00007100       ??_C@_0DL@DELNDLCL@?$CD?$CD?$CD?$CD?$CD?5Getting?5AccessibleTableRo@ 0000000180019100     AccessBridgeJavaEntryPoints.obj
 0002:00007140       ??_C@_0BP@MEJOIGMM@?$FLINFO?$FN?3?5?5?5?$CD?$CD?$CD?$CD?$CD?5table?5row?5?$DN?5?$CFd@ 0000000180019140     AccessBridgeJavaEntryPoints.obj
 0002:00007160       ??_C@_0DN@DIFOEGJK@?$FLERROR?$FN?3?5either?5env?5?$DN?$DN?50?5or?5get@ 0000000180019160     AccessBridgeJavaEntryPoints.obj
 0002:000071a0       ??_C@_0FC@BFBAOEGI@?$FLINFO?$FN?3?5?$CD?$CD?$CD?$CD?$CD?5AccessBridgeJavaE@ 00000001800191a0     AccessBridgeJavaEntryPoints.obj
 0002:000071f8       ??_C@_0DO@MBGEOOOH@?$CD?$CD?$CD?$CD?$CD?5Getting?5AccessibleTableCo@ 00000001800191f8     AccessBridgeJavaEntryPoints.obj
 0002:00007238       ??_C@_0CC@CJBEHFKG@?$FLINFO?$FN?3?5?5?5?$CD?$CD?$CD?$CD?$CD?5table?5column?5?$DN?5@ 0000000180019238     AccessBridgeJavaEntryPoints.obj
 0002:00007260       ??_C@_0EA@IFBLPNLC@?$FLERROR?$FN?3?5either?5env?5?$DN?$DN?50?5or?5get@ 0000000180019260     AccessBridgeJavaEntryPoints.obj
 0002:000072a0       ??_C@_0FH@GMMGKHHK@?$FLINFO?$FN?3?5?$CD?$CD?$CD?$CD?$CD?5AccessBridgeJavaE@ 00000001800192a0     AccessBridgeJavaEntryPoints.obj
 0002:00007300       ??_C@_0EA@IDLLLJIK@?$CD?$CD?$CD?$CD?$CD?5Getting?5getAccessibleTabl@ 0000000180019300     AccessBridgeJavaEntryPoints.obj
 0002:00007340       ??_C@_0CB@JIHDIDBK@?$FLINFO?$FN?3?5?5?5?$CD?$CD?$CD?$CD?$CD?5table?5index?5?$DN?5?$CF@ 0000000180019340     AccessBridgeJavaEntryPoints.obj
 0002:00007368       ??_C@_0DP@EPGMKJOF@?$FLERROR?$FN?3?5either?5env?5?$DN?$DN?50?5or?5get@ 0000000180019368     AccessBridgeJavaEntryPoints.obj
 0002:000073b0       ??_C@_0EM@OMNMKDMF@?$FLINFO?$FN?3?5?$CD?$CD?$CD?$CD?$CD?5AccessBridgeJavaE@ 00000001800193b0     AccessBridgeJavaEntryPoints.obj
 0002:00007400       ??_C@_0EA@LPBOBAAO@?$CD?$CD?$CD?$CD?$CD?5Getting?5AccessibleRelatio@ 0000000180019400     AccessBridgeJavaEntryPoints.obj
 0002:00007440       ??_C@_0CO@JNBGELMK@?$FLINFO?$FN?3?5?5?5?$CD?$CD?$CD?$CD?$CD?5AccessibleRelat@ 0000000180019440     AccessBridgeJavaEntryPoints.obj
 0002:00007470       ??_C@_0DL@KJPPMLJK@Getting?5AccessibleRelationKey?5?9@ 0000000180019470     AccessBridgeJavaEntryPoints.obj
 0002:000074b0       ??_C@_0DK@CJPLLCPL@Getting?5AccessibleRelation?5key?5@ 00000001800194b0     AccessBridgeJavaEntryPoints.obj
 0002:000074f0       ??_C@_0BP@LFNNPMOI@Getting?5AccessibleRelation?5key@ 00000001800194f0     AccessBridgeJavaEntryPoints.obj
 0002:00007510       ??_C@_0CL@LKNHIIFA@?$FLINFO?$FN?3?5?$CD?$CD?$CD?$CD?$CD?5AccessibleRelatio@ 0000000180019510     AccessBridgeJavaEntryPoints.obj
 0002:00007540       ??_C@_0DK@OHAOHAGF@Getting?5AccessibleRelation?5key?5@ 0000000180019540     AccessBridgeJavaEntryPoints.obj
 0002:00007580       ??_C@_0CK@FLLDFIHJ@?$FLWARN?$FN?3?5?5?5AccessibleRelation?5ke@ 0000000180019580     AccessBridgeJavaEntryPoints.obj
 0002:000075b0       ??_C@_0DL@FOJGEEOM@Getting?5AccessibleRelationSet?5?9@ 00000001800195b0     AccessBridgeJavaEntryPoints.obj
 0002:000075f0       ??_C@_0DH@OOCHFOKL@Getting?5AccessibleRelationSet?5?9@ 00000001800195f0     AccessBridgeJavaEntryPoints.obj
 0002:00007628       ??_C@_0CA@NHODALDJ@?$FLINFO?$FN?3?5?5?5relation?5set?5item?3?5?$CFp@ 0000000180019628     AccessBridgeJavaEntryPoints.obj
 0002:00007650       ??_C@_0FA@NBCFFMGI@?$FLINFO?$FN?3?5?5?5?$CD?$CD?$CD?$CD?$CD?5AccessBridgeJav@ 0000000180019650     AccessBridgeJavaEntryPoints.obj
 0002:000076a0       ??_C@_0EK@KKPLDFBH@?$FLINFO?$FN?3?5?$CD?$CD?$CD?$CD?$CD?5AccessBridgeJavaE@ 00000001800196a0     AccessBridgeJavaEntryPoints.obj
 0002:000076f0       ??_C@_0DP@KAHCJAMC@?$CD?$CD?$CD?$CD?$CD?5Getting?5AccessibleHyperte@ 00000001800196f0     AccessBridgeJavaEntryPoints.obj
 0002:00007730       ??_C@_0DL@BCGGEGFO@?$CD?$CD?$CD?$CD?$CD?5Getting?5AccessibleHyperte@ 0000000180019730     AccessBridgeJavaEntryPoints.obj
 0002:00007770       ??_C@_0CJ@KAIOACGL@?$FLINFO?$FN?3?5?5?5?$CD?$CD?$CD?$CD?$CD?5AccessibleHyper@ 0000000180019770     AccessBridgeJavaEntryPoints.obj
 0002:000077a0       ??_C@_0DK@IMJHJIPP@?$FLWARN?$FN?3?5?5?5?$CD?$CD?$CD?$CD?$CD?5null?5Accessible@ 00000001800197a0     AccessBridgeJavaEntryPoints.obj
 0002:000077e0       ??_C@_0DI@FEBHIMOE@?$CD?$CD?$CD?$CD?$CD?5Getting?5hyperlink?5count?5?9@ 00000001800197e0     AccessBridgeJavaEntryPoints.obj
 0002:00007818       ??_C@_0CF@OFPNIMKK@?$FLINFO?$FN?3?5?5?5?$CD?$CD?$CD?$CD?$CD?5hyperlink?5count@ 0000000180019818     AccessBridgeJavaEntryPoints.obj
 0002:00007840       ??_C@_0DP@CIGIOMPM@?$CD?$CD?$CD?$CD?$CD?5Getting?5AccessibleHyperli@ 0000000180019840     AccessBridgeJavaEntryPoints.obj
 0002:00007880       ??_C@_0DL@PDIOCHOJ@?$CD?$CD?$CD?$CD?$CD?5Getting?5AccessibleHyperli@ 0000000180019880     AccessBridgeJavaEntryPoints.obj
 0002:000078c0       ??_C@_0CJ@FJIBOEOI@?$FLINFO?$FN?3?5?5?5?$CD?$CD?$CD?$CD?$CD?5AccessibleHyper@ 00000001800198c0     AccessBridgeJavaEntryPoints.obj
 0002:000078f0       ??_C@_0DE@FAMBBMPD@Getting?5hyperlink?5text?5?9?5call?5t@ 00000001800198f0     AccessBridgeJavaEntryPoints.obj
 0002:00007928       ??_C@_0DM@FFPIAIEA@Getting?5AccessibleHyperlink?5tex@ 0000000180019928     AccessBridgeJavaEntryPoints.obj
 0002:00007968       ??_C@_0CB@GINGGJOG@Getting?5AccessibleHyperlink?5tex@ 0000000180019968     AccessBridgeJavaEntryPoints.obj
 0002:00007990       ??_C@_0CN@IIHGCCLN@?$FLINFO?$FN?3?5?$CD?$CD?$CD?$CD?$CD?5AccessibleHyperli@ 0000000180019990     AccessBridgeJavaEntryPoints.obj
 0002:000079c0       ??_C@_0DM@JLANMKNO@Getting?5AccessibleHyperlink?5tex@ 00000001800199c0     AccessBridgeJavaEntryPoints.obj
 0002:00007a00       ??_C@_0CM@DKPAOLF@?$FLWARN?$FN?3?5?5?5AccessibleHyperlink?5t@ 0000000180019a00     AccessBridgeJavaEntryPoints.obj
 0002:00007a30       ??_C@_0DO@DJICJOGB@?$CD?$CD?$CD?$CD?$CD?5Getting?5hyperlink?5start?5i@ 0000000180019a30     AccessBridgeJavaEntryPoints.obj
 0002:00007a70       ??_C@_0CL@GNKIIEKN@?$FLINFO?$FN?3?5?5?5?$CD?$CD?$CD?$CD?$CD?5hyperlink?5start@ 0000000180019a70     AccessBridgeJavaEntryPoints.obj
 0002:00007aa0       ??_C@_0DM@MGHLFEBK@?$CD?$CD?$CD?$CD?$CD?5Getting?5hyperlink?5end?5ind@ 0000000180019aa0     AccessBridgeJavaEntryPoints.obj
 0002:00007ae0       ??_C@_0CJ@POHPAAGA@?$FLINFO?$FN?3?5?5?5?$CD?$CD?$CD?$CD?$CD?5hyperlink?5end?5i@ 0000000180019ae0     AccessBridgeJavaEntryPoints.obj
 0002:00007b10       ??_C@_0EO@MCEJOGLJ@?$FLINFO?$FN?3?5?5?5?$CD?$CD?$CD?$CD?$CD?5AccessBridgeJav@ 0000000180019b10     AccessBridgeJavaEntryPoints.obj
 0002:00007b60       ??_C@_0FC@PJEJEFPL@?$FLINFO?$FN?3?5Calling?5AccessBridgeJav@ 0000000180019b60     AccessBridgeJavaEntryPoints.obj
 0002:00007bb8       ??_C@_0DK@IAFPEHK@activateAccessibleHyperlink?5?9?5c@ 0000000180019bb8     AccessBridgeJavaEntryPoints.obj
 0002:00007c00       ??_C@_0EG@NBDJGANF@?$FLERROR?$FN?3?5either?5jniEnv?5?$DN?$DN?50?5or?5@ 0000000180019c00     AccessBridgeJavaEntryPoints.obj
 0002:00007c50       ??_C@_0FO@LCEKGOMG@?$FLINFO?$FN?3?5?$CD?$CD?$CD?$CD?$CD?5AccessBridgeJavaE@ 0000000180019c50     AccessBridgeJavaEntryPoints.obj
 0002:00007cb0       ??_C@_0CD@FKJEEIHP@?$FLINFO?$FN?3?5?5?5getting?5hyperlink?5?$CFd?5@ 0000000180019cb0     AccessBridgeJavaEntryPoints.obj
 0002:00007ce0       ??_C@_0FB@LIBMBPHJ@?$FLINFO?$FN?3?5?5?5?$CD?$CD?$CD?$CD?$CD?5AccessBridgeJav@ 0000000180019ce0     AccessBridgeJavaEntryPoints.obj
 0002:00007d40       ??_C@_0EL@OJOFGNCE@?$FLINFO?$FN?3?5?$CD?$CD?$CD?$CD?$CD?5AccessBridgeJavaE@ 0000000180019d40     AccessBridgeJavaEntryPoints.obj
 0002:00007d90       ??_C@_0FL@JFFPJPNI@?$FLINFO?$FN?3?5?$CD?$CD?$CD?$CD?$CD?5AccessBridgeJavaE@ 0000000180019d90     AccessBridgeJavaEntryPoints.obj
 0002:00007df0       ??_C@_0DI@MNABDACM@?$CD?$CD?$CD?$CD?$CD?5Getting?5hyperlink?5index?5?9@ 0000000180019df0     AccessBridgeJavaEntryPoints.obj
 0002:00007e28       ??_C@_0CF@MJOBJPAA@?$FLINFO?$FN?3?5?5?5?$CD?$CD?$CD?$CD?$CD?5hyperlink?5index@ 0000000180019e28     AccessBridgeJavaEntryPoints.obj
 0002:00007e50       ??_C@_0FC@MDIFEEKA@?$FLINFO?$FN?3?5?$CD?$CD?$CD?$CD?$CD?5AccessBridgeJavaE@ 0000000180019e50     AccessBridgeJavaEntryPoints.obj
 0002:00007eb0       ??_C@_0EM@DFNHGKKP@?$FLINFO?$FN?3?5?$CD?$CD?$CD?$CD?$CD?5AccessBridgeJavaE@ 0000000180019eb0     AccessBridgeJavaEntryPoints.obj
 0002:00007f00       ??_C@_0DL@CLKJJKNH@?$CD?$CD?$CD?$CD?$CD?5Getting?5key?5bindings?5coun@ 0000000180019f00     AccessBridgeJavaEntryPoints.obj
 0002:00007f40       ??_C@_0CI@OKJNHPKA@?$FLINFO?$FN?3?5?5?5?$CD?$CD?$CD?$CD?$CD?5key?5bindings?5co@ 0000000180019f40     AccessBridgeJavaEntryPoints.obj
 0002:00007f68       ??_C@_0DP@FMCKMBKC@?$CD?$CD?$CD?$CD?$CD?5Getting?5key?5binding?5chara@ 0000000180019f68     AccessBridgeJavaEntryPoints.obj
 0002:00007fb0       ??_C@_0FN@DCEDCNML@?$FLINFO?$FN?3?5?5?5?$CD?$CD?$CD?$CD?$CD?5key?5binding?5cha@ 0000000180019fb0     AccessBridgeJavaEntryPoints.obj
 0002:00008010       ??_C@_0DO@HKGJEFDO@?$CD?$CD?$CD?$CD?$CD?5Getting?5key?5binding?5modif@ 000000018001a010     AccessBridgeJavaEntryPoints.obj
 0002:00008050       ??_C@_0CK@OFBJGPDI@?$FLINFO?$FN?3?5?5?$CD?$CD?$CD?$CD?$CD?5key?5binding?5modi@ 000000018001a050     AccessBridgeJavaEntryPoints.obj
 0002:00008080       ??_C@_0EG@MKCABNJD@?$FLINFO?$FN?3?5?$CD?$CD?$CD?$CD?$CD?5AccessBridgeJavaE@ 000000018001a080     AccessBridgeJavaEntryPoints.obj
 0002:000080c8       ??_C@_0CG@IDHCCFPM@?$FLWARN?$FN?3?5?5?5?$CD?$CD?$CD?$CD?$CD?5missing?5method?$CI@ 000000018001a0c8     AccessBridgeJavaEntryPoints.obj
 0002:000080f0       ??_C@_0DE@JDHACCPK@?$CD?$CD?$CD?$CD?$CD?5Getting?5icons?5count?5?9?5cal@ 000000018001a0f0     AccessBridgeJavaEntryPoints.obj
 0002:00008128       ??_C@_0CB@DPKCEABK@?$FLINFO?$FN?3?5?5?5?$CD?$CD?$CD?$CD?$CD?5icons?5count?5?$DN?5?$CF@ 000000018001a128     AccessBridgeJavaEntryPoints.obj
 0002:00008150       ??_C@_0DG@HKLCCMCD@Getting?5icon?5description?5?9?5call@ 000000018001a150     AccessBridgeJavaEntryPoints.obj
 0002:00008188       ??_C@_0DO@JICPIJF@Getting?5AccessibleIcon?5descript@ 000000018001a188     AccessBridgeJavaEntryPoints.obj
 0002:000081c8       ??_C@_0CD@GHIFDBCH@Getting?5AccessibleIcon?5descript@ 000000018001a1c8     AccessBridgeJavaEntryPoints.obj
 0002:000081f0       ??_C@_0CP@OGEOHJKD@?$FLINFO?$FN?3?5?$CD?$CD?$CD?$CD?$CD?5AccessibleIcon?5de@ 000000018001a1f0     AccessBridgeJavaEntryPoints.obj
 0002:00008220       ??_C@_0DO@MHHHDKAL@Getting?5AccessibleIcon?5descript@ 000000018001a220     AccessBridgeJavaEntryPoints.obj
 0002:00008260       ??_C@_0CO@EGEFBBBG@?$FLWARN?$FN?3?5?5?5AccessibleIcon?5descri@ 000000018001a260     AccessBridgeJavaEntryPoints.obj
 0002:00008290       ??_C@_0DE@GOAGCEO@?$CD?$CD?$CD?$CD?$CD?5Getting?5icon?5height?5?9?5cal@ 000000018001a290     AccessBridgeJavaEntryPoints.obj
 0002:000082c8       ??_C@_0CB@BMHPADNP@?$FLINFO?$FN?3?5?5?5?$CD?$CD?$CD?$CD?$CD?5icon?5height?5?$DN?5?$CF@ 000000018001a2c8     AccessBridgeJavaEntryPoints.obj
 0002:000082f0       ??_C@_0DD@EHAOAGFJ@?$CD?$CD?$CD?$CD?$CD?5Getting?5icon?5width?5?9?5call@ 000000018001a2f0     AccessBridgeJavaEntryPoints.obj
 0002:00008328       ??_C@_0CA@DPEBDDDD@?$FLINFO?$FN?3?5?5?5?$CD?$CD?$CD?$CD?$CD?5icon?5width?5?$DN?5?$CFd@ 000000018001a328     AccessBridgeJavaEntryPoints.obj
 0002:00008348       ??_C@_0DG@DLFAKGJK@?$CD?$CD?$CD?$CD?$CD?5Getting?5actions?5count?5?9?5c@ 000000018001a348     AccessBridgeJavaEntryPoints.obj
 0002:00008380       ??_C@_0CH@EOBAHIJB@?$FLINFO?$FN?3?5?5?5?$CD?$CD?$CD?$CD?$CD?5key?5actions?5cou@ 000000018001a380     AccessBridgeJavaEntryPoints.obj
 0002:000083a8       ??_C@_0DC@LHBGBJKA@Getting?5Action?5Name?5?5?9?5call?5to?5@ 000000018001a3a8     AccessBridgeJavaEntryPoints.obj
 0002:000083e0       ??_C@_0DK@MCEEGDOO@Getting?5AccessibleAction?5Name?5?5@ 000000018001a3e0     AccessBridgeJavaEntryPoints.obj
 0002:00008420       ??_C@_0BO@FCFGOMO@Getting?5AccessibleAction?5name@ 000000018001a420     AccessBridgeJavaEntryPoints.obj
 0002:00008440       ??_C@_0CL@LDPKEJLA@?$FLINFO?$FN?3?5?$CD?$CD?$CD?$CD?$CD?5AccessibleAction?5@ 000000018001a440     AccessBridgeJavaEntryPoints.obj
 0002:00008470       ??_C@_0DK@GEFGKAFF@Getting?5AccessibleAction?5name?5?5@ 000000018001a470     AccessBridgeJavaEntryPoints.obj
 0002:000084b0       ??_C@_0CK@GFGPDCKK@?$FLWARN?$FN?3?5?5?5AccessibleAction?5name@ 000000018001a4b0     AccessBridgeJavaEntryPoints.obj
 0002:000084e0       ??_C@_0FG@HPHLKACM@?$FLINFO?$FN?3?5Calling?5AccessBridgeJav@ 000000018001a4e0     AccessBridgeJavaEntryPoints.obj
 0002:00008538       ??_C@_0CB@NAFFMPJL@?$FLINFO?$FN?3?5?5?5?5?5doing?5?$CFd?5actions?5?4?4@ 000000018001a538     AccessBridgeJavaEntryPoints.obj
 0002:00008560       ??_C@_0CE@MIPOFJEF@?$FLINFO?$FN?3?5?5?5?5?5doing?5action?5?$CFd?3?5?$CFs@ 000000018001a560     AccessBridgeJavaEntryPoints.obj
 0002:00008588       ??_C@_0DC@PKIFPAKH@doAccessibleActions?5?9?5call?5to?5C@ 000000018001a588     AccessBridgeJavaEntryPoints.obj
 0002:000085c0       ??_C@_0BO@OONLHHCL@?$FLERROR?$FN?3?5?5?5?5?5Action?5?$CFd?5failed@ 000000018001a5c0     AccessBridgeJavaEntryPoints.obj
 0002:000085e0       ??_C@_0FA@KEPHMGGF@?$FLINFO?$FN?3?5Calling?5AccessBridgeJav@ 000000018001a5e0     AccessBridgeJavaEntryPoints.obj
 0002:00008630       ??_C@_0DG@GCJDNJFK@Getting?5AccessibleCharCount?5?9?5c@ 000000018001a630     AccessBridgeJavaEntryPoints.obj
 0002:00008668       ??_C@_0BK@OIDALDPI@?$FLINFO?$FN?3?5?5?5Char?5count?5?$DN?5?$CFd@ 000000018001a668     AccessBridgeJavaEntryPoints.obj
 0002:00008690       ??_C@_0EJ@JKPJJPMH@?$FLERROR?$FN?3?5either?5env?5?$DN?$DN?50?5or?5get@ 000000018001a690     AccessBridgeJavaEntryPoints.obj
 0002:000086e0       ??_C@_0DK@EFHALPMO@Getting?5AccessibleCaretPosition@ 000000018001a6e0     AccessBridgeJavaEntryPoints.obj
 0002:00008720       ??_C@_0BO@CCCENNB@?$FLINFO?$FN?3?5?5?5Index?5at?5caret?5?$DN?5?$CFd@ 000000018001a720     AccessBridgeJavaEntryPoints.obj
 0002:00008740       ??_C@_0EN@DJGOBIMD@?$FLERROR?$FN?3?5either?5env?5?$DN?$DN?50?5or?5get@ 000000018001a740     AccessBridgeJavaEntryPoints.obj
 0002:00008790       ??_C@_0DJ@MLOJKMJI@Getting?5AccessibleIndexAtPoint?5@ 000000018001a790     AccessBridgeJavaEntryPoints.obj
 0002:000087d0       ??_C@_0BO@FIAABPFC@?$FLINFO?$FN?3?5?5?5Index?5at?5point?5?$DN?5?$CFd@ 000000018001a7d0     AccessBridgeJavaEntryPoints.obj
 0002:000087f0       ??_C@_0EM@ENNBLMPC@?$FLERROR?$FN?3?5either?5env?5?$DN?$DN?50?5or?5get@ 000000018001a7f0     AccessBridgeJavaEntryPoints.obj
 0002:00008840       ??_C@_0EJ@KDHBNGHD@?$FLINFO?$FN?3?5Calling?5AccessBridgeJav@ 000000018001a840     AccessBridgeJavaEntryPoints.obj
 0002:00008890       ??_C@_0DK@CALJAPAO@Getting?5AccessibleLetterAtIndex@ 000000018001a890     AccessBridgeJavaEntryPoints.obj
 0002:000088d0       ??_C@_0DL@JDJLEMDG@Getting?5AccessibleLetterAtIndex@ 000000018001a8d0     AccessBridgeJavaEntryPoints.obj
 0002:00008910       ??_C@_0DP@BIFOHJBB@Getting?5AccessibleLetterAtIndex@ 000000018001a910     AccessBridgeJavaEntryPoints.obj
 0002:00008950       ??_C@_0DL@OOLFPOBK@Getting?5AccessibleLetterAtIndex@ 000000018001a950     AccessBridgeJavaEntryPoints.obj
 0002:00008990       ??_C@_0CG@BAFOKJKC@?$FLINFO?$FN?3?5?5?5Accessible?5Text?5lette@ 000000018001a990     AccessBridgeJavaEntryPoints.obj
 0002:000089b8       ??_C@_0DL@FNGOIOKI@Getting?5AccessibleLetterAtIndex@ 000000018001a9b8     AccessBridgeJavaEntryPoints.obj
 0002:000089f8       ??_C@_0CK@KNLDNGDN@?$FLWARN?$FN?3?5?5?5Accessible?5Text?5lette@ 000000018001a9f8     AccessBridgeJavaEntryPoints.obj
 0002:00008a30       ??_C@_0EN@GBFAECFE@?$FLERROR?$FN?3?5either?5env?5?$DN?$DN?50?5or?5get@ 000000018001aa30     AccessBridgeJavaEntryPoints.obj
 0002:00008a80       ??_C@_0DI@DFJMLOME@Getting?5AccessibleWordAtIndex?5?9@ 000000018001aa80     AccessBridgeJavaEntryPoints.obj
 0002:00008ab8       ??_C@_0DJ@OIDPECCJ@Getting?5AccessibleWordAtIndex?5?9@ 000000018001aab8     AccessBridgeJavaEntryPoints.obj
 0002:00008af8       ??_C@_0BO@NGEDADOF@Getting?5AccessibleWordAtIndex@ 000000018001aaf8     AccessBridgeJavaEntryPoints.obj
 0002:00008b18       ??_C@_0DJ@JFBBPAAF@Getting?5AccessibleWordAtIndex?5?9@ 000000018001ab18     AccessBridgeJavaEntryPoints.obj
 0002:00008b60       ??_C@_1EK@ODCBDMFL@?$AA?$FL?$AAI?$AAN?$AAF?$AAO?$AA?$FN?$AA?3?$AA?5?$AA?5?$AA?5?$AAA?$AAc?$AAc?$AAe?$AAs@ 000000018001ab60     AccessBridgeJavaEntryPoints.obj
 0002:00008bb0       ??_C@_0DJ@CGMKIALH@Getting?5AccessibleWordAtIndex?5?9@ 000000018001abb0     AccessBridgeJavaEntryPoints.obj
 0002:00008bf0       ??_C@_0CI@JLGHFNHI@?$FLWARN?$FN?3?5?5?5Accessible?5Text?5word?5@ 000000018001abf0     AccessBridgeJavaEntryPoints.obj
 0002:00008c20       ??_C@_0EL@NKGFFDIO@?$FLERROR?$FN?3?5either?5env?5?$DN?$DN?50?5or?5get@ 000000018001ac20     AccessBridgeJavaEntryPoints.obj
 0002:00008c70       ??_C@_0DP@OGFHHBKC@Getting?5AccessibleSentenceAtInd@ 000000018001ac70     AccessBridgeJavaEntryPoints.obj
 0002:00008cb0       ??_C@_0DN@MGFPCBII@Getting?5AccessibleSentenceAtInd@ 000000018001acb0     AccessBridgeJavaEntryPoints.obj
 0002:00008cf0       ??_C@_0CC@BFJMFDHP@Getting?5AccessibleSentenceAtInd@ 000000018001acf0     AccessBridgeJavaEntryPoints.obj
 0002:00008d18       ??_C@_0DN@LLHBJDKE@Getting?5AccessibleSentenceAtInd@ 000000018001ad18     AccessBridgeJavaEntryPoints.obj
 0002:00008d60       ??_C@_1FC@FOIECOHK@?$AA?$FL?$AAI?$AAN?$AAF?$AAO?$AA?$FN?$AA?3?$AA?5?$AA?5?$AA?5?$AAA?$AAc?$AAc?$AAe?$AAs@ 000000018001ad60     AccessBridgeJavaEntryPoints.obj
 0002:00008db8       ??_C@_0DN@IKKODBG@Getting?5AccessibleSentenceAtInd@ 000000018001adb8     AccessBridgeJavaEntryPoints.obj
 0002:00008df8       ??_C@_0CM@EBOEJDBD@?$FLWARN?$FN?3?5?5?5Accessible?5Text?5sente@ 000000018001adf8     AccessBridgeJavaEntryPoints.obj
 0002:00008e30       ??_C@_0EP@JMGAHICJ@?$FLERROR?$FN?3?5either?5env?5?$DN?$DN?50?5or?5get@ 000000018001ae30     AccessBridgeJavaEntryPoints.obj
 0002:00008e80       ??_C@_0FB@DGBDAMEN@?$FLINFO?$FN?3?5Calling?5AccessBridgeJav@ 000000018001ae80     AccessBridgeJavaEntryPoints.obj
 0002:00008ed8       ??_C@_0DP@BBIGIAAH@Getting?5AccessibleTextSelection@ 000000018001aed8     AccessBridgeJavaEntryPoints.obj
 0002:00008f18       ??_C@_0BP@MPEDAFPO@?$FLINFO?$FN?3?5?5?5Selection?5start?5?$DN?5?$CFd@ 000000018001af18     AccessBridgeJavaEntryPoints.obj
 0002:00008f40       ??_C@_0FD@EDCFOMDB@?$FLERROR?$FN?3?5?5either?5env?5?$DN?$DN?50?5or?5ge@ 000000018001af40     AccessBridgeJavaEntryPoints.obj
 0002:00008f98       ??_C@_0DN@MBOJJHKP@Getting?5AccessibleTextSelection@ 000000018001af98     AccessBridgeJavaEntryPoints.obj
 0002:00008fd8       ??_C@_0BN@JAKAFPAN@?$FLINFO?$FN?3?5?5?5Selection?5end?5?$DN?5?$CFd@ 000000018001afd8     AccessBridgeJavaEntryPoints.obj
 0002:00009000       ??_C@_0FA@HPMPKGDO@?$FLERROR?$FN?3?5either?5env?5?$DN?$DN?50?5or?5get@ 000000018001b000     AccessBridgeJavaEntryPoints.obj
 0002:00009050       ??_C@_0EA@KGAPFINL@Getting?5AccessibleTextSelectedT@ 000000018001b050     AccessBridgeJavaEntryPoints.obj
 0002:00009090       ??_C@_0DO@OMODBJBJ@Getting?5AccessibleTextSelectedT@ 000000018001b090     AccessBridgeJavaEntryPoints.obj
 0002:000090d0       ??_C@_0CD@CMKAHLON@Getting?5AccessibleTextSelectedT@ 000000018001b0d0     AccessBridgeJavaEntryPoints.obj
 0002:000090f8       ??_C@_0DO@JBMNKLDF@Getting?5AccessibleTextSelectedT@ 000000018001b0f8     AccessBridgeJavaEntryPoints.obj
 0002:00009138       ??_C@_0CK@DDDAABEG@?$FLINFO?$FN?3?5?5?5Accessible?8s?5selected@ 000000018001b138     AccessBridgeJavaEntryPoints.obj
 0002:00009168       ??_C@_0DO@CCBGNLIH@Getting?5AccessibleTextSelectedT@ 000000018001b168     AccessBridgeJavaEntryPoints.obj
 0002:000091a8       ??_C@_0CO@GAOLMCL@?$FLWARN?$FN?3?5?5?5Accessible?8s?5selected@ 000000018001b1a8     AccessBridgeJavaEntryPoints.obj
 0002:000091e0       ??_C@_0EP@FNBFNNLO@?$FLWARN?$FN?3?5either?5env?5?$DN?$DN?50?5or?5getA@ 000000018001b1e0     AccessBridgeJavaEntryPoints.obj
 0002:00009230       ??_C@_0EO@HEMIPALC@?$FLINFO?$FN?3?5Calling?5AccessBridgeJav@ 000000018001b230     AccessBridgeJavaEntryPoints.obj
 0002:00009280       ??_C@_0CK@OGCGGLCF@?$FLINFO?$FN?3?5?5Getting?5AttributeSet?5a@ 000000018001b280     AccessBridgeJavaEntryPoints.obj
 0002:000092b0       ??_C@_0ED@CGONELLD@Getting?5AccessibleAttributeSetA@ 000000018001b2b0     AccessBridgeJavaEntryPoints.obj
 0002:00009300       ??_C@_0FD@BNPBOBD@?$FLERROR?$FN?3?5either?5env?5?$DN?$DN?50?5or?5get@ 000000018001b300     AccessBridgeJavaEntryPoints.obj
 0002:00009360       ??_C@_0FG@OPHHFMC@?$FLWARN?$FN?3?5?5AttributeSet?5returned?5@ 000000018001b360     AccessBridgeJavaEntryPoints.obj
 0002:000093b8       ??_C@_0CL@BFGDEBIA@?$FLINFO?$FN?3?5?5Getting?5bold?5from?5Attr@ 000000018001b3b8     AccessBridgeJavaEntryPoints.obj
 0002:000093e8       ??_C@_0DL@NGCGOJOD@Getting?5BoldFromAttributeSet?5?9?5@ 000000018001b3e8     AccessBridgeJavaEntryPoints.obj
 0002:00009428       ??_C@_0DP@GPLAEKHL@?$FLERROR?$FN?3?5either?5env?5?$DN?$DN?50?5or?5get@ 000000018001b428     AccessBridgeJavaEntryPoints.obj
 0002:00009468       ??_C@_0DI@GHAHHMIG@Getting?5BoldFromAttributeSet?5?9?5@ 000000018001b468     AccessBridgeJavaEntryPoints.obj
 0002:000094a0       ??_C@_0DI@NENMAMDE@Getting?5BoldFromAttributeSet?5?9?5@ 000000018001b4a0     AccessBridgeJavaEntryPoints.obj
 0002:000094d8       ??_C@_0CN@DLPNJKCI@?$FLINFO?$FN?3?5?5Getting?5italic?5from?5At@ 000000018001b4d8     AccessBridgeJavaEntryPoints.obj
 0002:00009508       ??_C@_0DN@FALJGLGH@Getting?5ItalicFromAttributeSet?5@ 000000018001b508     AccessBridgeJavaEntryPoints.obj
 0002:00009550       ??_C@_0EC@PFKOONOF@?$FLERROR?$FN?3?5either?5env?5?$DN?$DN?50?5or?5get@ 000000018001b550     AccessBridgeJavaEntryPoints.obj
 0002:00009598       ??_C@_0DK@CEDKJPGF@Getting?5ItalicFromAttributeSet?5@ 000000018001b598     AccessBridgeJavaEntryPoints.obj
 0002:000095d8       ??_C@_0DK@JHOBOPNH@Getting?5ItalicFromAttributeSet?5@ 000000018001b5d8     AccessBridgeJavaEntryPoints.obj
 0002:00009618       ??_C@_0DA@HJAHPBCP@?$FLINFO?$FN?3?5?5Getting?5underline?5from@ 000000018001b618     AccessBridgeJavaEntryPoints.obj
 0002:00009650       ??_C@_0EA@LFOJMIBN@Getting?5UnderlineFromAttributeS@ 000000018001b650     AccessBridgeJavaEntryPoints.obj
 0002:00009690       ??_C@_0EF@LMCHMLNC@?$FLERROR?$FN?3?5?5either?5env?5?$DN?$DN?50?5or?5ge@ 000000018001b690     AccessBridgeJavaEntryPoints.obj
 0002:000096d8       ??_C@_0DN@GEOGGPCN@Getting?5UnderlineFromAttributeS@ 000000018001b6d8     AccessBridgeJavaEntryPoints.obj
 0002:00009718       ??_C@_0DN@NHDNBPJP@Getting?5UnderlineFromAttributeS@ 000000018001b718     AccessBridgeJavaEntryPoints.obj
 0002:00009758       ??_C@_0DE@MIAPKOHI@?$FLINFO?$FN?3?5?5Getting?5strikethrough?5@ 000000018001b758     AccessBridgeJavaEntryPoints.obj
 0002:00009790       ??_C@_0EE@DDJIBELI@Getting?5StrikethroughFromAttrib@ 000000018001b790     AccessBridgeJavaEntryPoints.obj
 0002:000097e0       ??_C@_0EI@HMMOGEKC@?$FLERROR?$FN?3?5either?5env?5?$DN?$DN?50?5or?5get@ 000000018001b7e0     AccessBridgeJavaEntryPoints.obj
 0002:00009830       ??_C@_0EB@GCIGLCLO@Getting?5StrikethroughFromAttrib@ 000000018001b830     AccessBridgeJavaEntryPoints.obj
 0002:00009880       ??_C@_0EB@NBFNMCAM@Getting?5StrikethroughFromAttrib@ 000000018001b880     AccessBridgeJavaEntryPoints.obj
 0002:000098c8       ??_C@_0DC@ENJFOBHI@?$FLINFO?$FN?3?5?5Getting?5superscript?5fr@ 000000018001b8c8     AccessBridgeJavaEntryPoints.obj
 0002:00009900       ??_C@_0EC@BAJDPNIO@Getting?5SuperscriptFromAttribut@ 000000018001b900     AccessBridgeJavaEntryPoints.obj
 0002:00009950       ??_C@_0EH@EIIKEOA@?$FLERROR?$FN?3?5either?5env?5?$DN?$DN?50?5or?5get@ 000000018001b950     AccessBridgeJavaEntryPoints.obj
 0002:00009998       ??_C@_0DP@LNAJFDKJ@Getting?5SuperscriptFromAttribut@ 000000018001b998     AccessBridgeJavaEntryPoints.obj
 0002:000099d8       ??_C@_0DP@ONCCDBL@Getting?5SuperscriptFromAttribut@ 000000018001b9d8     AccessBridgeJavaEntryPoints.obj
 0002:00009a18       ??_C@_0DA@KLOJONPP@?$FLINFO?$FN?3?5?5Getting?5subscript?5from@ 000000018001ba18     AccessBridgeJavaEntryPoints.obj
 0002:00009a50       ??_C@_0EA@NMFFGPLI@Getting?5SubscriptFromAttributeS@ 000000018001ba50     AccessBridgeJavaEntryPoints.obj
 0002:00009a90       ??_C@_0EE@EGHOMMOM@?$FLERROR?$FN?3?5either?5env?5?$DN?$DN?50?5or?5get@ 000000018001ba90     AccessBridgeJavaEntryPoints.obj
 0002:00009ad8       ??_C@_0DN@NJLPKKJA@Getting?5SubscriptFromAttributeS@ 000000018001bad8     AccessBridgeJavaEntryPoints.obj
 0002:00009b18       ??_C@_0DN@GKGENKCC@Getting?5SubscriptFromAttributeS@ 000000018001bb18     AccessBridgeJavaEntryPoints.obj
 0002:00009b58       ??_C@_0DG@JDMMILDN@?$FLINFO?$FN?3?5?5Getting?5backgroundColo@ 000000018001bb58     AccessBridgeJavaEntryPoints.obj
 0002:00009b90       ??_C@_0EF@CPKEHGFF@Getting?5BackgroundColorFromAttr@ 000000018001bb90     AccessBridgeJavaEntryPoints.obj
 0002:00009be0       ??_C@_0ED@OOEECCFB@Getting?5BackgroundColorFromAttr@ 000000018001bbe0     AccessBridgeJavaEntryPoints.obj
 0002:00009c28       ??_C@_0CI@JBOBOECB@Getting?5BackgroundColorFromAttr@ 000000018001bc28     AccessBridgeJavaEntryPoints.obj
 0002:00009c50       ??_C@_0ED@JDGKJAHN@Getting?5BackgroundColorFromAttr@ 000000018001bc50     AccessBridgeJavaEntryPoints.obj
 0002:00009ca0       ??_C@_1GA@PMLMKIMP@?$AA?$FL?$AAI?$AAN?$AAF?$AAO?$AA?$FN?$AA?3?$AA?5?$AA?5?$AA?5?$AAA?$AAt?$AAt?$AAr?$AAi@ 000000018001bca0     AccessBridgeJavaEntryPoints.obj
 0002:00009d00       ??_C@_0ED@CALBOAMP@Getting?5BackgroundColorFromAttr@ 000000018001bd00     AccessBridgeJavaEntryPoints.obj
 0002:00009d48       ??_C@_0DD@DIMBBLFG@?$FLWARN?$FN?3?5?5?5AttributeSet?8s?5backgr@ 000000018001bd48     AccessBridgeJavaEntryPoints.obj
 0002:00009d80       ??_C@_0EK@LDLFAHLP@?$FLERROR?$FN?3?5either?5env?5?$DN?$DN?50?5or?5get@ 000000018001bd80     AccessBridgeJavaEntryPoints.obj
 0002:00009dd0       ??_C@_0DG@OAPFKBJG@?$FLINFO?$FN?3?5?5Getting?5foregroundColo@ 000000018001bdd0     AccessBridgeJavaEntryPoints.obj
 0002:00009e10       ??_C@_0EF@CFMCBGOA@Getting?5ForegroundColorFromAttr@ 000000018001be10     AccessBridgeJavaEntryPoints.obj
 0002:00009e60       ??_C@_0ED@CGONGGIL@Getting?5ForegroundColorFromAttr@ 000000018001be60     AccessBridgeJavaEntryPoints.obj
 0002:00009ea8       ??_C@_0CI@MCDFAAFE@Getting?5ForegroundColorFromAttr@ 000000018001bea8     AccessBridgeJavaEntryPoints.obj
 0002:00009ed0       ??_C@_0ED@FLMDNEKH@Getting?5ForegroundColorFromAttr@ 000000018001bed0     AccessBridgeJavaEntryPoints.obj
 0002:00009f20       ??_C@_1GA@DDCOJJLA@?$AA?$FL?$AAI?$AAN?$AAF?$AAO?$AA?$FN?$AA?3?$AA?5?$AA?5?$AA?5?$AAA?$AAt?$AAt?$AAr?$AAi@ 000000018001bf20     AccessBridgeJavaEntryPoints.obj
 0002:00009f80       ??_C@_0ED@OIBIKEBF@Getting?5ForegroundColorFromAttr@ 000000018001bf80     AccessBridgeJavaEntryPoints.obj
 0002:00009fc8       ??_C@_0DD@EGLIFJNP@?$FLWARN?$FN?3?5?5?5AttributeSet?8s?5foregr@ 000000018001bfc8     AccessBridgeJavaEntryPoints.obj
 0002:0000a000       ??_C@_0EK@JAILLABF@?$FLERROR?$FN?3?5either?5env?5?$DN?$DN?50?5or?5get@ 000000018001c000     AccessBridgeJavaEntryPoints.obj
 0002:0000a050       ??_C@_0DB@NPCHLNMB@?$FLINFO?$FN?3?5?5Getting?5fontFamily?5fro@ 000000018001c050     AccessBridgeJavaEntryPoints.obj
 0002:0000a090       ??_C@_0EA@OFLFMJOA@Getting?5FontFamilyFromAttribute@ 000000018001c090     AccessBridgeJavaEntryPoints.obj
 0002:0000a0d0       ??_C@_0DO@ECEGIKHO@Getting?5FontFamilyFromAttribute@ 000000018001c0d0     AccessBridgeJavaEntryPoints.obj
 0002:0000a110       ??_C@_0CD@ELONJGOI@Getting?5FontFamilyFromAttribute@ 000000018001c110     AccessBridgeJavaEntryPoints.obj
 0002:0000a138       ??_C@_0DO@DPGIDIFC@Getting?5FontFamilyFromAttribute@ 000000018001c138     AccessBridgeJavaEntryPoints.obj
 0002:0000a180       ??_C@_1FE@LCMANMIC@?$AA?$FL?$AAI?$AAN?$AAF?$AAO?$AA?$FN?$AA?3?$AA?5?$AA?5?$AA?5?$AAA?$AAt?$AAt?$AAr?$AAi@ 000000018001c180     AccessBridgeJavaEntryPoints.obj
 0002:0000a1d8       ??_C@_0DO@IMLDEIOA@Getting?5FontFamilyFromAttribute@ 000000018001c1d8     AccessBridgeJavaEntryPoints.obj
 0002:0000a218       ??_C@_0CN@DFPIBNDO@?$FLWARN?$FN?3?5?5?5AttributeSet?8s?5fontFa@ 000000018001c218     AccessBridgeJavaEntryPoints.obj
 0002:0000a250       ??_C@_0EF@MEIJBCDI@?$FLERROR?$FN?3?5either?5env?5?$DN?$DN?50?5or?5get@ 000000018001c250     AccessBridgeJavaEntryPoints.obj
 0002:0000a298       ??_C@_0DA@NKBCCHCB@?$FLINFO?$FN?3?5?5Getting?5font?5size?5from@ 000000018001c298     AccessBridgeJavaEntryPoints.obj
 0002:0000a2c8       ??_C@_0DL@OGKGFGCH@Getting?5FontSizeFromAttributeSe@ 000000018001c2c8     AccessBridgeJavaEntryPoints.obj
 0002:0000a308       ??_C@_0CI@MMDBDPDB@?$FLINFO?$FN?3?5?5?5AttributeSet?8s?5font?5s@ 000000018001c308     AccessBridgeJavaEntryPoints.obj
 0002:0000a330       ??_C@_0EE@EGBGOKJP@?$FLERROR?$FN?3?5either?5env?5?$DN?$DN?50?5or?5get@ 000000018001c330     AccessBridgeJavaEntryPoints.obj
 0002:0000a378       ??_C@_0DM@KMMBHJCP@Getting?5FontSizeFromAttributeSe@ 000000018001c378     AccessBridgeJavaEntryPoints.obj
 0002:0000a3b8       ??_C@_0DM@BPBKAJJN@Getting?5FontSizeFromAttributeSe@ 000000018001c3b8     AccessBridgeJavaEntryPoints.obj
 0002:0000a3f8       ??_C@_0CI@DPJLKBCH@?5Getting?5alignment?5from?5Attribu@ 000000018001c3f8     AccessBridgeJavaEntryPoints.obj
 0002:0000a420       ??_C@_0DM@IEKBPPGN@Getting?5AlignmentFromAttributeS@ 000000018001c420     AccessBridgeJavaEntryPoints.obj
 0002:0000a460       ??_C@_0DN@DKKKNGAI@Getting?5AlignmentFromAttributeS@ 000000018001c460     AccessBridgeJavaEntryPoints.obj
 0002:0000a4a0       ??_C@_0DN@IJHBKGLK@Getting?5AlignmentFromAttributeS@ 000000018001c4a0     AccessBridgeJavaEntryPoints.obj
 0002:0000a4e0       ??_C@_0DA@IEHDNKCA@?$FLINFO?$FN?3?5?5Getting?5bidiLevel?5from@ 000000018001c4e0     AccessBridgeJavaEntryPoints.obj
 0002:0000a510       ??_C@_0DM@HHHEIBLO@Getting?5BidiLevelFromAttributeS@ 000000018001c510     AccessBridgeJavaEntryPoints.obj
 0002:0000a550       ??_C@_0EE@FHPLAGJN@?$FLERROR?$FN?3?5either?5env?5?$DN?$DN?50?5or?5get@ 000000018001c550     AccessBridgeJavaEntryPoints.obj
 0002:0000a598       ??_C@_0DN@CFIDIABI@Getting?5BidiLevelFromAttributeS@ 000000018001c598     AccessBridgeJavaEntryPoints.obj
 0002:0000a5d8       ??_C@_0DN@JGFIPAKK@Getting?5BidiLevelFromAttributeS@ 000000018001c5d8     AccessBridgeJavaEntryPoints.obj
 0002:0000a618       ??_C@_0DH@CAJPMJAH@?$FLERROR?$FN?3?5?5Getting?5firstLineInde@ 000000018001c618     AccessBridgeJavaEntryPoints.obj
 0002:0000a650       ??_C@_0EC@GDNCLBBP@Getting?5FirstLineIndentFromAttr@ 000000018001c650     AccessBridgeJavaEntryPoints.obj
 0002:0000a6a0       ??_C@_0EK@JNGBIMLH@?$FLERROR?$FN?3?5either?5env?5?$DN?$DN?50?5or?5get@ 000000018001c6a0     AccessBridgeJavaEntryPoints.obj
 0002:0000a6f0       ??_C@_0ED@IEEGLFFG@Getting?5FirstLineIndentFromAttr@ 000000018001c6f0     AccessBridgeJavaEntryPoints.obj
 0002:0000a740       ??_C@_0ED@DHJNMFOE@Getting?5FirstLineIndentFromAttr@ 000000018001c740     AccessBridgeJavaEntryPoints.obj
 0002:0000a788       ??_C@_0DB@GIKOBABF@?$FLINFO?$FN?3?5?5Getting?5leftIndent?5fro@ 000000018001c788     AccessBridgeJavaEntryPoints.obj
 0002:0000a7c0       ??_C@_0DN@GGPJCLGF@Getting?5LeftIndentFromAttribute@ 000000018001c7c0     AccessBridgeJavaEntryPoints.obj
 0002:0000a800       ??_C@_0EF@JFNBAGAC@?$FLERROR?$FN?3?5either?5env?5?$DN?$DN?50?5or?5get@ 000000018001c800     AccessBridgeJavaEntryPoints.obj
 0002:0000a848       ??_C@_0DO@DEJDAGOO@Getting?5LeftIndentFromAttribute@ 000000018001c848     AccessBridgeJavaEntryPoints.obj
 0002:0000a888       ??_C@_0DO@IHEIHGFM@Getting?5LeftIndentFromAttribute@ 000000018001c888     AccessBridgeJavaEntryPoints.obj
 0002:0000a8c8       ??_C@_0DC@OHJHAPPB@?$FLINFO?$FN?3?5?5Getting?5rightIndent?5fr@ 000000018001c8c8     AccessBridgeJavaEntryPoints.obj
 0002:0000a900       ??_C@_0DO@GPANPNCO@Getting?5RightIndentFromAttribut@ 000000018001c900     AccessBridgeJavaEntryPoints.obj
 0002:0000a940       ??_C@_0EG@FKGIOCMJ@?$FLERROR?$FN?3?5either?5env?5?$DN?$DN?50?5or?5get@ 000000018001c940     AccessBridgeJavaEntryPoints.obj
 0002:0000a988       ??_C@_0DP@NFJEGKCA@Getting?5RightIndentFromAttribut@ 000000018001c988     AccessBridgeJavaEntryPoints.obj
 0002:0000a9c8       ??_C@_0DP@GGEPBKJC@Getting?5RightIndentFromAttribut@ 000000018001c9c8     AccessBridgeJavaEntryPoints.obj
 0002:0000aa08       ??_C@_0DC@FBCMPKE@?$FLINFO?$FN?3?5?5Getting?5lineSpacing?5fr@ 000000018001ca08     AccessBridgeJavaEntryPoints.obj
 0002:0000aa40       ??_C@_0DO@OLMNNFJE@Getting?5LineSpacingFromAttribut@ 000000018001ca40     AccessBridgeJavaEntryPoints.obj
 0002:0000aa80       ??_C@_0EH@DJGGHDHL@?$FLERROR?$FN?3?5?5either?5env?5?$DN?$DN?50?5or?5ge@ 000000018001ca80     AccessBridgeJavaEntryPoints.obj
 0002:0000aac8       ??_C@_0DP@POKEPAJK@Getting?5LineSpacingFromAttribut@ 000000018001cac8     AccessBridgeJavaEntryPoints.obj
 0002:0000ab08       ??_C@_0DP@ENHPIACI@Getting?5LineSpacingFromAttribut@ 000000018001cb08     AccessBridgeJavaEntryPoints.obj
 0002:0000ab48       ??_C@_0DB@BBFBINOC@?$FLINFO?$FN?3?5?5Getting?5spaceAbove?5fro@ 000000018001cb48     AccessBridgeJavaEntryPoints.obj
 0002:0000ab80       ??_C@_0DN@LICNMEPC@Getting?5SpaceAboveFromAttribute@ 000000018001cb80     AccessBridgeJavaEntryPoints.obj
 0002:0000abc0       ??_C@_0EG@DEAABEIJ@?$FLERROR?$FN?3?5?5either?5env?5?$DN?$DN?50?5or?5ge@ 000000018001cbc0     AccessBridgeJavaEntryPoints.obj
 0002:0000ac08       ??_C@_0DO@FKCGNEOG@Getting?5SpaceAboveFromAttribute@ 000000018001cc08     AccessBridgeJavaEntryPoints.obj
 0002:0000ac48       ??_C@_0DO@OJPNKEFE@Getting?5SpaceAboveFromAttribute@ 000000018001cc48     AccessBridgeJavaEntryPoints.obj
 0002:0000ac88       ??_C@_0DB@IPEMBOFF@?$FLINFO?$FN?3?5?5Getting?5spaceBelow?5fro@ 000000018001cc88     AccessBridgeJavaEntryPoints.obj
 0002:0000acc0       ??_C@_0DN@KGEHENNL@Getting?5SpaceBelowFromAttribute@ 000000018001ccc0     AccessBridgeJavaEntryPoints.obj
 0002:0000ad00       ??_C@_0EG@PAJHHADM@?$FLERROR?$FN?3?5?5either?5env?5?$DN?$DN?50?5or?5ge@ 000000018001cd00     AccessBridgeJavaEntryPoints.obj
 0002:0000ad48       ??_C@_0DO@BIIKCGAD@Getting?5SpaceBelowFromAttribute@ 000000018001cd48     AccessBridgeJavaEntryPoints.obj
 0002:0000ad88       ??_C@_0DO@KLFBFGLB@Getting?5SpaceBelowFromAttribute@ 000000018001cd88     AccessBridgeJavaEntryPoints.obj
 0002:0000adc8       ??_C@_0DD@NEPODHGJ@?$FLINFO?$FN?3?5?5Decrementing?5reference@ 000000018001cdc8     AccessBridgeJavaEntryPoints.obj
 0002:0000ae00       ??_C@_0DJ@KDCCLHCF@Releasing?5AttributeSet?5object?5?9@ 000000018001ce00     AccessBridgeJavaEntryPoints.obj
 0002:0000ae40       ??_C@_0DF@KOJHMOGM@?$FLERROR?$FN?3?5?5either?5env?5?$DN?$DN?50?5or?5ac@ 000000018001ce40     AccessBridgeJavaEntryPoints.obj
 0002:0000ae78       ??_C@_0DJ@BAPJMHJH@Releasing?5AttributeSet?5object?5?9@ 000000018001ce78     AccessBridgeJavaEntryPoints.obj
 0002:0000aeb8       ??_C@_0DI@FAAGAOKI@?$FLINFO?$FN?3?5?5Getting?5full?5attribute@ 000000018001ceb8     AccessBridgeJavaEntryPoints.obj
 0002:0000aef0       ??_C@_0DD@BPFGOEDD@?$FLINFO?$FN?3?5?5returned?5from?5CallObje@ 000000018001cef0     AccessBridgeJavaEntryPoints.obj
 0002:0000af30       ??_C@_1FG@IBEGPOLG@?$AA?$FL?$AAI?$AAN?$AAF?$AAO?$AA?$FN?$AA?3?$AA?5?$AA?5?$AA?5?$AAA?$AAc?$AAc?$AAe?$AAs@ 000000018001cf30     AccessBridgeJavaEntryPoints.obj
 0002:0000af90       ??_C@_0FC@NKKMDLMK@?$FLERROR?$FN?3?5?5either?5env?5?$DN?$DN?50?5or?5ge@ 000000018001cf90     AccessBridgeJavaEntryPoints.obj
 0002:0000aff0       ??_C@_0EB@FOBGJMBG@Getting?5AccessibleAttributeSetA@ 000000018001cff0     AccessBridgeJavaEntryPoints.obj
 0002:0000b040       ??_C@_0FD@ONBHOKNL@?$FLINFO?$FN?3?5Calling?5AccessBridgeJav@ 000000018001d040     AccessBridgeJavaEntryPoints.obj
 0002:0000b098       ??_C@_0DL@PJLLEMMJ@Getting?5AccessibleXcoordTextRec@ 000000018001d098     AccessBridgeJavaEntryPoints.obj
 0002:0000b0d8       ??_C@_0BG@CDBEIJEJ@?$FLINFO?$FN?3?5?5X?5coord?5?$DN?5?$CFd@ 000000018001d0d8     AccessBridgeJavaEntryPoints.obj
 0002:0000b0f0       ??_C@_0FF@CICHONC@?$FLERROR?$FN?3?5either?5env?5?$DN?$DN?50?5or?5get@ 000000018001d0f0     AccessBridgeJavaEntryPoints.obj
 0002:0000b148       ??_C@_0DL@BBKMNMGI@Getting?5AccessibleYcoordTextRec@ 000000018001d148     AccessBridgeJavaEntryPoints.obj
 0002:0000b190       ??_C@_0FF@LPGHAKKN@?$FLINFO?$FN?3?5?5either?5env?5?$DN?$DN?50?5or?5get@ 000000018001d190     AccessBridgeJavaEntryPoints.obj
 0002:0000b1e8       ??_C@_0DK@GOMAAIJJ@Getting?5AccessibleWidthTextRect@ 000000018001d1e8     AccessBridgeJavaEntryPoints.obj
 0002:0000b228       ??_C@_0BD@PFFPBFHC@?$FLINFO?$FN?3?5Width?5?$DN?5?$CFd@ 000000018001d228     AccessBridgeJavaEntryPoints.obj
 0002:0000b240       ??_C@_0FD@LFKJAPPJ@?$FLINFO?$FN?3?5either?5env?5?$DN?$DN?50?5or?5getA@ 000000018001d240     AccessBridgeJavaEntryPoints.obj
 0002:0000b298       ??_C@_0DL@LIFPGLAA@Getting?5AccessibleHeightTextRec@ 000000018001d298     AccessBridgeJavaEntryPoints.obj
 0002:0000b2d8       ??_C@_0BE@BNGOGMPP@?$FLINFO?$FN?3?5Height?5?$DN?5?$CFd@ 000000018001d2d8     AccessBridgeJavaEntryPoints.obj
 0002:0000b2f0       ??_C@_0FG@JCNMAPKJ@?$FLERROR?$FN?3?5?5either?5env?5?$DN?$DN?50?5or?5ge@ 000000018001d2f0     AccessBridgeJavaEntryPoints.obj
 0002:0000b350       ??_C@_0EO@GAEGCFMP@?$FLINFO?$FN?3?5Calling?5AccessBridgeJav@ 000000018001d350     AccessBridgeJavaEntryPoints.obj
 0002:0000b3a0       ??_C@_0DF@JPKJOLBB@Getting?5caret?5X?5coordinate?5?9?5ca@ 000000018001d3a0     AccessBridgeJavaEntryPoints.obj
 0002:0000b3d8       ??_C@_0DK@INHGMNIG@?$FLERROR?$FN?3?5?5either?5env?5?$DN?$DN?50?5or?5ge@ 000000018001d3d8     AccessBridgeJavaEntryPoints.obj
 0002:0000b418       ??_C@_0DF@NBCAOALI@Getting?5caret?5Y?5coordinate?5?9?5ca@ 000000018001d418     AccessBridgeJavaEntryPoints.obj
 0002:0000b450       ??_C@_0DK@FAOABEAD@?$FLERROR?$FN?3?5?5either?5env?5?$DN?$DN?50?5or?5ge@ 000000018001d450     AccessBridgeJavaEntryPoints.obj
 0002:0000b490       ??_C@_0CO@LPKJFNHN@Getting?5caret?5width?5?9?5call?5to?5C@ 000000018001d490     AccessBridgeJavaEntryPoints.obj
 0002:0000b4c0       ??_C@_0DO@KCIKCBGA@?$FLERROR?$FN?3?5?5either?5env?5?$DN?$DN?50?5or?5ge@ 000000018001d4c0     AccessBridgeJavaEntryPoints.obj
 0002:0000b500       ??_C@_0CP@DKBLCBME@Getting?5caret?5height?5?9?5call?5to?5@ 000000018001d500     AccessBridgeJavaEntryPoints.obj
 0002:0000b530       ??_C@_0DP@MHKONHOK@?$FLERROR?$FN?3?5?5either?5env?5?$DN?$DN?50?5or?5ge@ 000000018001d530     AccessBridgeJavaEntryPoints.obj
 0002:0000b570       ??_C@_0EO@OPGMODFN@?$FLINFO?$FN?3?5Calling?5AccessBridgeJav@ 000000018001d570     AccessBridgeJavaEntryPoints.obj
 0002:0000b5c0       ??_C@_0DP@HIDGMFDD@Getting?5AccessibleTextLineLeftB@ 000000018001d5c0     AccessBridgeJavaEntryPoints.obj
 0002:0000b600       ??_C@_0BK@INECDNLO@?$FLINFO?$FN?3?5?5?5startIndex?5?$DN?5?$CFd@ 000000018001d600     AccessBridgeJavaEntryPoints.obj
 0002:0000b620       ??_C@_0FD@BGKHJCDH@?$FLERROR?$FN?3?5?5either?5env?5?$DN?$DN?50?5or?5ge@ 000000018001d620     AccessBridgeJavaEntryPoints.obj
 0002:0000b680       ??_C@_0EA@OJGAJNKG@Getting?5AccessibleTextLineRight@ 000000018001d680     AccessBridgeJavaEntryPoints.obj
 0002:0000b6c0       ??_C@_0BI@NAKKCMDP@?$FLINFO?$FN?3?5?5?5endIndex?5?$DN?5?$CFd@ 000000018001d6c0     AccessBridgeJavaEntryPoints.obj
 0002:0000b6e0       ??_C@_0FE@HOJFBBNL@?$FLERROR?$FN?3?5?5either?5env?5?$DN?$DN?50?5or?5ge@ 000000018001d6e0     AccessBridgeJavaEntryPoints.obj
 0002:0000b740       ??_C@_0FM@PBOJPFBI@?$FLINFO?$FN?3?5Calling?5AccessBridgeJav@ 000000018001d740     AccessBridgeJavaEntryPoints.obj
 0002:0000b7a0       ??_C@_0BH@GCPBFEO@?$FLERROR?$FN?3?5?5end?5?$DM?5start?$CB@ 000000018001d7a0     AccessBridgeJavaEntryPoints.obj
 0002:0000b7b8       ??_C@_0DJ@OHJBLKEE@Getting?5AccessibleTextRange?5?9?5c@ 000000018001d7b8     AccessBridgeJavaEntryPoints.obj
 0002:0000b7f8       ??_C@_0DH@MLKPAEJI@Getting?5AccessibleTextRange?5?9?5c@ 000000018001d7f8     AccessBridgeJavaEntryPoints.obj
 0002:0000b830       ??_C@_1HO@MOIAIALP@?$AA?$FL?$AAI?$AAN?$AAF?$AAO?$AA?$FN?$AA?3?$AA?5?$AA?5?$AA?5?$AAA?$AAc?$AAc?$AAe?$AAs@ 000000018001d830     AccessBridgeJavaEntryPoints.obj
 0002:0000b8b0       ??_C@_0DB@GEMONLMO@?$FLINFO?$FN?3?5?5Accessible?5Text?5string@ 000000018001d8b0     AccessBridgeJavaEntryPoints.obj
 0002:0000b8f0       ??_C@_1HM@KJDBDPH@?$AA?$FL?$AAI?$AAN?$AAF?$AAO?$AA?$FN?$AA?3?$AA?5?$AA?5?$AA?5?$AAA?$AAc?$AAc?$AAe?$AAs@ 000000018001d8f0     AccessBridgeJavaEntryPoints.obj
 0002:0000b970       ??_C@_0BM@KMPFPDHC@Getting?5AccessibleTextRange@ 000000018001d970     AccessBridgeJavaEntryPoints.obj
 0002:0000b990       ??_C@_0DH@LGIBLGLE@Getting?5AccessibleTextRange?5?9?5c@ 000000018001d990     AccessBridgeJavaEntryPoints.obj
 0002:0000b9d0       ??_C@_1EM@MAOOPBBK@?$AA?$FL?$AAI?$AAN?$AAF?$AAO?$AA?$FN?$AA?3?$AA?5?$AA?5?$AA?5?$AAA?$AAc?$AAc?$AAe?$AAs@ 000000018001d9d0     AccessBridgeJavaEntryPoints.obj
 0002:0000ba20       ??_C@_0DH@FFKMGAG@Getting?5AccessibleTextRange?5?9?5c@ 000000018001da20     AccessBridgeJavaEntryPoints.obj
 0002:0000ba58       ??_C@_0DB@ENPGLEMN@?$FLWARN?$FN?3?5?5?5current?5Accessible?5Te@ 000000018001da58     AccessBridgeJavaEntryPoints.obj
 0002:0000ba90       ??_C@_0EJ@IGDKNKCL@?$FLERROR?$FN?3?5either?5env?5?$DN?$DN?50?5or?5get@ 000000018001da90     AccessBridgeJavaEntryPoints.obj
 0002:0000bae0       ??_C@_0FH@DFGPJEBI@?$FLINFO?$FN?3?5Calling?5AccessBridgeJav@ 000000018001dae0     AccessBridgeJavaEntryPoints.obj
 0002:0000bb38       ??_C@_0DM@FMEJNEAF@Getting?5CurrentAccessibleValue?5@ 000000018001db38     AccessBridgeJavaEntryPoints.obj
 0002:0000bb78       ??_C@_0DK@DEBJEKPP@Getting?5CurrentAccessibleValue?5@ 000000018001db78     AccessBridgeJavaEntryPoints.obj
 0002:0000bbb8       ??_C@_0BP@PMLFPGML@Getting?5CurrentAccessibleValue@ 000000018001dbb8     AccessBridgeJavaEntryPoints.obj
 0002:0000bbd8       ??_C@_0DK@EJDHPIND@Getting?5CurrentAccessibleValue?5@ 000000018001dbd8     AccessBridgeJavaEntryPoints.obj
 0002:0000bc18       ??_C@_0CI@LHBKPIPL@?$FLINFO?$FN?3?5?5?5current?5Accessible?5Va@ 000000018001dc18     AccessBridgeJavaEntryPoints.obj
 0002:0000bc40       ??_C@_0DK@PKOMIIGB@Getting?5CurrentAccessibleValue?5@ 000000018001dc40     AccessBridgeJavaEntryPoints.obj
 0002:0000bc80       ??_C@_0CM@JBCHBMHL@?$FLWARN?$FN?3?5?5?5current?5Accessible?5Va@ 000000018001dc80     AccessBridgeJavaEntryPoints.obj
 0002:0000bcb0       ??_C@_0EN@CEFCJCHP@?$FLERROR?$FN?3?5?5either?5env?5?$DN?$DN?50?5or?5ge@ 000000018001dcb0     AccessBridgeJavaEntryPoints.obj
 0002:0000bd00       ??_C@_0FH@LDANAJBK@?$FLINFO?$FN?3?5Calling?5AccessBridgeJav@ 000000018001dd00     AccessBridgeJavaEntryPoints.obj
 0002:0000bd58       ??_C@_0DM@CNMGLEAD@Getting?5MaximumAccessibleValue?5@ 000000018001dd58     AccessBridgeJavaEntryPoints.obj
 0002:0000bd98       ??_C@_0DK@LPOBNFBI@Getting?5MaximumAccessibleValue?5@ 000000018001dd98     AccessBridgeJavaEntryPoints.obj
 0002:0000bdd8       ??_C@_0BP@FLCAAJND@Getting?5MaximumAccessibleValue@ 000000018001ddd8     AccessBridgeJavaEntryPoints.obj
 0002:0000bdf8       ??_C@_0DK@MCMPGHDE@Getting?5MaximumAccessibleValue?5@ 000000018001ddf8     AccessBridgeJavaEntryPoints.obj
 0002:0000be38       ??_C@_0CI@MOLFAIEC@?$FLINFO?$FN?3?5?5?5maximum?5Accessible?5Va@ 000000018001de38     AccessBridgeJavaEntryPoints.obj
 0002:0000be60       ??_C@_0DK@HBBEBHIG@Getting?5MaximumAccessibleValue?5@ 000000018001de60     AccessBridgeJavaEntryPoints.obj
 0002:0000bea0       ??_C@_0CM@EENPAHAF@?$FLWARN?$FN?3?5?5?5maximum?5Accessible?5Va@ 000000018001dea0     AccessBridgeJavaEntryPoints.obj
 0002:0000bed0       ??_C@_0EM@DECMFMLP@?$FLERROR?$FN?3?5either?5env?5?$DN?$DN?50?5or?5get@ 000000018001ded0     AccessBridgeJavaEntryPoints.obj
 0002:0000bf20       ??_C@_0FH@NCJCNBPB@?$FLINFO?$FN?3?5Calling?5AccessBridgeJav@ 000000018001df20     AccessBridgeJavaEntryPoints.obj
 0002:0000bf78       ??_C@_0DM@EKOMNNCH@Getting?5MinimumAccessibleValue?5@ 000000018001df78     AccessBridgeJavaEntryPoints.obj
 0002:0000bfb8       ??_C@_0DK@POFOBDIM@Getting?5MinimumAccessibleValue?5@ 000000018001dfb8     AccessBridgeJavaEntryPoints.obj
 0002:0000bff8       ??_C@_0BP@FPLKDIPJ@Getting?5MinimumAccessibleValue@ 000000018001dff8     AccessBridgeJavaEntryPoints.obj
 0002:0000c018       ??_C@_0DK@IDHAKBKA@Getting?5MinimumAccessibleValue?5@ 000000018001e018     AccessBridgeJavaEntryPoints.obj
 0002:0000c058       ??_C@_0CI@HMFEBFFJ@?$FLINFO?$FN?3?5?5?5mimimum?5Accessible?5Va@ 000000018001e058     AccessBridgeJavaEntryPoints.obj
 0002:0000c080       ??_C@_0DK@DAKLNBBC@Getting?5MinimumAccessibleValue?5@ 000000018001e080     AccessBridgeJavaEntryPoints.obj
 0002:0000c0c0       ??_C@_0CM@LFDDPHLF@?$FLWARN?$FN?3?5?5?5mimimum?5Accessible?5Va@ 000000018001e0c0     AccessBridgeJavaEntryPoints.obj
 0002:0000c0f0       ??_C@_0EM@FNBMNDID@?$FLERROR?$FN?3?5either?5env?5?$DN?$DN?50?5or?5get@ 000000018001e0f0     AccessBridgeJavaEntryPoints.obj
 0002:0000c140       ??_C@_0FE@GLAEHJLA@?$FLINFO?$FN?3?5Calling?5AccessBridgeJav@ 000000018001e140     AccessBridgeJavaEntryPoints.obj
 0002:0000c198       ??_C@_0DI@HFNIIMHH@Doing?5addAccessibleSelection?5?9?5@ 000000018001e198     AccessBridgeJavaEntryPoints.obj
 0002:0000c1d0       ??_C@_0CP@EBNEHGHB@?$FLERROR?$FN?3?5?$CK?$CK?$CK?5Exception?5occured?5@ 000000018001e1d0     AccessBridgeJavaEntryPoints.obj
 0002:0000c200       ??_C@_0CL@OKIJNCBD@?$FLINFO?$FN?3?5?5?5returned?5from?5CallObj@ 000000018001e200     AccessBridgeJavaEntryPoints.obj
 0002:0000c230       ??_C@_0EK@CMGGDKGL@?$FLERROR?$FN?3?5?5either?5env?5?$DN?$DN?50?5or?5ad@ 000000018001e230     AccessBridgeJavaEntryPoints.obj
 0002:0000c280       ??_C@_0FG@JICCBONC@?$FLINFO?$FN?3?5Calling?5AccessBridgeJav@ 000000018001e280     AccessBridgeJavaEntryPoints.obj
 0002:0000c2d8       ??_C@_0DK@GPKPKKON@Doing?5clearAccessibleSelection?5@ 000000018001e2d8     AccessBridgeJavaEntryPoints.obj
 0002:0000c320       ??_C@_0EM@NKPDGGGN@?$FLERROR?$FN?3?5?5either?5env?5?$DN?$DN?50?5or?5cl@ 000000018001e320     AccessBridgeJavaEntryPoints.obj
 0002:0000c370       ??_C@_0FE@PIPHOHFI@?$FLINFO?$FN?3?5Calling?5AccessBridgeJav@ 000000018001e370     AccessBridgeJavaEntryPoints.obj
 0002:0000c3d0       ??_C@_0EA@EDHDCMHP@Getting?5AccessibleSelectionCont@ 000000018001e3d0     AccessBridgeJavaEntryPoints.obj
 0002:0000c410       ??_C@_0DM@IFLFNJN@Getting?5AccessibleSelectionCont@ 000000018001e410     AccessBridgeJavaEntryPoints.obj
 0002:0000c450       ??_C@_0DO@FEBBEFGL@Getting?5AccessibleSelectionCont@ 000000018001e450     AccessBridgeJavaEntryPoints.obj
 0002:0000c490       ??_C@_0FA@KGJFECGD@?$FLERROR?$FN?3?5either?5env?5?$DN?$DN?50?5or?5get@ 000000018001e490     AccessBridgeJavaEntryPoints.obj
 0002:0000c4e0       ??_C@_0FJ@KDCCHMFP@?$FLINFO?$FN?3?5Calling?5AccessBridgeJav@ 000000018001e4e0     AccessBridgeJavaEntryPoints.obj
 0002:0000c540       ??_C@_0DL@JPLKCOEB@Getting?5AccessibleSelectionCoun@ 000000018001e540     AccessBridgeJavaEntryPoints.obj
 0002:0000c580       ??_C@_0EO@LLPLNNDE@?$FLERROR?$FN?3?5either?5env?5?$DN?$DN?50?5or?5get@ 000000018001e580     AccessBridgeJavaEntryPoints.obj
 0002:0000c5d0       ??_C@_0FH@BEGAHKNM@?$FLINFO?$FN?3?5Calling?5AccessBridgeJav@ 000000018001e5d0     AccessBridgeJavaEntryPoints.obj
 0002:0000c628       ??_C@_0DO@DGOGEINB@Doing?5isAccessibleChildSelected@ 000000018001e628     AccessBridgeJavaEntryPoints.obj
 0002:0000c670       ??_C@_0EM@FIJEFPDC@?$FLERROR?$FN?3?5either?5env?5?$DN?$DN?50?5or?5isA@ 000000018001e670     AccessBridgeJavaEntryPoints.obj
 0002:0000c6c0       ??_C@_0FH@DBFJFKMJ@?$FLINFO?$FN?3?5Calling?5AccessBridgeJav@ 000000018001e6c0     AccessBridgeJavaEntryPoints.obj
 0002:0000c718       ??_C@_0DL@BHDCMLKI@Doing?5removeAccessibleSelection@ 000000018001e718     AccessBridgeJavaEntryPoints.obj
 0002:0000c760       ??_C@_0EN@HJFMAEOO@?$FLERROR?$FN?3?5?5either?5env?5?$DN?$DN?50?5or?5re@ 000000018001e760     AccessBridgeJavaEntryPoints.obj
 0002:0000c7b0       ??_C@_0FK@MANGNIPE@?$FLINFO?$FN?3?5Calling?5AccessBridgeJav@ 000000018001e7b0     AccessBridgeJavaEntryPoints.obj
 0002:0000c810       ??_C@_0DO@JHGLNKHC@Doing?5selectAllAccessibleSelect@ 000000018001e810     AccessBridgeJavaEntryPoints.obj
 0002:0000c850       ??_C@_0EP@JCKDPHMN@?$FLERROR?$FN?3?5either?5env?5?$DN?$DN?50?5or?5sel@ 000000018001e850     AccessBridgeJavaEntryPoints.obj
 0002:0000c8a0       ??_C@_0EO@IEPNANKM@?$FLINFO?$FN?3?5?5?5in?5AccessBridgeJavaEn@ 000000018001e8a0     AccessBridgeJavaEntryPoints.obj
 0002:0000c8f0       ??_C@_0DK@GPMPKEMH@Doing?5addJavaEventNotification?5@ 000000018001e8f0     AccessBridgeJavaEntryPoints.obj
 0002:0000c930       ??_C@_0EA@IOOHIHIM@?$FLERROR?$FN?3?5either?5env?5?$DN?$DN?50?5or?5add@ 000000018001e930     AccessBridgeJavaEntryPoints.obj
 0002:0000c970       ??_C@_0FA@BBNLJKAK@?$FLINFO?$FN?3?5?5in?5AccessBridgeJavaEnt@ 000000018001e970     AccessBridgeJavaEntryPoints.obj
 0002:0000c9c0       ??_C@_0DN@IBNHMLMO@Doing?5removeJavaEventNotificati@ 000000018001e9c0     AccessBridgeJavaEntryPoints.obj
 0002:0000ca00       ??_C@_0ED@LKLPMFCD@?$FLERROR?$FN?3?5either?5env?5?$DN?$DN?50?5or?5rem@ 000000018001ea00     AccessBridgeJavaEntryPoints.obj
 0002:0000ca50       ??_C@_0FH@ICFBIMPG@?$FLINFO?$FN?3?5?5?5in?5AccessBridgeJavaEn@ 000000018001ea50     AccessBridgeJavaEntryPoints.obj
 0002:0000cab0       ??_C@_0FL@OCFIPKDP@?$FLINFO?$FN?3?5?5?5?5addAccessibilityEven@ 000000018001eab0     AccessBridgeJavaEntryPoints.obj
 0002:0000cb10       ??_C@_0DH@DNDEHAJF@Doing?5addAccessibilityEvent?5?9?5c@ 000000018001eb10     AccessBridgeJavaEntryPoints.obj
 0002:0000cb50       ??_C@_0EJ@BAMHEIMC@?$FLERROR?$FN?3?5either?5env?5?$DN?$DN?50?5or?5add@ 000000018001eb50     AccessBridgeJavaEntryPoints.obj
 0002:0000cba0       ??_C@_0ED@BCNEMPCF@?$FLINFO?$FN?3?5?5?5?5?5addAccessibilityEve@ 000000018001eba0     AccessBridgeJavaEntryPoints.obj
 0002:0000cbf0       ??_C@_0FJ@JPJKPKP@?$FLINFO?$FN?3?5?5in?5AccessBridgeJavaEnt@ 000000018001ebf0     AccessBridgeJavaEntryPoints.obj
 0002:0000cc50       ??_C@_0DK@KGOHAMJ@Doing?5removeAccessibilityEvent?5@ 000000018001ec50     AccessBridgeJavaEntryPoints.obj
 0002:0000cc90       ??_C@_0EM@MPLDCCAE@?$FLERROR?$FN?3?5either?5env?5?$DN?$DN?50?5or?5rem@ 000000018001ec90     AccessBridgeJavaEntryPoints.obj
 0002:0000cce0       ??_C@_0BM@BIAOFPJG@AccessBridge?9FromJava?9Hello@ 000000018001ece0     AccessBridgeMessages.obj
 0002:0000cd00       ??_C@_0BP@OELHMMDF@AccessBridge?9FromWindows?9Hello@ 000000018001ed00     AccessBridgeMessages.obj
 0002:0000cd20       ??_C@_0CN@HNEPECB@?$FLINFO?$FN?3?5JavaAccessBridge?4DLL?5ru@ 000000018001ed20     JavaAccessBridge.obj
 0002:0000cd50       ??_C@_0CN@OBDABACD@?$FLINFO?$FN?3?5In?5AccessBridgeDialog?5?9@ 000000018001ed50     JavaAccessBridge.obj
 0002:0000cd80       ??_C@_0DM@LEGKGBDC@?$FLINFO?$FN?3?5In?5AccessBridgeDialog?5?9@ 000000018001ed80     JavaAccessBridge.obj
 0002:0000cdc0       ??_C@_0DP@KFGJNONL@?$FLINFO?$FN?3?5In?5AccessBridgeDialog?5?9@ 000000018001edc0     JavaAccessBridge.obj
 0002:0000ce00       ??_C@_0DN@BOPHDCMF@?$FLINFO?$FN?3?5In?5AccessBridgeDialog?5?9@ 000000018001ee00     JavaAccessBridge.obj
 0002:0000ce40       ??_C@_0EG@LODLDNEL@?$FLINFO?$FN?3?5In?5AccessBridgeDialog?5?9@ 000000018001ee40     JavaAccessBridge.obj
 0002:0000ce90       ??_C@_0EE@OLIPFHDH@?$FLINFO?$FN?3?5In?5AccessBridgeDialog?5?9@ 000000018001ee90     JavaAccessBridge.obj
 0002:0000ced8       ??_C@_0DO@KFBCLDPM@?$FLINFO?$FN?3?5In?5AccessBridgeDialog?5?9@ 000000018001eed8     JavaAccessBridge.obj
 0002:0000cf20       ??_C@_0EF@PPOLOLIM@?$FLINFO?$FN?3?5In?5AccessBridgeDialog?5?9@ 000000018001ef20     JavaAccessBridge.obj
 0002:0000cf68       ??_C@_0BD@BOAKDBCO@java_access_bridge@ 000000018001ef68     JavaAccessBridge.obj
 0002:0000cf80       ??_C@_0DB@JHKNDMME@?$FLINFO?$FN?3?5in?5JavaAccessBridge?3?3?$HOJ@ 000000018001ef80     JavaAccessBridge.obj
 0002:0000cfb8       ??_C@_0CF@DJNKIAAH@?$FLINFO?$FN?3?5?5telling?5?$CFp?5we?8re?5going@ 000000018001efb8     JavaAccessBridge.obj
 0002:0000cfe0       ??_C@_0CP@BKDEGDJC@?$FLINFO?$FN?3?5?5finished?5telling?5ATs?5a@ 000000018001efe0     JavaAccessBridge.obj
 0002:0000d010       ??_C@_0CA@EIEOEDOI@?$FLINFO?$FN?3?5?5?5finished?5deleting?5ATs@ 000000018001f010     JavaAccessBridge.obj
 0002:0000d030       ??_C@_0BP@EBFMIPOK@?$FLINFO?$FN?3?5GOODBYE?5CRUEL?5WORLD?4?4?4@ 000000018001f030     JavaAccessBridge.obj
 0002:0000d050       ??_C@_0DB@BKKBMMIL@?$FLINFO?$FN?3?5JavaAccessBridge?3?3javaR@ 000000018001f050     JavaAccessBridge.obj
 0002:0000d088       ??_C@_0BJ@CDAHIMFI@?$FLINFO?$FN?3?5?5?5?9?$DO?5javaVM?5?$DN?5?$CFp@ 000000018001f088     JavaAccessBridge.obj
 0002:0000d0a8       ??_C@_0CF@HBJLLMBP@?$FLINFO?$FN?3?5?5?9?$DO?5windowsThreadJNIEnv@ 000000018001f0a8     JavaAccessBridge.obj
 0002:0000d0d0       ??_C@_0DL@EDCIECNK@?$FLINFO?$FN?3?5?5?5all?5Java?5thread?5entry@ 000000018001f0d0     JavaAccessBridge.obj
 0002:0000d110       ??_C@_0DO@DHHHOLPH@?$FLINFO?$FN?3?5?5?5all?5Windows?5thread?5en@ 000000018001f110     JavaAccessBridge.obj
 0002:0000d150       ??_C@_0CF@FINMKFHO@?$FLINFO?$FN?3?5?5?5Window?5created?4?5?5HWND@ 000000018001f150     JavaAccessBridge.obj
 0002:0000d178       ??_C@_0CG@KCHIBPOJ@?$FLERROR?$FN?3?5?5?5FAILED?5TO?5CREATE?5WIN@ 000000018001f178     JavaAccessBridge.obj
 0002:0000d1a0       ??_C@_0BJ@LMONFDOG@ACCESSBRIDGESTATUSWINDOW@ 000000018001f1a0     JavaAccessBridge.obj
 0002:0000d1c0       ??_C@_0DG@HAJICJFK@?$FLINFO?$FN?3?5In?5JavaAccessBridge?3?3po@ 000000018001f1c0     JavaAccessBridge.obj
 0002:0000d1f8       ??_C@_0CO@FLLNHCIG@?$FLINFO?$FN?3?5?5?5calling?5PostMessage?$CI?$CF@ 000000018001f1f8     JavaAccessBridge.obj
 0002:0000d228       ??_C@_0CM@DCNJAPPO@?$FLERROR?$FN?3?5ATs?5?$DN?$DN?50?$CB?5?$CIshouldn?8t?5h@ 000000018001f228     JavaAccessBridge.obj
 0002:0000d258       ??_C@_0DH@JMPJBGDF@?$FLINFO?$FN?3?5JavaAccessBridge?3?3recei@ 000000018001f258     JavaAccessBridge.obj
 0002:0000d290       ??_C@_0EB@GECAJJE@?$FLERROR?$FN?3?5?9?5ATs?5?$DN?$DN?50?5?$CIshouldn?8t?5@ 000000018001f290     JavaAccessBridge.obj
 0002:0000d2d8       ??_C@_0DL@FAPEODKG@?$FLERROR?$FN?3?5receiving?5memory?5packa@ 000000018001f2d8     JavaAccessBridge.obj
 0002:0000d318       ??_C@_0DM@MJCPMIJG@?$FLINFO?$FN?3?5Processing?5package?5sent@ 000000018001f318     JavaAccessBridge.obj
 0002:0000d358       ??_C@_0BL@EFABEHOK@?$FLINFO?$FN?3?5?5PackageType?5?$DN?5?$CFX?3@ 000000018001f358     JavaAccessBridge.obj
 0002:0000d378       ??_C@_0DC@HOEDKHHL@?$FLINFO?$FN?3?5?5?5type?5?$DN?$DN?5cMemoryMapped@ 000000018001f378     JavaAccessBridge.obj
 0002:0000d3b0       ??_C@_0EC@JELBKKLB@?$FLERROR?$FN?3?5?5?5?5processing?5FAILED?$CB?$CB@ 000000018001f3b0     JavaAccessBridge.obj
 0002:0000d3f8       ??_C@_0CM@EGHIFACB@?$FLINFO?$FN?3?5?5?5type?5?$DN?$DN?5cReleaseJavaO@ 000000018001f3f8     JavaAccessBridge.obj
 0002:0000d430       ??_C@_0EB@PCOLNIOI@?$FLERROR?$FN?3?5?5?5processing?5FAILED?$CB?$CB?5@ 000000018001f430     JavaAccessBridge.obj
 0002:0000d478       ??_C@_0DB@HJBBLNK@?$FLINFO?$FN?3?5?5?5type?5?$DN?$DN?5cGetAccessBri@ 000000018001f478     JavaAccessBridge.obj
 0002:0000d4b0       ??_C@_0CH@OGPNINNH@?$FLINFO?$FN?3?5?5?5type?5?$DN?$DN?5cIsJavaWindow@ 000000018001f4b0     JavaAccessBridge.obj
 0002:0000d4d8       ??_C@_0CF@KCGBFLNL@?$FLINFO?$FN?3?5?5?5?5?5?9?$DO?5returning?5result@ 000000018001f4d8     JavaAccessBridge.obj
 0002:0000d500       ??_C@_0CH@FFMGBMGP@?$FLINFO?$FN?3?5?5?5type?5?$DN?$DN?5cIsSameObject@ 000000018001f500     JavaAccessBridge.obj
 0002:0000d528       ??_C@_0DI@FGDPIMOI@?$FLINFO?$FN?3?5?5?5?5type?5?$DN?$DN?5cGetAccessib@ 000000018001f528     JavaAccessBridge.obj
 0002:0000d560       ??_C@_0CN@KFALDIEC@?$FLINFO?$FN?3?5?5?5?5?5?5?9?$DO?5returning?5AC?5?$DN?5@ 000000018001f560     JavaAccessBridge.obj
 0002:0000d590       ??_C@_0DI@ICOCNDDM@?$FLINFO?$FN?3?5?5?5?5type?5?$DN?$DN?5cGetHWNDFrom@ 000000018001f590     JavaAccessBridge.obj
 0002:0000d5c8       ??_C@_0CD@DNCFKFDK@?$FLINFO?$FN?3?5?5?5?5?5?9?$DO?5returning?5HWND?5?$DN@ 000000018001f5c8     JavaAccessBridge.obj
 0002:0000d5f0       ??_C@_0CK@DBBKGOKJ@?$FLINFO?$FN?3?5?5?5type?5?$DN?$DN?5cSetTextConte@ 000000018001f5f0     JavaAccessBridge.obj
 0002:0000d620       ??_C@_0JK@BDICEONN@?$FLINFO?$FN?3?5?5?5type?5?$DN?$DN?5cGetParentWit@ 000000018001f620     JavaAccessBridge.obj
 0002:0000d6c0       ??_C@_0CM@FMGIHPCP@?$FLINFO?$FN?3?5?5?5type?5?$DN?$DN?5cGetTopLevelO@ 000000018001f6c0     JavaAccessBridge.obj
 0002:0000d6f0       ??_C@_0DC@EMOAFCHE@?$FLINFO?$FN?3?5?5?5?5?5?5?9?$DO?5returning?5rAcce@ 000000018001f6f0     JavaAccessBridge.obj
 0002:0000d728       ??_C@_0DE@EHPIAHAD@?$FLINFO?$FN?3?5?5?5type?5?$DN?$DN?5cGetParentWit@ 000000018001f728     JavaAccessBridge.obj
 0002:0000d760       ??_C@_0CJ@CIIOKEJA@?$FLINFO?$FN?3?5?5?5type?5?$DN?$DN?5cGetObjectDep@ 000000018001f760     JavaAccessBridge.obj
 0002:0000d790       ??_C@_0CG@CCMHCDED@?$FLINFO?$FN?3?5?5?5?5?5?9?$DO?5returning?5rResul@ 000000018001f790     JavaAccessBridge.obj
 0002:0000d7b8       ??_C@_0CO@HPDBNII@?$FLINFO?$FN?3?5?5?5type?5?$DN?$DN?5cGetActiveDes@ 000000018001f7b8     JavaAccessBridge.obj
 0002:0000d7e8       ??_C@_0CO@EEGIDCBJ@?$FLINFO?$FN?3?5?5?9?$DO?5returning?5rAccessib@ 000000018001f7e8     JavaAccessBridge.obj
 0002:0000d818       ??_C@_0DB@BLNOEMHA@?$FLINFO?$FN?3?5?5?5type?5?$DN?$DN?5cGetAccessibl@ 000000018001f818     JavaAccessBridge.obj
 0002:0000d850       ??_C@_0DI@BBJPLAPN@?$FLINFO?$FN?3?5?5?5type?5?$DN?$DN?5cGetAccessibl@ 000000018001f850     JavaAccessBridge.obj
 0002:0000d888       ??_C@_0DD@EKFFDOAF@?$FLINFO?$FN?3?5?5?5type?5?$DN?$DN?5cGetAccessibl@ 000000018001f888     JavaAccessBridge.obj
 0002:0000d8c0       ??_C@_0DI@HCCMIAAH@?$FLINFO?$FN?3?5?5?5type?5?$DN?$DN?5cGetAccessibl@ 000000018001f8c0     JavaAccessBridge.obj
 0002:0000d8f8       ??_C@_0DK@EHNJMPFO@?$FLINFO?$FN?3?5?5?5?5type?5?$DN?$DN?5cGetAccessib@ 000000018001f8f8     JavaAccessBridge.obj
 0002:0000d938       ??_C@_0DI@DNENMOMG@?$FLINFO?$FN?3?5?5?5?5?$CD?$CD?$CD?$CD?$CD?5type?5?$DN?$DN?5cGetAc@ 000000018001f938     JavaAccessBridge.obj
 0002:0000d970       ??_C@_0CG@KFAMLONA@?$FLINFO?$FN?3?5?5?5?5?$CD?$CD?$CD?$CD?$CD?5processing?5suc@ 000000018001f970     JavaAccessBridge.obj
 0002:0000d9a0       ??_C@_0EI@KKCFGLCL@?$FLERROR?$FN?3?5?5?5?5?$CD?$CD?$CD?$CD?$CD?5processing?5FA@ 000000018001f9a0     JavaAccessBridge.obj
 0002:0000d9e8       ??_C@_0DM@ONBKHFBE@?$FLINFO?$FN?3?5?5?5?5?$CD?$CD?$CD?$CD?$CD?5type?5?$DN?$DN?5cGetAc@ 000000018001f9e8     JavaAccessBridge.obj
 0002:0000da28       ??_C@_0DN@MOEKMKGM@?$FLINFO?$FN?3?5?5?5?5?$CD?$CD?$CD?$CD?$CD?5type?5?$DN?$DN?5cGetAc@ 000000018001fa28     JavaAccessBridge.obj
 0002:0000da70       ??_C@_0EA@CAKJDHMA@?$FLINFO?$FN?3?5?5?5?5?$CD?$CD?$CD?$CD?$CD?5type?5?$DN?$DN?5cGetAc@ 000000018001fa70     JavaAccessBridge.obj
 0002:0000dab0       ??_C@_0EC@JLIHGBEM@?$FLINFO?$FN?3?5?5?5?5?$CD?$CD?$CD?$CD?$CD?5type?5?$DN?$DN?5cGetAc@ 000000018001fab0     JavaAccessBridge.obj
 0002:0000db00       ??_C@_0EF@DBAFGNDK@?$FLINFO?$FN?3?5?5?5?5?$CD?$CD?$CD?$CD?$CD?5type?5?$DN?$DN?5cGetAc@ 000000018001fb00     JavaAccessBridge.obj
 0002:0000db50       ??_C@_0EI@BCPJNOBP@?$FLINFO?$FN?3?5?5?5?5?$CD?$CD?$CD?$CD?$CD?5type?5?$DN?$DN?5cGetAc@ 000000018001fb50     JavaAccessBridge.obj
 0002:0000dba0       ??_C@_0EF@ONIGGHFH@?$FLINFO?$FN?3?5?5?5?5?$CD?$CD?$CD?$CD?$CD?5type?5?$DN?$DN?5cGetAc@ 000000018001fba0     JavaAccessBridge.obj
 0002:0000dbe8       ??_C@_0DO@ENBHEGBB@?$FLINFO?$FN?3?5?5?5?5?$CD?$CD?$CD?$CD?$CD?5type?5?$DN?$DN?5cIsAcc@ 000000018001fbe8     JavaAccessBridge.obj
 0002:0000dc30       ??_C@_0EB@PMALJKOF@?$FLINFO?$FN?3?5?5?5?5?$CD?$CD?$CD?$CD?$CD?5type?5?$DN?$DN?5cIsAcc@ 000000018001fc30     JavaAccessBridge.obj
 0002:0000dc80       ??_C@_0EE@NFLEEFCE@?$FLINFO?$FN?3?5?5?5?5?$CD?$CD?$CD?$CD?$CD?5type?5?$DN?$DN?5cGetAc@ 000000018001fc80     JavaAccessBridge.obj
 0002:0000dcd0       ??_C@_0EH@DNDNECPC@?$FLINFO?$FN?3?5?5?5?5?5?5?$CD?$CD?$CD?$CD?$CD?5cGetAccessib@ 000000018001fcd0     JavaAccessBridge.obj
 0002:0000dd20       ??_C@_0EF@PFDKDHMH@?$FLINFO?$FN?3?5?5?5?5?5?5?$CD?$CD?$CD?$CD?$CD?5cGetAccessib@ 000000018001fd20     JavaAccessBridge.obj
 0002:0000dd70       ??_C@_0EB@FNPEGMEK@?$FLINFO?$FN?3?5?5?5?5?$CD?$CD?$CD?$CD?$CD?5type?5?$DN?$DN?5cGetAc@ 000000018001fd70     JavaAccessBridge.obj
 0002:0000ddb8       ??_C@_0DH@HGKABJI@?$FLINFO?$FN?3?5?5?5?5?$CD?$CD?$CD?$CD?$CD?5type?5?$DN?$DN?5cGetAc@ 000000018001fdb8     JavaAccessBridge.obj
 0002:0000ddf0       ??_C@_0DK@PHHNIBJB@?$FLINFO?$FN?3?5?5?5?5?$CD?$CD?$CD?$CD?$CD?5type?5?$DN?$DN?5cGetAc@ 000000018001fdf0     JavaAccessBridge.obj
 0002:0000de30       ??_C@_0DJ@ECCDOPKO@?$FLINFO?$FN?3?5?5?5?5?$CD?$CD?$CD?$CD?$CD?5type?5?$DN?$DN?5cGetAc@ 000000018001fe30     JavaAccessBridge.obj
 0002:0000de70       ??_C@_0DK@GDIGFCLP@?$FLINFO?$FN?3?5?5?5?5?$CD?$CD?$CD?$CD?$CD?5type?5?$DN?$DN?5cGetAc@ 000000018001fe70     JavaAccessBridge.obj
 0002:0000deb0       ??_C@_0DI@BPKDDCHO@?$FLINFO?$FN?3?5?5?5?5?$CD?$CD?$CD?$CD?$CD?5type?5?$DN?$DN?5cGetAc@ 000000018001feb0     JavaAccessBridge.obj
 0002:0000dee8       ??_C@_0DN@OAAMPEIM@?$FLINFO?$FN?3?5?5?5?5?$CD?$CD?$CD?$CD?$CD?5type?5?$DN?$DN?5cActiv@ 000000018001fee8     JavaAccessBridge.obj
 0002:0000df28       ??_C@_0DN@GBPFAJCJ@?$FLINFO?$FN?3?5?5?5?5?$CD?$CD?$CD?$CD?$CD?5type?5?$DN?$DN?5cGetAc@ 000000018001ff28     JavaAccessBridge.obj
 0002:0000df68       ??_C@_0DM@HFKCAKHD@?$FLINFO?$FN?3?5?5?5?5?$CD?$CD?$CD?$CD?$CD?5processing?5suc@ 000000018001ff68     JavaAccessBridge.obj
 0002:0000dfa8       ??_C@_0DL@BKPFGPAI@?$FLINFO?$FN?3?5?5?5?5?$CD?$CD?$CD?$CD?$CD?5type?5?$DN?$DN?5cGetAc@ 000000018001ffa8     JavaAccessBridge.obj
 0002:0000dff0       ??_C@_0EB@HBBMKHLL@?$FLINFO?$FN?3?5?5?5?5?$CD?$CD?$CD?$CD?$CD?5type?5?$DN?$DN?5cGetAc@ 000000018001fff0     JavaAccessBridge.obj
 0002:0000e038       ??_C@_0DI@EGGEEHLE@?$FLINFO?$FN?3?5?5?5?5?$CD?$CD?$CD?$CD?$CD?5type?5?$DN?$DN?5cGetAc@ 0000000180020038     JavaAccessBridge.obj
 0002:0000e070       ??_C@_0DK@LOBFOEFG@?$FLINFO?$FN?3?5?5?5?5?$CD?$CD?$CD?$CD?$CD?5type?5?$DN?$DN?5cGetAc@ 0000000180020070     JavaAccessBridge.obj
 0002:0000e0b0       ??_C@_0DE@NCPKKLJG@?$FLINFO?$FN?3?5?5?5?5?$CD?$CD?$CD?$CD?$CD?5type?5?$DN?$DN?5cGetAc@ 00000001800200b0     JavaAccessBridge.obj
 0002:0000e0f0       ??_C@_0EH@OKFMNJOP@?$FLERROR?$FN?3?5?5?5?$CD?$CD?$CD?$CD?$CD?5processing?5FAI@ 00000001800200f0     JavaAccessBridge.obj
 0002:0000e138       ??_C@_0DG@CDFKKFMN@?$FLINFO?$FN?3?5?5?5?5?$CD?$CD?$CD?$CD?$CD?5type?5?$DN?$DN?5cGetAc@ 0000000180020138     JavaAccessBridge.obj
 0002:0000e170       ??_C@_0DF@GOCDLFHO@?$FLINFO?$FN?3?5?5?5?5?$CD?$CD?$CD?$CD?$CD?5type?5?$DN?$DN?5cDoAcc@ 0000000180020170     JavaAccessBridge.obj
 0002:0000e1a8       ??_C@_0DJ@FOPNGHK@?$FLINFO?$FN?3?5?5?5?5?$CD?$CD?$CD?$CD?$CD?5type?5?$DN?$DN?5GetVir@ 00000001800201a8     JavaAccessBridge.obj
 0002:0000e1e8       ??_C@_0CN@KKAHFJLP@?$FLINFO?$FN?3?5?5?5?5?$CD?$CD?$CD?$CD?$CD?5type?5?$DN?$DN?5Reques@ 00000001800201e8     JavaAccessBridge.obj
 0002:0000e218       ??_C@_0DA@BDJNNLOI@?$FLINFO?$FN?3?5?5?5?5?$CD?$CD?$CD?$CD?$CD?5type?5?$DN?$DN?5Select@ 0000000180020218     JavaAccessBridge.obj
 0002:0000e248       ??_C@_0DJ@JNPDLANK@?$FLINFO?$FN?3?5?5?5?5?$CD?$CD?$CD?$CD?$CD?5type?5?$DN?$DN?5GetTex@ 0000000180020248     JavaAccessBridge.obj
 0002:0000e288       ??_C@_0DI@KCHGBBIN@?$FLINFO?$FN?3?5?5?5?5?$CD?$CD?$CD?$CD?$CD?5type?5?$DN?$DN?5GetVis@ 0000000180020288     JavaAccessBridge.obj
 0002:0000e2c0       ??_C@_0DD@HFEKHIPA@?$FLINFO?$FN?3?5?5?5?5?$CD?$CD?$CD?$CD?$CD?5type?5?$DN?$DN?5GetVis@ 00000001800202c0     JavaAccessBridge.obj
 0002:0000e2f8       ??_C@_0DB@HDPFDIKC@?$FLINFO?$FN?3?5?5?5?5?$CD?$CD?$CD?$CD?$CD?5type?5?$DN?$DN?5SetCar@ 00000001800202f8     JavaAccessBridge.obj
 0002:0000e330       ??_C@_0DB@MBKJOFKA@?$FLINFO?$FN?3?5?5?5?5type?5?$DN?$DN?5cGetAccessib@ 0000000180020330     JavaAccessBridge.obj
 0002:0000e368       ??_C@_0DC@FACNMLJM@?$FLINFO?$FN?3?5?5?5?5type?5?$DN?$DN?5cGetAccessib@ 0000000180020368     JavaAccessBridge.obj
 0002:0000e3a0       ??_C@_0DK@BMAJHBGM@?$FLINFO?$FN?3?5?5?5?5type?5?$DN?$DN?5cGetAccessib@ 00000001800203a0     JavaAccessBridge.obj
 0002:0000e3e0       ??_C@_0DK@KLKIIEMH@?$FLINFO?$FN?3?5?5?5?5type?5?$DN?$DN?5cGetAccessib@ 00000001800203e0     JavaAccessBridge.obj
 0002:0000e420       ??_C@_0DF@LJIJJCFL@?$FLINFO?$FN?3?5?5?5?5type?5?$DN?$DN?5cGetAccessib@ 0000000180020420     JavaAccessBridge.obj
 0002:0000e458       ??_C@_0CM@DKHFKJOD@?$FLINFO?$FN?3?5?5?5?5type?5?$DN?$DN?5cGetCaretLoc@ 0000000180020458     JavaAccessBridge.obj
 0002:0000e488       ??_C@_0DH@CHPJDHJL@?$FLINFO?$FN?3?5?5?5?5type?5?$DN?$DN?5cGetAccessib@ 0000000180020488     JavaAccessBridge.obj
 0002:0000e4c0       ??_C@_0DC@HMIBGEHP@?$FLINFO?$FN?3?5?5?5?5type?5?$DN?$DN?5cGetAccessib@ 00000001800204c0     JavaAccessBridge.obj
 0002:0000e500       ??_C@_0EA@OJBBPFCG@?$FLINFO?$FN?3?5?5?5?5type?5?$DN?$DN?5cGetCurrentA@ 0000000180020500     JavaAccessBridge.obj
 0002:0000e540       ??_C@_0EA@FFJJPODP@?$FLINFO?$FN?3?5?5?5?5type?5?$DN?$DN?5cGetMaximumA@ 0000000180020540     JavaAccessBridge.obj
 0002:0000e580       ??_C@_0EA@GABLOPGB@?$FLINFO?$FN?3?5?5?5?5type?5?$DN?$DN?5cGetMinimumA@ 0000000180020580     JavaAccessBridge.obj
 0002:0000e5c0       ??_C@_0DN@NHMKNOBO@?$FLINFO?$FN?3?5?5?5?5type?5?$DN?$DN?5cAddAccessib@ 00000001800205c0     JavaAccessBridge.obj
 0002:0000e600       ??_C@_0DP@CDAIIOJL@?$FLINFO?$FN?3?5?5?5?5type?5?$DN?$DN?5cClearAccess@ 0000000180020600     JavaAccessBridge.obj
 0002:0000e640       ??_C@_0DN@FGNKIKEK@?$FLINFO?$FN?3?5?5?5?5type?5?$DN?$DN?5cGetAccessib@ 0000000180020640     JavaAccessBridge.obj
 0002:0000e680       ??_C@_0EC@JGIFJEAP@?$FLINFO?$FN?3?5?5?5?5type?5?$DN?$DN?5cGetAccessib@ 0000000180020680     JavaAccessBridge.obj
 0002:0000e6d0       ??_C@_0EA@BDFAJBM@?$FLINFO?$FN?3?5?5?5?5type?5?$DN?$DN?5cIsAccessibl@ 00000001800206d0     JavaAccessBridge.obj
 0002:0000e710       ??_C@_0EA@NOOOKPJ@?$FLINFO?$FN?3?5?5?5?5type?5?$DN?$DN?5cRemoveAcces@ 0000000180020710     JavaAccessBridge.obj
 0002:0000e750       ??_C@_0ED@CNEBOKEO@?$FLINFO?$FN?3?5?5?5?5type?5?$DN?$DN?5cSelectAllAc@ 0000000180020750     JavaAccessBridge.obj
 0002:0000e798       ??_C@_0DD@FDABBAIG@?$FLINFO?$FN?3?5?5?5?5type?5?$DN?5cAddJavaEvent@ 0000000180020798     JavaAccessBridge.obj
 0002:0000e7d0       ??_C@_0DG@CJJGFHBD@?$FLINFO?$FN?3?5?5?5?5type?5?$DN?5cRemoveJavaEv@ 00000001800207d0     JavaAccessBridge.obj
 0002:0000e808       ??_C@_0DM@IHHPMOM@?$FLINFO?$FN?3?5?5?5?5type?5?$DN?5cAddAccessibi@ 0000000180020808     JavaAccessBridge.obj
 0002:0000e848       ??_C@_0DP@CLPLFGHM@?$FLINFO?$FN?3?5?5?5?5type?5?$DN?5cRemoveAccess@ 0000000180020848     JavaAccessBridge.obj
 0002:0000e890       ??_C@_0EG@DADDGPDA@?$FLERROR?$FN?3?5?5?5?5processing?5FAILED?$CB?$CB@ 0000000180020890     JavaAccessBridge.obj
 0002:0000e8d8       ??_C@_0CI@PMGDCMNI@?$FLINFO?$FN?3?5?5?5?5package?5processing?5c@ 00000001800208d8     JavaAccessBridge.obj
 0002:0000e900       ??_C@_0CO@NOIJCKLH@?$FLINFO?$FN?3?5?5?5in?5MemoryMappedFileCr@ 0000000180020900     JavaAccessBridge.obj
 0002:0000e930       ??_C@_0DJ@MGBOAEHL@?$FLINFO?$FN?3?5?5?5?5?5just?5created?5a?5new?5@ 0000000180020930     JavaAccessBridge.obj
 0002:0000e970       ??_C@_0DA@PCLBAGKL@?$FLINFO?$FN?3?5?5?5Successfully?5initiate@ 0000000180020970     JavaAccessBridge.obj
 0002:0000e9a0       ??_C@_0CL@IAFANAPB@?$FLERROR?$FN?3?5Failed?5to?5initiate?5IPC@ 00000001800209a0     JavaAccessBridge.obj
 0002:0000e9d0       ??_C@_0DE@FDNKAIDO@?$FLINFO?$FN?3?5in?5JavaAccessBridge?3?3Wi@ 00000001800209d0     JavaAccessBridge.obj
 0002:0000ea08       ??_C@_0CO@DDCCLLBJ@?$FLERROR?$FN?3?5?9?$DO?5ATs?5?$DN?$DN?50?$CB?5?$CIshouldn?8@ 0000000180020a08     JavaAccessBridge.obj
 0002:0000ea38       ??_C@_0CP@IIHJFGGB@?$FLINFO?$FN?3?5?5?5data?5structures?5succe@ 0000000180020a38     JavaAccessBridge.obj
 0002:0000ea68       ??_C@_0DB@JABMCGEJ@?$FLERROR?$FN?3?5couldn?8t?5find?5matching@ 0000000180020a68     JavaAccessBridge.obj
 0002:0000eaa0       ??_C@_0CP@LEPCODGO@?$FLINFO?$FN?3?5In?5JavaAccessBridge?3?3re@ 0000000180020aa0     JavaAccessBridge.obj
 0002:0000ead0       ??_C@_0BH@GNOIGMFE@?$FLINFO?$FN?3?5?5?5object?5X?3?5?$CFp@ 0000000180020ad0     JavaAccessBridge.obj
 0002:0000eae8       ??_C@_0CE@NAEKPPND@?$FLINFO?$FN?3?5?5?5global?5reference?5dele@ 0000000180020ae8     JavaAccessBridge.obj
 0002:0000eb10       ??_C@_0CC@DPMNCGAA@?$FLERROR?$FN?3?5windowsThreadJNIEnv?5?$DN?$DN@ 0000000180020b10     JavaAccessBridge.obj
 0002:0000eb38       ??_C@_0DF@HMNKBJGB@?$FLINFO?$FN?3?5?5?5adding?5Java?5event?5typ@ 0000000180020b38     JavaAccessBridge.obj
 0002:0000eb70       ??_C@_0CO@OPGCCICC@?$FLINFO?$FN?3?5?5?5found?5HWND?0?5javaEvent@ 0000000180020b70     JavaAccessBridge.obj
 0002:0000eba0       ??_C@_0CP@MJMPLPDN@?$FLINFO?$FN?3?5?5?5union?5of?5all?5Java?5AT?5@ 0000000180020ba0     JavaAccessBridge.obj
 0002:0000ebd0       ??_C@_0FO@PMMLAHPF@?$FLINFO?$FN?3?5?5?5no?5other?5AT?5wanted?5th@ 0000000180020bd0     JavaAccessBridge.obj
 0002:0000ec30       ??_C@_0DJ@DFJLLFAC@?$FLINFO?$FN?3?5?5?5removing?5Java?5event?5t@ 0000000180020c30     JavaAccessBridge.obj
 0002:0000ec70       ??_C@_0FO@LBFBGKHJ@?$FLINFO?$FN?3?5?5?5no?5other?5AT?5wanted?5th@ 0000000180020c70     JavaAccessBridge.obj
 0002:0000ecd0       ??_C@_0DN@PDHOAFNL@?$FLINFO?$FN?3?5?5?5adding?5Accesibility?5e@ 0000000180020cd0     JavaAccessBridge.obj
 0002:0000ed10       ??_C@_0DH@EPKDBDGJ@?$FLINFO?$FN?3?5?5?5found?5HWND?0?5accessibi@ 0000000180020d10     JavaAccessBridge.obj
 0002:0000ed48       ??_C@_0DI@IJKEHAJM@?$FLINFO?$FN?3?5?5?5union?5of?5all?5Accessib@ 0000000180020d48     JavaAccessBridge.obj
 0002:0000ed80       ??_C@_0GG@CGBBDJFJ@?$FLINFO?$FN?3?5?5?5no?5other?5AT?5wanted?5th@ 0000000180020d80     JavaAccessBridge.obj
 0002:0000edf0       ??_C@_0EB@PJLIMJAJ@?$FLINFO?$FN?3?5?5?5removing?5Accesibility@ 0000000180020df0     JavaAccessBridge.obj
 0002:0000ee40       ??_C@_0GH@FGGMCIOE@?$FLINFO?$FN?3?5?5?5no?5other?5AT?5wanted?5th@ 0000000180020e40     JavaAccessBridge.obj
 0002:0000eeb0       ??_C@_0GL@DLLNHKDB@?$FLINFO?$FN?3?5Java_com_sun_java_acces@ 0000000180020eb0     JavaAccessBridge.obj
 0002:0000ef20       ??_C@_0BI@GOJFHMPI@?$FLINFO?$FN?3?5?5?5sending?5to?5AT@ 0000000180020f20     JavaAccessBridge.obj
 0002:0000ef40       ??_C@_0EM@NDPMFJGH@?$FLINFO?$FN?3?5?5?5GlobalRef?8d?5Event?3?5?$CF0@ 0000000180020f40     JavaAccessBridge.obj
 0002:0000ef90       ??_C@_0CN@HLLEMELD@?$FLINFO?$FN?3?5?5done?5with?5propertyCare@ 0000000180020f90     JavaAccessBridge.obj
 0002:0000efc0       ??_C@_0HB@FIEPPBDD@?$FLINFO?$FN?3?5Java_com_sun_java_acces@ 0000000180020fc0     JavaAccessBridge.obj
 0002:0000f040       ??_C@_0ED@LNNGOPDA@?$FLINFO?$FN?3?5?5GlobalRef?8d?5Event?3?5?$CF01@ 0000000180021040     JavaAccessBridge.obj
 0002:0000f088       ??_C@_0BL@ENCPOIKC@java?1lang?1OutOfMemoryError@ 0000000180021088     JavaAccessBridge.obj
 0002:0000f0a8       ??_C@_1O@CEDCILHN@?$AA?$CI?$AAn?$AAu?$AAl?$AAl?$AA?$CJ@ 00000001800210a8     JavaAccessBridge.obj
 0002:0000f0b8       ??_C@_0DE@IIPLELBE@?$FLINFO?$FN?3?5?5?5done?5with?5propertyDes@ 00000001800210b8     JavaAccessBridge.obj
 0002:0000f0f0       ??_C@_0GK@FGEOELMA@?$FLINFO?$FN?3?5Java_com_sun_java_acces@ 00000001800210f0     JavaAccessBridge.obj
 0002:0000f160       ??_C@_0EK@CCMALPPF@?$FLINFO?$FN?3?5?5GlobalRef?8d?5Event?3?5?$CF01@ 0000000180021160     JavaAccessBridge.obj
 0002:0000f1b0       ??_C@_0CM@LHIINGJI@?$FLINFO?$FN?3?5?5done?5with?5propertyName@ 00000001800211b0     JavaAccessBridge.obj
 0002:0000f1e0       ??_C@_0GH@NDFIEILD@?$FLINFO?$FN?3?5Java_com_sun_java_acces@ 00000001800211e0     JavaAccessBridge.obj
 0002:0000f248       ??_C@_0DC@IDEPNPKP@?$FLINFO?$FN?3?5?5?5done?5with?5propertySel@ 0000000180021248     JavaAccessBridge.obj
 0002:0000f280       ??_C@_0GL@LHHKNKCF@?$FLINFO?$FN?3?5Java_com_sun_java_acces@ 0000000180021280     JavaAccessBridge.obj
 0002:0000f2f0       ??_C@_0CN@HPCDPOIL@?$FLINFO?$FN?3?5?5done?5with?5propertyStat@ 00000001800212f0     JavaAccessBridge.obj
 0002:0000f320       ??_C@_0GC@GKPNHBKM@?$FLINFO?$FN?3?5Java_com_sun_java_acces@ 0000000180021320     JavaAccessBridge.obj
 0002:0000f388       ??_C@_0CM@MKJMCAOF@?$FLINFO?$FN?3?5?5done?5with?5propertyText@ 0000000180021388     JavaAccessBridge.obj
 0002:0000f3c0       ??_C@_0GL@LMHLMBIC@?$FLINFO?$FN?3?5Java_com_sun_java_acces@ 00000001800213c0     JavaAccessBridge.obj
 0002:0000f430       ??_C@_0CO@LJOPOKFE@?$FLINFO?$FN?3?5?5?5done?5with?5propertyVal@ 0000000180021430     JavaAccessBridge.obj
 0002:0000f460       ??_C@_0GJ@PEJPEKID@?$FLINFO?$FN?3?5Java_com_sun_java_acces@ 0000000180021460     JavaAccessBridge.obj
 0002:0000f4d0       ??_C@_0DD@LNFBPAKO@?$FLINFO?$FN?3?5?5done?5with?5propertyVisi@ 00000001800214d0     JavaAccessBridge.obj
 0002:0000f510       ??_C@_0HD@JKCIIIAC@?$FLINFO?$FN?3?5Java_com_sun_java_acces@ 0000000180021510     JavaAccessBridge.obj
 0002:0000f588       ??_C@_0BH@HMENLEAO@?$FLINFO?$FN?3?5?5sending?5to?5AT@ 0000000180021588     JavaAccessBridge.obj
 0002:0000f5a0       ??_C@_0II@CFAAOCOP@?$FLINFO?$FN?3?5?5?5GlobalRef?8d?5Event?3?5?$CF0@ 00000001800215a0     JavaAccessBridge.obj
 0002:0000f628       ??_C@_0CN@LGDOHOEO@?$FLINFO?$FN?3?5?5done?5with?5propertyChil@ 0000000180021628     JavaAccessBridge.obj
 0002:0000f660       ??_C@_0HO@MNNKGDDP@?$FLINFO?$FN?3?5Java_com_sun_java_acces@ 0000000180021660     JavaAccessBridge.obj
 0002:0000f6e0       ??_C@_0JN@BMGHKMMD@?$FLINFO?$FN?3?5?5GlobalRef?8d?5Event?3?5?$CF01@ 00000001800216e0     JavaAccessBridge.obj
 0002:0000f780       ??_C@_0CO@GOOPPCJH@?$FLINFO?$FN?3?5?5done?5with?5propertyActi@ 0000000180021780     JavaAccessBridge.obj
 0002:0000f7b0       ??_C@_0GP@NILNKGMP@?$FLINFO?$FN?3?5Java_com_sun_java_acces@ 00000001800217b0     JavaAccessBridge.obj
 0002:0000f820       ??_C@_0BA@KOMOFG@?5?5sending?5to?5AT@ 0000000180021820     JavaAccessBridge.obj
 0002:0000f830       ??_C@_0DC@FMNGEBKI@?$FLINFO?$FN?3?5?5done?5with?5propertyTabl@ 0000000180021830     JavaAccessBridge.obj
 0002:0000f868       ??_C@_0DA@ODJJOIDA@?$FLINFO?$FN?3?5Firing?5event?5id?5?$DN?5?$CFd?$CI?$CFp@ 0000000180021868     JavaAccessBridge.obj
 0002:0000f898       ??_C@_0CF@EPNHEIBO@?$FLINFO?$FN?3?5?5?5done?5with?5firing?5AWT?5@ 0000000180021898     JavaAccessBridge.obj
 0002:0000f8c0       ??_C@_0DI@NNGMMOBO@?$FLINFO?$FN?3?5Firing?5event?5id?5?$DN?5?$CFd?$CI?$CFp@ 00000001800218c0     JavaAccessBridge.obj
 0002:0000f8f8       ??_C@_0DJ@GLLLDFPO@?$FLINFO?$FN?3?5javaEventMask?5?$DN?5?$CFX?5even@ 00000001800218f8     JavaAccessBridge.obj
 0002:0000f938       ??_C@_1CO@CCIONPKC@?$AAA?$AAc?$AAc?$AAe?$AAs?$AAs?$AAB?$AAr?$AAi?$AAd?$AAg?$AAe?$AA?4?$AAj?$AAa@ 0000000180021938     JavaAccessBridge.obj
 0002:0000f968       _pDefaultRawDllMain        0000000180021968     MSVCRT:dll_dllmain.obj
 0002:0000f968       _pRawDllMain               0000000180021968     MSVCRT:dll_dllmain.obj
 0002:0000f978       ??_7exception@std@@6B@     0000000180021978     MSVCRT:throw_bad_alloc.obj
 0002:0000f988       ??_C@_0BC@EOODALEL@Unknown?5exception@ 0000000180021988     MSVCRT:throw_bad_alloc.obj
 0002:0000f9a8       ??_7bad_alloc@std@@6B@     00000001800219a8     MSVCRT:throw_bad_alloc.obj
 0002:0000f9b8       ??_C@_0P@GHFPNOJB@bad?5allocation@ 00000001800219b8     MSVCRT:throw_bad_alloc.obj
 0002:0000f9d0       ??_7bad_array_new_length@std@@6B@ 00000001800219d0     MSVCRT:throw_bad_alloc.obj
 0002:0000f9e0       ??_C@_0BF@KINCDENJ@bad?5array?5new?5length@ 00000001800219e0     MSVCRT:throw_bad_alloc.obj
 0002:0000fa10       __xmm@ffffffffffffffffffffffffffffffff 0000000180021a10     MSVCRT:utility.obj
 0002:0000fa28       ??_7type_info@@6B@         0000000180021a28     MSVCRT:std_type_info_static.obj
 0002:0000fa30       _load_config_used          0000000180021a30     MSVCRT:loadcfg.obj
 0002:0000fc00       ??_R4exception@std@@6B@    0000000180021c00     MSVCRT:throw_bad_alloc.obj
 0002:0000fc28       ??_R3exception@std@@8      0000000180021c28     MSVCRT:throw_bad_alloc.obj
 0002:0000fc40       ??_R2exception@std@@8      0000000180021c40     MSVCRT:throw_bad_alloc.obj
 0002:0000fc50       ??_R1A@?0A@EA@exception@std@@8 0000000180021c50     MSVCRT:throw_bad_alloc.obj
 0002:0000fc78       ??_R4bad_alloc@std@@6B@    0000000180021c78     MSVCRT:throw_bad_alloc.obj
 0002:0000fca0       ??_R3bad_alloc@std@@8      0000000180021ca0     MSVCRT:throw_bad_alloc.obj
 0002:0000fcb8       ??_R2bad_alloc@std@@8      0000000180021cb8     MSVCRT:throw_bad_alloc.obj
 0002:0000fcd0       ??_R1A@?0A@EA@bad_alloc@std@@8 0000000180021cd0     MSVCRT:throw_bad_alloc.obj
 0002:0000fcf8       ??_R4bad_array_new_length@std@@6B@ 0000000180021cf8     MSVCRT:throw_bad_alloc.obj
 0002:0000fd20       ??_R3bad_array_new_length@std@@8 0000000180021d20     MSVCRT:throw_bad_alloc.obj
 0002:0000fd38       ??_R2bad_array_new_length@std@@8 0000000180021d38     MSVCRT:throw_bad_alloc.obj
 0002:0000fd58       ??_R1A@?0A@EA@bad_array_new_length@std@@8 0000000180021d58     MSVCRT:throw_bad_alloc.obj
 0002:0000fd80       ??_R4type_info@@6B@        0000000180021d80     MSVCRT:std_type_info_static.obj
 0002:0000fda8       ??_R3type_info@@8          0000000180021da8     MSVCRT:std_type_info_static.obj
 0002:0000fdc0       ??_R2type_info@@8          0000000180021dc0     MSVCRT:std_type_info_static.obj
 0002:0000fdd0       ??_R1A@?0A@EA@type_info@@8 0000000180021dd0     MSVCRT:std_type_info_static.obj
 0002:0000fdf4       __volatile_metadata        0000000180021df4     <linker-defined>
 0002:00010168       __rtc_iaa                  0000000180022168     MSVCRT:initsect.obj
 0002:00010170       __rtc_izz                  0000000180022170     MSVCRT:initsect.obj
 0002:00010178       __rtc_taa                  0000000180022178     MSVCRT:initsect.obj
 0002:00010180       __rtc_tzz                  0000000180022180     MSVCRT:initsect.obj
 0002:00010608       _TI2?AVbad_alloc@std@@     0000000180022608     MSVCRT:throw_bad_alloc.obj
 0002:00010628       _CTA2?AVbad_alloc@std@@    0000000180022628     MSVCRT:throw_bad_alloc.obj
 0002:00010640       _CT??_R0?AVbad_alloc@std@@@8??0bad_alloc@std@@QEAA@AEBV01@@Z24 0000000180022640     MSVCRT:throw_bad_alloc.obj
 0002:00010668       _CT??_R0?AVexception@std@@@8??0exception@std@@QEAA@AEBV01@@Z24 0000000180022668     MSVCRT:throw_bad_alloc.obj
 0002:00010690       _TI3?AVbad_array_new_length@std@@ 0000000180022690     MSVCRT:throw_bad_alloc.obj
 0002:000106b0       _CTA3?AVbad_array_new_length@std@@ 00000001800226b0     MSVCRT:throw_bad_alloc.obj
 0002:000106d0       _CT??_R0?AVbad_array_new_length@std@@@8??0bad_array_new_length@std@@QEAA@AEBV01@@Z24 00000001800226d0     MSVCRT:throw_bad_alloc.obj
 0002:00011100       __IMPORT_DESCRIPTOR_KERNEL32 0000000180023100     kernel32:KERNEL32.dll
 0002:00011114       __IMPORT_DESCRIPTOR_USER32 0000000180023114     user32:USER32.dll
 0002:00011128       __IMPORT_DESCRIPTOR_jawt   0000000180023128     jawt:jawt.dll
 0002:0001113c       __IMPORT_DESCRIPTOR_VCRUNTIME140 000000018002313c     vcruntime:VCRUNTIME140.dll
 0002:00011150       __IMPORT_DESCRIPTOR_api-ms-win-crt-string-l1-1-0 0000000180023150     ucrt:api-ms-win-crt-string-l1-1-0.dll
 0002:00011164       __IMPORT_DESCRIPTOR_api-ms-win-crt-runtime-l1-1-0 0000000180023164     ucrt:api-ms-win-crt-runtime-l1-1-0.dll
 0002:00011178       __IMPORT_DESCRIPTOR_api-ms-win-crt-stdio-l1-1-0 0000000180023178     ucrt:api-ms-win-crt-stdio-l1-1-0.dll
 0002:0001118c       __IMPORT_DESCRIPTOR_api-ms-win-crt-environment-l1-1-0 000000018002318c     ucrt:api-ms-win-crt-environment-l1-1-0.dll
 0002:000111a0       __IMPORT_DESCRIPTOR_api-ms-win-crt-heap-l1-1-0 00000001800231a0     ucrt:api-ms-win-crt-heap-l1-1-0.dll
 0002:000111b4       __NULL_IMPORT_DESCRIPTOR   00000001800231b4     kernel32:KERNEL32.dll
 0003:00000000       __security_cookie_complement 0000000180024000     MSVCRT:gs_cookie.obj
 0003:00000008       __security_cookie          0000000180024008     MSVCRT:gs_cookie.obj
 0003:00000010       _fltused                   0000000180024010     MSVCRT:fltused.obj
 0003:00000014       __scrt_native_dllmain_reason 0000000180024014     MSVCRT:utility.obj
 0003:00000018       __isa_available            0000000180024018     MSVCRT:cpu_disp.obj
 0003:0000001c       __isa_enabled              000000018002401c     MSVCRT:cpu_disp.obj
 0003:00000020       __memset_fast_string_threshold 0000000180024020     MSVCRT:cpu_disp.obj
 0003:00000028       __memset_nt_threshold      0000000180024028     MSVCRT:cpu_disp.obj
 0003:00000030       __scrt_ucrt_dll_is_in_use  0000000180024030     MSVCRT:ucrt_stubs.obj
 0003:00000038       ??_R0?AVbad_alloc@std@@@8  0000000180024038     MSVCRT:throw_bad_alloc.obj
 0003:00000060       ??_R0?AVexception@std@@@8  0000000180024060     MSVCRT:throw_bad_alloc.obj
 0003:00000088       ??_R0?AVbad_array_new_length@std@@@8 0000000180024088     MSVCRT:throw_bad_alloc.obj
 0003:000000b8       ??_R0?AVtype_info@@@8      00000001800240b8     MSVCRT:std_type_info_static.obj
 0003:000000e0       ?JavaBridgeThreadId@@3KA   00000001800240e0     AccessBridgeATInstance.obj
 0003:000000e8       ?_OptionsStorage@?1??__local_stdio_printf_options@@9@4_KA 00000001800240e8     AccessBridgeDebug.obj
 0003:000000f8       ?theFromJavaHelloMsgID@@3IA 00000001800240f8     AccessBridgeMessages.obj
 0003:000000fc       ?theFromWindowsHelloMsgID@@3IA 00000001800240fc     AccessBridgeMessages.obj
 0003:00000100       ?theJavaAccessBridge@@3PEAVJavaAccessBridge@@EA 0000000180024100     JavaAccessBridge.obj
 0003:00000108       ?theDialogWindow@@3PEAUHWND__@@EA 0000000180024108     JavaAccessBridge.obj
 0003:00000110       ?receiveMemoryIPCLock@@3U_RTL_CRITICAL_SECTION@@A 0000000180024110     JavaAccessBridge.obj
 0003:000006b0       ?__type_info_root_node@@3U__type_info_node@@A 00000001800246b0     MSVCRT:tncleanup.obj
 0003:000006c0       ?_OptionsStorage@?1??__local_stdio_scanf_options@@9@4_KA 00000001800246c0     MSVCRT:default_local_stdio_options.obj
 0003:000006c8       __scrt_current_native_startup_state 00000001800246c8     MSVCRT:utility.obj
 0003:000006d0       __scrt_native_startup_lock 00000001800246d0     MSVCRT:utility.obj
 0003:00000710       __scrt_debugger_hook_flag  0000000180024710     MSVCRT:utility_desktop.obj
 0003:00000714       __favor                    0000000180024714     MSVCRT:cpu_disp.obj
 0003:00000718       __dyn_tls_init_callback    0000000180024718     <common>

 entry point at        0001:0000f9e0

 Static symbols

 0000:fffd8000       .debug$S                   0000000180000000     javaaccessbridge.exp
 0000:fffd8000       .debug$S                   0000000180000000     vcruntime:VCRUNTIME140.dll
 0000:fffd8000       .debug$S                   0000000180000000     vcruntime:VCRUNTIME140.dll
 0000:fffd8000       .debug$S                   0000000180000000     vcruntime:VCRUNTIME140.dll
 0000:fffd8000       .debug$S                   0000000180000000     vcruntime:VCRUNTIME140.dll
 0000:fffd8000       .debug$S                   0000000180000000     vcruntime:VCRUNTIME140.dll
 0000:fffd8000       .debug$S                   0000000180000000     vcruntime:VCRUNTIME140.dll
 0000:fffd8000       .debug$S                   0000000180000000     vcruntime:VCRUNTIME140.dll
 0000:fffd8000       .debug$S                   0000000180000000     vcruntime:VCRUNTIME140.dll
 0000:fffd8000       .debug$S                   0000000180000000     vcruntime:VCRUNTIME140.dll
 0000:fffd8000       .debug$S                   0000000180000000     ucrt:api-ms-win-crt-environment-l1-1-0.dll
 0000:fffd8000       .debug$S                   0000000180000000     ucrt:api-ms-win-crt-heap-l1-1-0.dll
 0000:fffd8000       .debug$S                   0000000180000000     ucrt:api-ms-win-crt-heap-l1-1-0.dll
 0000:fffd8000       .debug$S                   0000000180000000     ucrt:api-ms-win-crt-heap-l1-1-0.dll
 0000:fffd8000       .debug$S                   0000000180000000     ucrt:api-ms-win-crt-runtime-l1-1-0.dll
 0000:fffd8000       .debug$S                   0000000180000000     ucrt:api-ms-win-crt-runtime-l1-1-0.dll
 0000:fffd8000       .debug$S                   0000000180000000     ucrt:api-ms-win-crt-runtime-l1-1-0.dll
 0000:fffd8000       .debug$S                   0000000180000000     ucrt:api-ms-win-crt-runtime-l1-1-0.dll
 0000:fffd8000       .debug$S                   0000000180000000     ucrt:api-ms-win-crt-runtime-l1-1-0.dll
 0000:fffd8000       .debug$S                   0000000180000000     ucrt:api-ms-win-crt-runtime-l1-1-0.dll
 0000:fffd8000       .debug$S                   0000000180000000     ucrt:api-ms-win-crt-runtime-l1-1-0.dll
 0000:fffd8000       .debug$S                   0000000180000000     ucrt:api-ms-win-crt-runtime-l1-1-0.dll
 0000:fffd8000       .debug$S                   0000000180000000     ucrt:api-ms-win-crt-runtime-l1-1-0.dll
 0000:fffd8000       .debug$S                   0000000180000000     ucrt:api-ms-win-crt-runtime-l1-1-0.dll
 0000:fffd8000       .debug$S                   0000000180000000     ucrt:api-ms-win-crt-runtime-l1-1-0.dll
 0000:fffd8000       .debug$S                   0000000180000000     ucrt:api-ms-win-crt-runtime-l1-1-0.dll
 0000:fffd8000       .debug$S                   0000000180000000     ucrt:api-ms-win-crt-runtime-l1-1-0.dll
 0000:fffd8000       .debug$S                   0000000180000000     ucrt:api-ms-win-crt-stdio-l1-1-0.dll
 0000:fffd8000       .debug$S                   0000000180000000     ucrt:api-ms-win-crt-stdio-l1-1-0.dll
 0000:fffd8000       .debug$S                   0000000180000000     ucrt:api-ms-win-crt-stdio-l1-1-0.dll
 0000:fffd8000       .debug$S                   0000000180000000     ucrt:api-ms-win-crt-stdio-l1-1-0.dll
 0000:fffd8000       .debug$S                   0000000180000000     ucrt:api-ms-win-crt-stdio-l1-1-0.dll
 0000:fffd8000       .debug$S                   0000000180000000     ucrt:api-ms-win-crt-string-l1-1-0.dll
 0000:fffd8000       .debug$S                   0000000180000000     ucrt:api-ms-win-crt-string-l1-1-0.dll
 0000:fffd8000       .debug$S                   0000000180000000     ucrt:api-ms-win-crt-string-l1-1-0.dll
 0000:fffd8000       .debug$S                   0000000180000000     ucrt:api-ms-win-crt-string-l1-1-0.dll
 0000:fffd8000       .debug$S                   0000000180000000     ucrt:api-ms-win-crt-string-l1-1-0.dll
 0000:fffd8000       .debug$S                   0000000180000000     ucrt:api-ms-win-crt-string-l1-1-0.dll
 0000:fffd8000       .debug$S                   0000000180000000     ucrt:api-ms-win-crt-string-l1-1-0.dll
 0000:fffd8000       .debug$S                   0000000180000000     ucrt:api-ms-win-crt-string-l1-1-0.dll
 0000:fffd8000       .debug$S                   0000000180000000     kernel32:KERNEL32.dll
 0000:fffd8000       .debug$S                   0000000180000000     kernel32:KERNEL32.dll
 0000:fffd8000       .debug$S                   0000000180000000     kernel32:KERNEL32.dll
 0000:fffd8000       .debug$S                   0000000180000000     kernel32:KERNEL32.dll
 0000:fffd8000       .debug$S                   0000000180000000     kernel32:KERNEL32.dll
 0000:fffd8000       .debug$S                   0000000180000000     kernel32:KERNEL32.dll
 0000:fffd8000       .debug$S                   0000000180000000     kernel32:KERNEL32.dll
 0000:fffd8000       .debug$S                   0000000180000000     kernel32:KERNEL32.dll
 0000:fffd8000       .debug$S                   0000000180000000     kernel32:KERNEL32.dll
 0000:fffd8000       .debug$S                   0000000180000000     kernel32:KERNEL32.dll
 0000:fffd8000       .debug$S                   0000000180000000     kernel32:KERNEL32.dll
 0000:fffd8000       .debug$S                   0000000180000000     kernel32:KERNEL32.dll
 0000:fffd8000       .debug$S                   0000000180000000     kernel32:KERNEL32.dll
 0000:fffd8000       .debug$S                   0000000180000000     kernel32:KERNEL32.dll
 0000:fffd8000       .debug$S                   0000000180000000     kernel32:KERNEL32.dll
 0000:fffd8000       .debug$S                   0000000180000000     kernel32:KERNEL32.dll
 0000:fffd8000       .debug$S                   0000000180000000     kernel32:KERNEL32.dll
 0000:fffd8000       .debug$S                   0000000180000000     kernel32:KERNEL32.dll
 0000:fffd8000       .debug$S                   0000000180000000     kernel32:KERNEL32.dll
 0000:fffd8000       .debug$S                   0000000180000000     kernel32:KERNEL32.dll
 0000:fffd8000       .debug$S                   0000000180000000     kernel32:KERNEL32.dll
 0000:fffd8000       .debug$S                   0000000180000000     kernel32:KERNEL32.dll
 0000:fffd8000       .debug$S                   0000000180000000     kernel32:KERNEL32.dll
 0000:fffd8000       .debug$S                   0000000180000000     kernel32:KERNEL32.dll
 0000:fffd8000       .debug$S                   0000000180000000     kernel32:KERNEL32.dll
 0000:fffd8000       .debug$S                   0000000180000000     kernel32:KERNEL32.dll
 0000:fffd8000       .debug$S                   0000000180000000     kernel32:KERNEL32.dll
 0000:fffd8000       .debug$S                   0000000180000000     user32:USER32.dll
 0000:fffd8000       .debug$S                   0000000180000000     user32:USER32.dll
 0000:fffd8000       .debug$S                   0000000180000000     user32:USER32.dll
 0000:fffd8000       .debug$S                   0000000180000000     user32:USER32.dll
 0000:fffd8000       .debug$S                   0000000180000000     user32:USER32.dll
 0000:fffd8000       .debug$S                   0000000180000000     user32:USER32.dll
 0000:fffd8000       .debug$S                   0000000180000000     user32:USER32.dll
 0000:fffd8000       .debug$S                   0000000180000000     user32:USER32.dll
 0000:fffd8000       .debug$S                   0000000180000000     user32:USER32.dll
 0000:fffd8000       .debug$S                   0000000180000000     jawt:jawt.dll
 0001:000000a4       ?JavaBridgeThread@@YAIPEAX@Z 00000001800010a4 f   AccessBridgeATInstance.obj
 0001:00000140       ?do_event@@YAXPEADHPEAUHWND__@@1@Z 0000000180001140 f   AccessBridgeATInstance.obj
 0001:0000f690       $$000000                   0000000180010690     MSVCRT:amdsecgs.obj
 0001:0000f6c0       ?dllmain_crt_dispatch@@YAHQEAUHINSTANCE__@@KQEAX@Z 00000001800106c0 f   MSVCRT:dll_dllmain.obj
 0001:0000f710       ?dllmain_crt_process_attach@@YAHQEAUHINSTANCE__@@QEAX@Z 0000000180010710 f   MSVCRT:dll_dllmain.obj
 0001:0000f828       ?dllmain_crt_process_detach@@YAH_N@Z 0000000180010828 f   MSVCRT:dll_dllmain.obj
 0001:0000f8ac       ?dllmain_dispatch@@YAHQEAUHINSTANCE__@@KQEAX@Z 00000001800108ac f   MSVCRT:dll_dllmain.obj
 0001:0000fcc8       capture_previous_context   0000000180010cc8 f   MSVCRT:gs_report.obj
 0001:000105b0       $$000000                   00000001800115b0     MSVCRT:guard_dispatch.obj
 0001:000105d0       $$000000                   00000001800115d0     MSVCRT:guard_xfg_dispatch.obj
 0001:000105e6       ?fin$0@?0??dllmain_crt_process_attach@@YAHQEAUHINSTANCE__@@QEAX@Z@4HA 00000001800115e6 f   MSVCRT:dll_dllmain.obj
 0001:000105fd       ?fin$0@?0??dllmain_crt_process_detach@@YAH_N@Z@4HA 00000001800115fd f   MSVCRT:dll_dllmain.obj
 0001:00010616       ?fin$1@?0??dllmain_crt_process_detach@@YAH_N@Z@4HA 0000000180011616 f   MSVCRT:dll_dllmain.obj
 0001:0001062a       ?filt$0@?0??dllmain_dispatch@@YAHQEAUHINSTANCE__@@KQEAX@Z@4HA 000000018001162a f   MSVCRT:dll_dllmain.obj
 0001:00010660       __scrt_is_nonwritable_in_current_image$filt$0 0000000180011660 f   MSVCRT:utility.obj
 0002:0000f9f8       GS_ExceptionPointers       00000001800219f8     MSVCRT:gs_report.obj
 0002:00010188       $unwind$??0AccessBridgeATInstance@@QEAA@PEAUHWND__@@0PEADPEAV0@@Z 0000000180022188     AccessBridgeATInstance.obj
 0002:00010188       $unwind$??1AccessBridgeATInstance@@QEAA@XZ 0000000180022188     AccessBridgeATInstance.obj
 0002:00010188       $unwind$??0AccessBridgeJavaEntryPoints@@QEAA@PEAUJNIEnv_@@PEAV_jobject@@@Z 0000000180022188     AccessBridgeJavaEntryPoints.obj
 0002:00010188       $unwind$??0JavaAccessBridge@@QEAA@PEAUHINSTANCE__@@@Z 0000000180022188     JavaAccessBridge.obj
 0002:00010188       $unwind$__raise_securityfailure 0000000180022188     MSVCRT:gs_report.obj
 0002:00010188       $unwind$??2@YAPEAX_K@Z     0000000180022188     MSVCRT:new_scalar.obj
 0002:00010188       $unwind$??_Gtype_info@@UEAAPEAXI@Z 0000000180022188     MSVCRT:std_type_info_static.obj
 0002:00010188       $unwind$??0bad_alloc@std@@QEAA@AEBV01@@Z 0000000180022188     MSVCRT:throw_bad_alloc.obj
 0002:00010188       $unwind$??0bad_array_new_length@std@@QEAA@AEBV01@@Z 0000000180022188     MSVCRT:throw_bad_alloc.obj
 0002:00010188       $unwind$??0exception@std@@QEAA@AEBV01@@Z 0000000180022188     MSVCRT:throw_bad_alloc.obj
 0002:00010188       $unwind$__scrt_initialize_crt 0000000180022188     MSVCRT:utility.obj
 0002:00010188       $unwind$__scrt_initialize_onexit_tables 0000000180022188     MSVCRT:utility.obj
 0002:00010188       $unwind$__scrt_release_startup_lock 0000000180022188     MSVCRT:utility.obj
 0002:00010188       $unwind$__scrt_uninitialize_crt 0000000180022188     MSVCRT:utility.obj
 0002:00010190       $unwind$?initiateIPC@AccessBridgeATInstance@@QEAA_JXZ 0000000180022190     AccessBridgeATInstance.obj
 0002:00010190       $unwind$?postHelloToWindowsDLLMsg@JavaAccessBridge@@QEAAXPEAUHWND__@@@Z 0000000180022190     JavaAccessBridge.obj
 0002:0001019c       $unwind$?sendAccessibilityEventPackage@AccessBridgeATInstance@@QEAA_JPEADHJ@Z 000000018002219c     AccessBridgeATInstance.obj
 0002:0001019c       $unwind$?sendJavaEventPackage@AccessBridgeATInstance@@QEAA_JPEADHJ@Z 000000018002219c     AccessBridgeATInstance.obj
 0002:0001019c       $unwind$?getAccessibleTableInfo@AccessBridgeJavaEntryPoints@@QEAAHPEAV_jobject@@PEAUAccessibleTableInfoTag@@@Z 000000018002219c     AccessBridgeJavaEntryPoints.obj
 0002:0001019c       $unwind$__scrt_dllmain_exception_filter 000000018002219c     MSVCRT:utility.obj
 0002:000101b0       $unwind$?JavaBridgeThread@@YAIPEAX@Z 00000001800221b0     AccessBridgeATInstance.obj
 0002:000101b8       $unwind$?do_event@@YAXPEADHPEAUHWND__@@1@Z 00000001800221b8     AccessBridgeATInstance.obj
 0002:000101b8       $unwind$?getAccessibleKeyBindings@AccessBridgeJavaEntryPoints@@QEAAHPEAV_jobject@@PEAUAccessibleKeyBindingsTag@@@Z 00000001800221b8     AccessBridgeJavaEntryPoints.obj
 0002:000101b8       $unwind$?getAccessibleTableCellInfo@AccessBridgeJavaEntryPoints@@QEAAHPEAV_jobject@@JJPEAUAccessibleTableCellInfoTag@@@Z 00000001800221b8     AccessBridgeJavaEntryPoints.obj
 0002:000101b8       $unwind$?getAccessibleTableColumnSelections@AccessBridgeJavaEntryPoints@@QEAAHPEAV_jobject@@JPEAJ@Z 00000001800221b8     AccessBridgeJavaEntryPoints.obj
 0002:000101b8       $unwind$?getAccessibleTableRowSelections@AccessBridgeJavaEntryPoints@@QEAAHPEAV_jobject@@JPEAJ@Z 00000001800221b8     AccessBridgeJavaEntryPoints.obj
 0002:000101b8       $unwind$?getAccessibleTextInfo@AccessBridgeJavaEntryPoints@@QEAAHPEAV_jobject@@PEAUAccessibleTextInfoTag@@JJ@Z 00000001800221b8     AccessBridgeJavaEntryPoints.obj
 0002:000101b8       $unwind$?processPackage@JavaAccessBridge@@QEAA_JPEADH@Z 00000001800221b8     JavaAccessBridge.obj
 0002:000101d0       $unwind$PrintDebugString   00000001800221d0     AccessBridgeDebug.obj
 0002:000101d0       $unwind$wPrintDebugString  00000001800221d0     AccessBridgeDebug.obj
 0002:000101d0       $unwind$wPrintJavaDebugString 00000001800221d0     AccessBridgeDebug.obj
 0002:000101d8       $unwind$initializeFileLogger 00000001800221d8     AccessBridgeDebug.obj
 0002:000101d8       $unwind$?getCurrentAccessibleValueFromContext@AccessBridgeJavaEntryPoints@@QEAAHPEAV_jobject@@PEAGF@Z 00000001800221d8     AccessBridgeJavaEntryPoints.obj
 0002:000101d8       $unwind$?getMaximumAccessibleValueFromContext@AccessBridgeJavaEntryPoints@@QEAAHPEAV_jobject@@PEAGF@Z 00000001800221d8     AccessBridgeJavaEntryPoints.obj
 0002:000101d8       $unwind$?getMinimumAccessibleValueFromContext@AccessBridgeJavaEntryPoints@@QEAAHPEAV_jobject@@PEAGF@Z 00000001800221d8     AccessBridgeJavaEntryPoints.obj
 0002:000101d8       $unwind$?getVirtualAccessibleName@AccessBridgeJavaEntryPoints@@QEAAHQEAV_jobject@@PEAGH@Z 00000001800221d8     AccessBridgeJavaEntryPoints.obj
 0002:000101f0       $unwind$finalizeFileLogger 00000001800221f0     AccessBridgeDebug.obj
 0002:000101f0       $unwind$getTimeStamp       00000001800221f0     AccessBridgeDebug.obj
 0002:000101f0       $unwind$?initBroadcastMessageIDs@@YAHXZ 00000001800221f0     AccessBridgeMessages.obj
 0002:000101f0       $unwind$__scrt_initialize_default_local_stdio_options 00000001800221f0     MSVCRT:default_local_stdio_options.obj
 0002:000101f0       $unwind$?dllmain_crt_dispatch@@YAHQEAUHINSTANCE__@@KQEAX@Z 00000001800221f0     MSVCRT:dll_dllmain.obj
 0002:000101f0       $unwind$__GSHandlerCheck   00000001800221f0     MSVCRT:gshandler.obj
 0002:000101f0       $unwind$__scrt_acquire_startup_lock 00000001800221f0     MSVCRT:utility.obj
 0002:000101f0       $unwind$__scrt_dllmain_after_initialize_c 00000001800221f0     MSVCRT:utility.obj
 0002:000101f0       $unwind$__scrt_dllmain_before_initialize_c 00000001800221f0     MSVCRT:utility.obj
 0002:000101f0       $unwind$__scrt_dllmain_crt_thread_attach 00000001800221f0     MSVCRT:utility.obj
 0002:000101f0       $unwind$__scrt_dllmain_crt_thread_detach 00000001800221f0     MSVCRT:utility.obj
 0002:000101f0       $unwind$__scrt_dllmain_uninitialize_c 00000001800221f0     MSVCRT:utility.obj
 0002:000101f0       $unwind$__scrt_dllmain_uninitialize_critical 00000001800221f0     MSVCRT:utility.obj
 0002:000101f8       $unwind$fprintf            00000001800221f8     AccessBridgeDebug.obj
 0002:00010204       $unwind$printf             0000000180022204     AccessBridgeDebug.obj
 0002:00010210       $unwind$?CallBooleanMethod@JNIEnv_@@QEAAEPEAV_jobject@@PEAU_jmethodID@@ZZ 0000000180022210     AccessBridgeJavaEntryPoints.obj
 0002:00010210       $unwind$?CallCharMethod@JNIEnv_@@QEAAGPEAV_jobject@@PEAU_jmethodID@@ZZ 0000000180022210     AccessBridgeJavaEntryPoints.obj
 0002:00010210       $unwind$?CallFloatMethod@JNIEnv_@@QEAAMPEAV_jobject@@PEAU_jmethodID@@ZZ 0000000180022210     AccessBridgeJavaEntryPoints.obj
 0002:00010210       $unwind$?CallIntMethod@JNIEnv_@@QEAAJPEAV_jobject@@PEAU_jmethodID@@ZZ 0000000180022210     AccessBridgeJavaEntryPoints.obj
 0002:00010210       $unwind$?CallObjectMethod@JNIEnv_@@QEAAPEAV_jobject@@PEAV2@PEAU_jmethodID@@ZZ 0000000180022210     AccessBridgeJavaEntryPoints.obj
 0002:00010210       $unwind$?CallVoidMethod@JNIEnv_@@QEAAXPEAV_jobject@@PEAU_jmethodID@@ZZ 0000000180022210     AccessBridgeJavaEntryPoints.obj
 0002:00010218       $unwind$?BuildJavaEntryPoints@AccessBridgeJavaEntryPoints@@QEAAHXZ 0000000180022218     AccessBridgeJavaEntryPoints.obj
 0002:00010230       $unwind$?addAccessibilityEventNotification@AccessBridgeJavaEntryPoints@@QEAAH_J@Z 0000000180022230     AccessBridgeJavaEntryPoints.obj
 0002:00010230       $unwind$?addJavaEventNotification@AccessBridgeJavaEntryPoints@@QEAAH_J@Z 0000000180022230     AccessBridgeJavaEntryPoints.obj
 0002:00010230       $unwind$?clearAccessibleSelectionFromContext@AccessBridgeJavaEntryPoints@@QEAAXPEAV_jobject@@@Z 0000000180022230     AccessBridgeJavaEntryPoints.obj
 0002:00010230       $unwind$?getAccessibleContextFromHWND@AccessBridgeJavaEntryPoints@@QEAAPEAV_jobject@@J@Z 0000000180022230     AccessBridgeJavaEntryPoints.obj
 0002:00010230       $unwind$?getAccessibleHyperlinkCount@AccessBridgeJavaEntryPoints@@QEAAJQEAV_jobject@@@Z 0000000180022230     AccessBridgeJavaEntryPoints.obj
 0002:00010230       $unwind$?getAccessibleSelectionCountFromContext@AccessBridgeJavaEntryPoints@@QEAAHPEAV_jobject@@@Z 0000000180022230     AccessBridgeJavaEntryPoints.obj
 0002:00010230       $unwind$?getAccessibleTableColumnSelectionCount@AccessBridgeJavaEntryPoints@@QEAAJPEAV_jobject@@@Z 0000000180022230     AccessBridgeJavaEntryPoints.obj
 0002:00010230       $unwind$?getAccessibleTableRowSelectionCount@AccessBridgeJavaEntryPoints@@QEAAJPEAV_jobject@@@Z 0000000180022230     AccessBridgeJavaEntryPoints.obj
 0002:00010230       $unwind$?getHWNDFromAccessibleContext@AccessBridgeJavaEntryPoints@@QEAAPEAUHWND__@@PEAV_jobject@@@Z 0000000180022230     AccessBridgeJavaEntryPoints.obj
 0002:00010230       $unwind$?getObjectDepth@AccessBridgeJavaEntryPoints@@QEAAJQEAV_jobject@@@Z 0000000180022230     AccessBridgeJavaEntryPoints.obj
 0002:00010230       $unwind$?getVisibleChildrenCount@AccessBridgeJavaEntryPoints@@QEAAHQEAV_jobject@@@Z 0000000180022230     AccessBridgeJavaEntryPoints.obj
 0002:00010230       $unwind$?isJavaWindow@AccessBridgeJavaEntryPoints@@QEAAHJ@Z 0000000180022230     AccessBridgeJavaEntryPoints.obj
 0002:00010230       $unwind$?removeAccessibilityEventNotification@AccessBridgeJavaEntryPoints@@QEAAH_J@Z 0000000180022230     AccessBridgeJavaEntryPoints.obj
 0002:00010230       $unwind$?removeJavaEventNotification@AccessBridgeJavaEntryPoints@@QEAAH_J@Z 0000000180022230     AccessBridgeJavaEntryPoints.obj
 0002:00010230       $unwind$?requestFocus@AccessBridgeJavaEntryPoints@@QEAAHQEAV_jobject@@@Z 0000000180022230     AccessBridgeJavaEntryPoints.obj
 0002:00010230       $unwind$?selectAllAccessibleSelectionFromContext@AccessBridgeJavaEntryPoints@@QEAAXPEAV_jobject@@@Z 0000000180022230     AccessBridgeJavaEntryPoints.obj
 0002:00010230       $unwind$??1JavaAccessBridge@@QEAA@XZ 0000000180022230     JavaAccessBridge.obj
 0002:00010230       $unwind$?releaseJavaObject@JavaAccessBridge@@QEAAXPEAV_jobject@@@Z 0000000180022230     JavaAccessBridge.obj
 0002:00010230       $unwind$AccessBridgeDialogProc 0000000180022230     JavaAccessBridge.obj
 0002:00010230       $unwind$DllMain            0000000180022230     JavaAccessBridge.obj
 0002:00010230       $unwind$Java_com_sun_java_accessibility_internal_AccessBridge_runDLL 0000000180022230     JavaAccessBridge.obj
 0002:00010230       $unwind$_RTC_Initialize    0000000180022230     MSVCRT:initsect.obj
 0002:00010230       $unwind$_RTC_Terminate     0000000180022230     MSVCRT:initsect.obj
 0002:00010230       $unwind$??_Gbad_alloc@std@@UEAAPEAXI@Z 0000000180022230     MSVCRT:throw_bad_alloc.obj
 0002:00010230       $unwind$??_Gbad_array_new_length@std@@UEAAPEAXI@Z 0000000180022230     MSVCRT:throw_bad_alloc.obj
 0002:00010230       $unwind$??_Gexception@std@@UEAAPEAXI@Z 0000000180022230     MSVCRT:throw_bad_alloc.obj
 0002:0001023c       $unwind$?getVersionInfo@AccessBridgeJavaEntryPoints@@QEAAHPEAUAccessBridgeVersionInfoTag@@@Z 000000018002223c     AccessBridgeJavaEntryPoints.obj
 0002:00010258       $unwind$?verifyAccessibleText@AccessBridgeJavaEntryPoints@@QEAAHPEAV_jobject@@@Z 0000000180022258     AccessBridgeJavaEntryPoints.obj
 0002:00010268       $unwind$?getAccessibleContextWithFocus@AccessBridgeJavaEntryPoints@@QEAAPEAV_jobject@@XZ 0000000180022268     AccessBridgeJavaEntryPoints.obj
 0002:00010268       $unwind$?getAccessibleParentFromContext@AccessBridgeJavaEntryPoints@@QEAAPEAV_jobject@@PEAV2@@Z 0000000180022268     AccessBridgeJavaEntryPoints.obj
 0002:00010268       $unwind$?getAccessibleTableColumnHeader@AccessBridgeJavaEntryPoints@@QEAAHPEAV_jobject@@PEAUAccessibleTableInfoTag@@@Z 0000000180022268     AccessBridgeJavaEntryPoints.obj
 0002:00010268       $unwind$?getAccessibleTableRowHeader@AccessBridgeJavaEntryPoints@@QEAAHPEAV_jobject@@PEAUAccessibleTableInfoTag@@@Z 0000000180022268     AccessBridgeJavaEntryPoints.obj
 0002:00010268       $unwind$?getActiveDescendent@AccessBridgeJavaEntryPoints@@QEAAPEAV_jobject@@QEAV2@@Z 0000000180022268     AccessBridgeJavaEntryPoints.obj
 0002:00010268       $unwind$?getTopLevelObject@AccessBridgeJavaEntryPoints@@QEAAPEAV_jobject@@QEAV2@@Z 0000000180022268     AccessBridgeJavaEntryPoints.obj
 0002:00010268       $unwind$?isSameObject@AccessBridgeJavaEntryPoints@@QEAAHPEAV_jobject@@0@Z 0000000180022268     AccessBridgeJavaEntryPoints.obj
 0002:00010268       $unwind$?WindowsATDestroyed@JavaAccessBridge@@QEAAXPEAUHWND__@@@Z 0000000180022268     JavaAccessBridge.obj
 0002:00010268       $unwind$?receiveMemoryPackage@JavaAccessBridge@@QEAAHPEAUHWND__@@J@Z 0000000180022268     JavaAccessBridge.obj
 0002:00010268       $unwind$Java_com_sun_java_accessibility_internal_AccessBridge_sendDebugString 0000000180022268     JavaAccessBridge.obj
 0002:00010268       $unwind$_DllMainCRTStartup 0000000180022268     MSVCRT:dll_dllmain.obj
 0002:00010278       $unwind$?activateAccessibleHyperlink@AccessBridgeJavaEntryPoints@@QEAAHPEAV_jobject@@0@Z 0000000180022278     AccessBridgeJavaEntryPoints.obj
 0002:00010278       $unwind$?addAccessibleSelectionFromContext@AccessBridgeJavaEntryPoints@@QEAAXPEAV_jobject@@H@Z 0000000180022278     AccessBridgeJavaEntryPoints.obj
 0002:00010278       $unwind$?getAccessibleChildFromContext@AccessBridgeJavaEntryPoints@@QEAAPEAV_jobject@@PEAV2@J@Z 0000000180022278     AccessBridgeJavaEntryPoints.obj
 0002:00010278       $unwind$?getAccessibleHypertextLinkIndex@AccessBridgeJavaEntryPoints@@QEAAJQEAV_jobject@@J@Z 0000000180022278     AccessBridgeJavaEntryPoints.obj
 0002:00010278       $unwind$?getAccessibleSelectionFromContext@AccessBridgeJavaEntryPoints@@QEAAPEAV_jobject@@PEAV2@H@Z 0000000180022278     AccessBridgeJavaEntryPoints.obj
 0002:00010278       $unwind$?getAccessibleTableColumn@AccessBridgeJavaEntryPoints@@QEAAJPEAV_jobject@@J@Z 0000000180022278     AccessBridgeJavaEntryPoints.obj
 0002:00010278       $unwind$?getAccessibleTableColumnDescription@AccessBridgeJavaEntryPoints@@QEAAPEAV_jobject@@PEAV2@J@Z 0000000180022278     AccessBridgeJavaEntryPoints.obj
 0002:00010278       $unwind$?getAccessibleTableRow@AccessBridgeJavaEntryPoints@@QEAAJPEAV_jobject@@J@Z 0000000180022278     AccessBridgeJavaEntryPoints.obj
 0002:00010278       $unwind$?getAccessibleTableRowDescription@AccessBridgeJavaEntryPoints@@QEAAPEAV_jobject@@PEAV2@J@Z 0000000180022278     AccessBridgeJavaEntryPoints.obj
 0002:00010278       $unwind$?getParentWithRole@AccessBridgeJavaEntryPoints@@QEAAPEAV_jobject@@QEAV2@PEBG@Z 0000000180022278     AccessBridgeJavaEntryPoints.obj
 0002:00010278       $unwind$?getParentWithRoleElseRoot@AccessBridgeJavaEntryPoints@@QEAAPEAV_jobject@@QEAV2@PEBG@Z 0000000180022278     AccessBridgeJavaEntryPoints.obj
 0002:00010278       $unwind$?isAccessibleChildSelectedFromContext@AccessBridgeJavaEntryPoints@@QEAAHPEAV_jobject@@H@Z 0000000180022278     AccessBridgeJavaEntryPoints.obj
 0002:00010278       $unwind$?isAccessibleTableColumnSelected@AccessBridgeJavaEntryPoints@@QEAAHPEAV_jobject@@J@Z 0000000180022278     AccessBridgeJavaEntryPoints.obj
 0002:00010278       $unwind$?isAccessibleTableRowSelected@AccessBridgeJavaEntryPoints@@QEAAHPEAV_jobject@@J@Z 0000000180022278     AccessBridgeJavaEntryPoints.obj
 0002:00010278       $unwind$?removeAccessibleSelectionFromContext@AccessBridgeJavaEntryPoints@@QEAAXPEAV_jobject@@H@Z 0000000180022278     AccessBridgeJavaEntryPoints.obj
 0002:00010278       $unwind$?setCaretPosition@AccessBridgeJavaEntryPoints@@QEAAHQEAV_jobject@@H@Z 0000000180022278     AccessBridgeJavaEntryPoints.obj
 0002:00010278       $unwind$?setTextContents@AccessBridgeJavaEntryPoints@@QEAAHQEAV_jobject@@PEBG@Z 0000000180022278     AccessBridgeJavaEntryPoints.obj
 0002:00010278       $unwind$?MemoryMappedFileCreated@JavaAccessBridge@@QEAA_JPEAUHWND__@@PEAD@Z 0000000180022278     JavaAccessBridge.obj
 0002:00010288       $unwind$?getAccessibleContextAt@AccessBridgeJavaEntryPoints@@QEAAPEAV_jobject@@JJPEAV2@@Z 0000000180022288     AccessBridgeJavaEntryPoints.obj
 0002:00010288       $unwind$?getAccessibleTableIndex@AccessBridgeJavaEntryPoints@@QEAAJPEAV_jobject@@JJ@Z 0000000180022288     AccessBridgeJavaEntryPoints.obj
 0002:00010288       $unwind$?getAccessibleTextLineBounds@AccessBridgeJavaEntryPoints@@QEAAHPEAV_jobject@@JPEAJ1@Z 0000000180022288     AccessBridgeJavaEntryPoints.obj
 0002:00010288       $unwind$?getAccessibleTextRect@AccessBridgeJavaEntryPoints@@QEAAHPEAV_jobject@@PEAUAccessibleTextRectInfoTag@@J@Z 0000000180022288     AccessBridgeJavaEntryPoints.obj
 0002:00010288       $unwind$?getCaretLocation@AccessBridgeJavaEntryPoints@@QEAAHPEAV_jobject@@PEAUAccessibleTextRectInfoTag@@J@Z 0000000180022288     AccessBridgeJavaEntryPoints.obj
 0002:00010288       $unwind$?selectTextRange@AccessBridgeJavaEntryPoints@@QEAAHQEAV_jobject@@HH@Z 0000000180022288     AccessBridgeJavaEntryPoints.obj
 0002:0001029c       $unwind$?getAccessibleContextInfo@AccessBridgeJavaEntryPoints@@QEAAHPEAV_jobject@@PEAUAccessibleContextInfoTag@@@Z 000000018002229c     AccessBridgeJavaEntryPoints.obj
 0002:000102b8       $unwind$?getAccessibleRelationSet@AccessBridgeJavaEntryPoints@@QEAAHPEAV_jobject@@PEAUAccessibleRelationSetInfoTag@@@Z 00000001800222b8     AccessBridgeJavaEntryPoints.obj
 0002:000102d0       $unwind$?getAccessibleActions@AccessBridgeJavaEntryPoints@@QEAAHPEAV_jobject@@PEAUAccessibleActionsTag@@@Z 00000001800222d0     AccessBridgeJavaEntryPoints.obj
 0002:000102d0       $unwind$?getAccessibleHypertext@AccessBridgeJavaEntryPoints@@QEAAHPEAV_jobject@@PEAUAccessibleHypertextInfoTag@@@Z 00000001800222d0     AccessBridgeJavaEntryPoints.obj
 0002:000102d0       $unwind$?getAccessibleHypertextExt@AccessBridgeJavaEntryPoints@@QEAAHQEAV_jobject@@JPEAUAccessibleHypertextInfoTag@@@Z 00000001800222d0     AccessBridgeJavaEntryPoints.obj
 0002:000102d0       $unwind$?getAccessibleIcons@AccessBridgeJavaEntryPoints@@QEAAHPEAV_jobject@@PEAUAccessibleIconsTag@@@Z 00000001800222d0     AccessBridgeJavaEntryPoints.obj
 0002:000102ec       $unwind$?getAccessibleHyperlink@AccessBridgeJavaEntryPoints@@QEAAHQEAV_jobject@@JPEAUAccessibleHyperlinkInfoTag@@@Z 00000001800222ec     AccessBridgeJavaEntryPoints.obj
 0002:00010304       $unwind$?doAccessibleActions@AccessBridgeJavaEntryPoints@@QEAAHPEAV_jobject@@PEAUAccessibleActionsToDoTag@@PEAJ@Z 0000000180022304     AccessBridgeJavaEntryPoints.obj
 0002:00010304       $unwind$?getAccessibleTextRange@AccessBridgeJavaEntryPoints@@QEAAHPEAV_jobject@@JJPEAGF@Z 0000000180022304     AccessBridgeJavaEntryPoints.obj
 0002:00010320       $unwind$?getAccessibleTextItems@AccessBridgeJavaEntryPoints@@QEAAHPEAV_jobject@@PEAUAccessibleTextItemsInfoTag@@J@Z 0000000180022320     AccessBridgeJavaEntryPoints.obj
 0002:0001033c       $unwind$?getAccessibleTextSelectionInfo@AccessBridgeJavaEntryPoints@@QEAAHPEAV_jobject@@PEAUAccessibleTextSelectionInfoTag@@@Z 000000018002233c     AccessBridgeJavaEntryPoints.obj
 0002:00010354       $unwind$?getAccessibleTextAttributes@AccessBridgeJavaEntryPoints@@QEAAHPEAV_jobject@@JPEAUAccessibleTextAttributesInfoTag@@@Z 0000000180022354     AccessBridgeJavaEntryPoints.obj
 0002:00010370       $unwind$?getTextAttributesInRange@AccessBridgeJavaEntryPoints@@QEAAHQEAV_jobject@@HHPEAUAccessibleTextAttributesInfoTag@@PEAF@Z 0000000180022370     AccessBridgeJavaEntryPoints.obj
 0002:00010390       $unwind$?getVisibleChildren@AccessBridgeJavaEntryPoints@@QEAAHQEAV_jobject@@HPEAUVisibleChildenInfoTag@@@Z 0000000180022390     AccessBridgeJavaEntryPoints.obj
 0002:000103ac       $unwind$?javaRun@JavaAccessBridge@@QEAAXPEAUJNIEnv_@@PEAV_jobject@@@Z 00000001800223ac     JavaAccessBridge.obj
 0002:000103c4       $unwind$?initWindow@JavaAccessBridge@@QEAAHXZ 00000001800223c4     JavaAccessBridge.obj
 0002:000103cc       $unwind$?addAccessibilityEventNotification@JavaAccessBridge@@QEAAX_JPEAUHWND__@@@Z 00000001800223cc     JavaAccessBridge.obj
 0002:000103cc       $unwind$?addJavaEventNotification@JavaAccessBridge@@QEAAX_JPEAUHWND__@@@Z 00000001800223cc     JavaAccessBridge.obj
 0002:000103cc       $unwind$?removeAccessibilityEventNotification@JavaAccessBridge@@QEAAX_JPEAUHWND__@@@Z 00000001800223cc     JavaAccessBridge.obj
 0002:000103cc       $unwind$?removeJavaEventNotification@JavaAccessBridge@@QEAAX_JPEAUHWND__@@@Z 00000001800223cc     JavaAccessBridge.obj
 0002:000103e4       $unwind$?javaShutdown@JavaAccessBridge@@QEAAXPEAUJNIEnv_@@PEAV_jobject@@@Z 00000001800223e4     JavaAccessBridge.obj
 0002:000103f8       $unwind$?fireCaretUpdate@JavaAccessBridge@@QEAAXPEAUJNIEnv_@@PEAV_jobject@@11@Z 00000001800223f8     JavaAccessBridge.obj
 0002:000103f8       $unwind$?fireFocusGained@JavaAccessBridge@@QEAAXPEAUJNIEnv_@@PEAV_jobject@@11@Z 00000001800223f8     JavaAccessBridge.obj
 0002:000103f8       $unwind$?fireFocusLost@JavaAccessBridge@@QEAAXPEAUJNIEnv_@@PEAV_jobject@@11@Z 00000001800223f8     JavaAccessBridge.obj
 0002:000103f8       $unwind$?fireMouseClicked@JavaAccessBridge@@QEAAXPEAUJNIEnv_@@PEAV_jobject@@11@Z 00000001800223f8     JavaAccessBridge.obj
 0002:000103f8       $unwind$?fireMouseEntered@JavaAccessBridge@@QEAAXPEAUJNIEnv_@@PEAV_jobject@@11@Z 00000001800223f8     JavaAccessBridge.obj
 0002:000103f8       $unwind$?fireMouseExited@JavaAccessBridge@@QEAAXPEAUJNIEnv_@@PEAV_jobject@@11@Z 00000001800223f8     JavaAccessBridge.obj
 0002:000103f8       $unwind$?fireMousePressed@JavaAccessBridge@@QEAAXPEAUJNIEnv_@@PEAV_jobject@@11@Z 00000001800223f8     JavaAccessBridge.obj
 0002:00010410       $unwind$?fireMenuCanceled@JavaAccessBridge@@QEAAXPEAUJNIEnv_@@PEAV_jobject@@11@Z 0000000180022410     JavaAccessBridge.obj
 0002:00010410       $unwind$?fireMenuDeselected@JavaAccessBridge@@QEAAXPEAUJNIEnv_@@PEAV_jobject@@11@Z 0000000180022410     JavaAccessBridge.obj
 0002:00010410       $unwind$?fireMenuSelected@JavaAccessBridge@@QEAAXPEAUJNIEnv_@@PEAV_jobject@@11@Z 0000000180022410     JavaAccessBridge.obj
 0002:00010410       $unwind$?fireMouseReleased@JavaAccessBridge@@QEAAXPEAUJNIEnv_@@PEAV_jobject@@11@Z 0000000180022410     JavaAccessBridge.obj
 0002:00010410       $unwind$?firePopupMenuCanceled@JavaAccessBridge@@QEAAXPEAUJNIEnv_@@PEAV_jobject@@11@Z 0000000180022410     JavaAccessBridge.obj
 0002:00010410       $unwind$?firePopupMenuWillBecomeInvisible@JavaAccessBridge@@QEAAXPEAUJNIEnv_@@PEAV_jobject@@11@Z 0000000180022410     JavaAccessBridge.obj
 0002:00010410       $unwind$?firePopupMenuWillBecomeVisible@JavaAccessBridge@@QEAAXPEAUJNIEnv_@@PEAV_jobject@@11@Z 0000000180022410     JavaAccessBridge.obj
 0002:0001042c       $unwind$?firePropertyCaretChange@JavaAccessBridge@@QEAAXPEAUJNIEnv_@@PEAV_jobject@@11JJ@Z 000000018002242c     JavaAccessBridge.obj
 0002:00010448       $unwind$?firePropertyDescriptionChange@JavaAccessBridge@@QEAAXPEAUJNIEnv_@@PEAV_jobject@@11PEAV_jstring@@2@Z 0000000180022448     JavaAccessBridge.obj
 0002:00010448       $unwind$?firePropertyNameChange@JavaAccessBridge@@QEAAXPEAUJNIEnv_@@PEAV_jobject@@11PEAV_jstring@@2@Z 0000000180022448     JavaAccessBridge.obj
 0002:00010448       $unwind$?firePropertyStateChange@JavaAccessBridge@@QEAAXPEAUJNIEnv_@@PEAV_jobject@@11PEAV_jstring@@2@Z 0000000180022448     JavaAccessBridge.obj
 0002:00010448       $unwind$?firePropertyTableModelChange@JavaAccessBridge@@QEAAXPEAUJNIEnv_@@PEAV_jobject@@11PEAV_jstring@@2@Z 0000000180022448     JavaAccessBridge.obj
 0002:00010448       $unwind$?firePropertyValueChange@JavaAccessBridge@@QEAAXPEAUJNIEnv_@@PEAV_jobject@@11PEAV_jstring@@2@Z 0000000180022448     JavaAccessBridge.obj
 0002:00010468       $unwind$?firePropertySelectionChange@JavaAccessBridge@@QEAAXPEAUJNIEnv_@@PEAV_jobject@@11@Z 0000000180022468     JavaAccessBridge.obj
 0002:00010468       $unwind$?firePropertyTextChange@JavaAccessBridge@@QEAAXPEAUJNIEnv_@@PEAV_jobject@@11@Z 0000000180022468     JavaAccessBridge.obj
 0002:00010468       $unwind$?firePropertyVisibleDataChange@JavaAccessBridge@@QEAAXPEAUJNIEnv_@@PEAV_jobject@@11@Z 0000000180022468     JavaAccessBridge.obj
 0002:00010480       $unwind$?firePropertyActiveDescendentChange@JavaAccessBridge@@QEAAXPEAUJNIEnv_@@PEAV_jobject@@1111@Z 0000000180022480     JavaAccessBridge.obj
 0002:00010480       $unwind$?firePropertyChildChange@JavaAccessBridge@@QEAAXPEAUJNIEnv_@@PEAV_jobject@@1111@Z 0000000180022480     JavaAccessBridge.obj
 0002:0001049c       $unwind$Java_com_sun_java_accessibility_internal_AccessBridge_jawtGetComponentFromNativeWindowHandle 000000018002249c     JavaAccessBridge.obj
 0002:0001049c       $unwind$Java_com_sun_java_accessibility_internal_AccessBridge_jawtGetNativeWindowHandleFromComponent 000000018002249c     JavaAccessBridge.obj
 0002:000104a8       $unwind$Java_com_sun_java_accessibility_internal_AccessBridge_propertyActiveDescendentChange 00000001800224a8     JavaAccessBridge.obj
 0002:000104a8       $unwind$Java_com_sun_java_accessibility_internal_AccessBridge_propertyCaretChange 00000001800224a8     JavaAccessBridge.obj
 0002:000104a8       $unwind$Java_com_sun_java_accessibility_internal_AccessBridge_propertyChildChange 00000001800224a8     JavaAccessBridge.obj
 0002:000104a8       $unwind$Java_com_sun_java_accessibility_internal_AccessBridge_propertyDescriptionChange 00000001800224a8     JavaAccessBridge.obj
 0002:000104a8       $unwind$Java_com_sun_java_accessibility_internal_AccessBridge_propertyNameChange 00000001800224a8     JavaAccessBridge.obj
 0002:000104a8       $unwind$Java_com_sun_java_accessibility_internal_AccessBridge_propertyStateChange 00000001800224a8     JavaAccessBridge.obj
 0002:000104a8       $unwind$Java_com_sun_java_accessibility_internal_AccessBridge_propertyTableModelChange 00000001800224a8     JavaAccessBridge.obj
 0002:000104a8       $unwind$Java_com_sun_java_accessibility_internal_AccessBridge_propertyValueChange 00000001800224a8     JavaAccessBridge.obj
 0002:000104a8       $unwind$?__scrt_throw_std_bad_alloc@@YAXXZ 00000001800224a8     MSVCRT:throw_bad_alloc.obj
 0002:000104a8       $unwind$?__scrt_throw_std_bad_array_new_length@@YAXXZ 00000001800224a8     MSVCRT:throw_bad_alloc.obj
 0002:000104b0       $unwind$Java_com_sun_java_accessibility_internal_AccessBridge_caretUpdate 00000001800224b0     JavaAccessBridge.obj
 0002:000104b0       $unwind$Java_com_sun_java_accessibility_internal_AccessBridge_focusGained 00000001800224b0     JavaAccessBridge.obj
 0002:000104b0       $unwind$Java_com_sun_java_accessibility_internal_AccessBridge_focusLost 00000001800224b0     JavaAccessBridge.obj
 0002:000104b0       $unwind$Java_com_sun_java_accessibility_internal_AccessBridge_menuCanceled 00000001800224b0     JavaAccessBridge.obj
 0002:000104b0       $unwind$Java_com_sun_java_accessibility_internal_AccessBridge_menuDeselected 00000001800224b0     JavaAccessBridge.obj
 0002:000104b0       $unwind$Java_com_sun_java_accessibility_internal_AccessBridge_menuSelected 00000001800224b0     JavaAccessBridge.obj
 0002:000104b0       $unwind$Java_com_sun_java_accessibility_internal_AccessBridge_mouseClicked 00000001800224b0     JavaAccessBridge.obj
 0002:000104b0       $unwind$Java_com_sun_java_accessibility_internal_AccessBridge_mouseEntered 00000001800224b0     JavaAccessBridge.obj
 0002:000104b0       $unwind$Java_com_sun_java_accessibility_internal_AccessBridge_mouseExited 00000001800224b0     JavaAccessBridge.obj
 0002:000104b0       $unwind$Java_com_sun_java_accessibility_internal_AccessBridge_mousePressed 00000001800224b0     JavaAccessBridge.obj
 0002:000104b0       $unwind$Java_com_sun_java_accessibility_internal_AccessBridge_mouseReleased 00000001800224b0     JavaAccessBridge.obj
 0002:000104b0       $unwind$Java_com_sun_java_accessibility_internal_AccessBridge_popupMenuCanceled 00000001800224b0     JavaAccessBridge.obj
 0002:000104b0       $unwind$Java_com_sun_java_accessibility_internal_AccessBridge_popupMenuWillBecomeInvisible 00000001800224b0     JavaAccessBridge.obj
 0002:000104b0       $unwind$Java_com_sun_java_accessibility_internal_AccessBridge_popupMenuWillBecomeVisible 00000001800224b0     JavaAccessBridge.obj
 0002:000104b0       $unwind$Java_com_sun_java_accessibility_internal_AccessBridge_propertySelectionChange 00000001800224b0     JavaAccessBridge.obj
 0002:000104b0       $unwind$Java_com_sun_java_accessibility_internal_AccessBridge_propertyTextChange 00000001800224b0     JavaAccessBridge.obj
 0002:000104b0       $unwind$Java_com_sun_java_accessibility_internal_AccessBridge_propertyVisibleDataChange 00000001800224b0     JavaAccessBridge.obj
 0002:000104b8       $unwind$__GSHandlerCheckCommon 00000001800224b8     MSVCRT:gshandler.obj
 0002:000104c0       $xdatasym                  00000001800224c0     MSVCRT:amdsecgs.obj
 0002:000104c4       $unwind$?dllmain_crt_process_attach@@YAHQEAUHINSTANCE__@@QEAX@Z 00000001800224c4     MSVCRT:dll_dllmain.obj
 0002:00010500       $unwind$?fin$0@?0??dllmain_crt_process_attach@@YAHQEAUHINSTANCE__@@QEAX@Z@4HA 0000000180022500     MSVCRT:dll_dllmain.obj
 0002:00010500       $unwind$?fin$0@?0??dllmain_crt_process_detach@@YAH_N@Z@4HA 0000000180022500     MSVCRT:dll_dllmain.obj
 0002:00010500       $unwind$?fin$1@?0??dllmain_crt_process_detach@@YAH_N@Z@4HA 0000000180022500     MSVCRT:dll_dllmain.obj
 0002:00010508       $unwind$?dllmain_crt_process_detach@@YAH_N@Z 0000000180022508     MSVCRT:dll_dllmain.obj
 0002:0001055c       $unwind$?dllmain_dispatch@@YAHQEAUHINSTANCE__@@KQEAX@Z 000000018002255c     MSVCRT:dll_dllmain.obj
 0002:00010584       $unwind$?filt$0@?0??dllmain_dispatch@@YAHQEAUHINSTANCE__@@KQEAX@Z@4HA 0000000180022584     MSVCRT:dll_dllmain.obj
 0002:0001058c       $unwind$__report_gsfailure 000000018002258c     MSVCRT:gs_report.obj
 0002:00010594       $unwind$capture_previous_context 0000000180022594     MSVCRT:gs_report.obj
 0002:000105a0       $unwind$__security_init_cookie 00000001800225a0     MSVCRT:gs_support.obj
 0002:000105ac       $unwind$__scrt_is_nonwritable_in_current_image 00000001800225ac     MSVCRT:utility.obj
 0002:000105cc       $unwind$__scrt_is_nonwritable_in_current_image$filt$0 00000001800225cc     MSVCRT:utility.obj
 0002:000105d4       $unwind$__scrt_fastfail    00000001800225d4     MSVCRT:utility_desktop.obj
 0002:000105e4       $unwind$__isa_available_init 00000001800225e4     MSVCRT:cpu_disp.obj
 0002:000105f8       $xdatasym                  00000001800225f8     MSVCRT:guard_dispatch.obj
 0002:00010600       $xdatasym                  0000000180022600     MSVCRT:guard_xfg_dispatch.obj
 0002:00010700       .edata                     0000000180022700     javaaccessbridge.exp
 0002:00010728       rgpv                       0000000180022728     javaaccessbridge.exp
 0002:000107a0       rgszName                   00000001800227a0     javaaccessbridge.exp
 0002:00010818       rgwOrd                     0000000180022818     javaaccessbridge.exp
 0002:00010854       szName                     0000000180022854     javaaccessbridge.exp
 0002:00010869       $N00001                    0000000180022869     javaaccessbridge.exp
 0002:000108ab       $N00002                    00000001800228ab     javaaccessbridge.exp
 0002:000108ed       $N00003                    00000001800228ed     javaaccessbridge.exp
 0002:0001092d       $N00004                    000000018002292d     javaaccessbridge.exp
 0002:00010970       $N00005                    0000000180022970     javaaccessbridge.exp
 0002:000109cd       $N00006                    00000001800229cd     javaaccessbridge.exp
 0002:00010a2a       $N00007                    0000000180022a2a     javaaccessbridge.exp
 0002:00010a6d       $N00008                    0000000180022a6d     javaaccessbridge.exp
 0002:00010ab2       $N00009                    0000000180022ab2     javaaccessbridge.exp
 0002:00010af5       $N00010                    0000000180022af5     javaaccessbridge.exp
 0002:00010b38       $N00011                    0000000180022b38     javaaccessbridge.exp
 0002:00010b7b       $N00012                    0000000180022b7b     javaaccessbridge.exp
 0002:00010bbd       $N00013                    0000000180022bbd     javaaccessbridge.exp
 0002:00010c00       $N00014                    0000000180022c00     javaaccessbridge.exp
 0002:00010c44       $N00015                    0000000180022c44     javaaccessbridge.exp
 0002:00010c8c       $N00016                    0000000180022c8c     javaaccessbridge.exp
 0002:00010cdf       $N00017                    0000000180022cdf     javaaccessbridge.exp
 0002:00010d30       $N00018                    0000000180022d30     javaaccessbridge.exp
 0002:00010d85       $N00019                    0000000180022d85     javaaccessbridge.exp
 0002:00010dcf       $N00020                    0000000180022dcf     javaaccessbridge.exp
 0002:00010e19       $N00021                    0000000180022e19     javaaccessbridge.exp
 0002:00010e69       $N00022                    0000000180022e69     javaaccessbridge.exp
 0002:00010eb2       $N00023                    0000000180022eb2     javaaccessbridge.exp
 0002:00010f00       $N00024                    0000000180022f00     javaaccessbridge.exp
 0002:00010f4a       $N00025                    0000000180022f4a     javaaccessbridge.exp
 0002:00010f99       $N00026                    0000000180022f99     javaaccessbridge.exp
 0002:00010fe2       $N00027                    0000000180022fe2     javaaccessbridge.exp
 0002:0001102c       $N00028                    000000018002302c     javaaccessbridge.exp
 0002:0001107c       $N00029                    000000018002307c     javaaccessbridge.exp
 0002:000110b9       $N00030                    00000001800230b9     javaaccessbridge.exp
 0002:000114fa       .idata$6                   00000001800234fa     kernel32:KERNEL32.dll
 0002:000115b6       .idata$6                   00000001800235b6     user32:USER32.dll
 0002:000115d0       .idata$6                   00000001800235d0     jawt:jawt.dll
 0002:0001166e       .idata$6                   000000018002366e     vcruntime:VCRUNTIME140.dll
 0002:00011800       .idata$6                   0000000180023800     ucrt:api-ms-win-crt-string-l1-1-0.dll
 0002:00011822       .idata$6                   0000000180023822     ucrt:api-ms-win-crt-runtime-l1-1-0.dll
 0002:00011844       .idata$6                   0000000180023844     ucrt:api-ms-win-crt-stdio-l1-1-0.dll
 0002:00011864       .idata$6                   0000000180023864     ucrt:api-ms-win-crt-environment-l1-1-0.dll
 0002:0001188a       .idata$6                   000000018002388a     ucrt:api-ms-win-crt-heap-l1-1-0.dll
 0003:000000f0       logFP                      00000001800240f0     AccessBridgeDebug.obj
 0003:00000138       ?__proc_attached@@3HA      0000000180024138     MSVCRT:dll_dllmain.obj
 0003:00000140       GS_ExceptionRecord         0000000180024140     MSVCRT:gs_report.obj
 0003:000001e0       GS_ContextRecord           00000001800241e0     MSVCRT:gs_report.obj
 0003:000006d8       ?is_initialized_as_dll@@3_NA 00000001800246d8     MSVCRT:utility.obj
 0003:000006d9       ?module_local_atexit_table_initialized@@3_NA 00000001800246d9     MSVCRT:utility.obj
 0003:000006e0       ?module_local_atexit_table@@3U_onexit_table_t@@A 00000001800246e0     MSVCRT:utility.obj
 0003:000006f8       ?module_local_at_quick_exit_table@@3U_onexit_table_t@@A 00000001800246f8     MSVCRT:utility.obj
 0005:00000120       $R000000                   0000000180026120     javaaccessbridge.dll.res
 0005:00000338       $R000218                   0000000180026338     javaaccessbridge.dll.res
 0005:000003c8       $R0002A8                   00000001800263c8     javaaccessbridge.dll.res
